:020000040802F0
:1000000010E300204901020821300208952B020864
:100010001D300208951E02084FA2020800000000D1
:10002000000000000000000000000000458A0208F7
:10003000052102080000000093010208519C0208FB
:100040006701020867010208670102084575020896
:100050006701020867010208412102080122020823
:1000600067010208670102086701020867010208C8
:100070006701020867010208511F020867010208B0
:1000800067010208A91F0208670102086701020848
:10009000650102086701020867010208452202089B
:1000A0006701020867010208670102086701020888
:1000B000670102083D9D0208FD9D020867010208D4
:1000C0006701020867010208670102086701020868
:1000D000670102083DA0020847A0020851A00208DB
:1000E000852102086701020867010208670102080A
:1000F0006701020867010208670102086701020838
:100100006701020867010208670102086701020827
:10011000DD9F0208E79F02086701020867010208E5
:100120006701020867010208670102086701020807
:10013000DFF810D000F042FF00480047E1F9020864
:10014000AFF3008010E300200748804707480047CE
:10015000FEE7FEE7FEE7FEE7FEE7FEE7FEE7FEE777
:10016000FEE7FEE7FEE7FEE7E99C02083101020830
:1001700018484FF0FF010170002080F309881648ED
:10018000016881F3088815484FF08051016062B61C
:10019000FEE772B6EFF3098028B1203880E8F00F4F
:1001A0000F490968086000B50E4880475DF804EB08
:1001B0000D480E490A78027009480D490A68026024
:1001C000106890E8F00F203080F309884EF0040E9C
:1001D00062B6704722ED00E0A803002004ED00E0C5
:1001E000A0030020914702084003002041030020A3
:1001F000A403002072B6704762B67047EFF3108018
:1002000072B6704780F310887047B0FA80F070477C
:1002100090FAA0F0704730BF704720BF70472DE9BB
:10022000F05F0546002092469B468846064681467A
:1002300040241BE0284641464746224600F021FD67
:1002400053465A46C01A914110D3114618462246C9
:1002500000F008FD2D1A67EB01084F4622460120E9
:10026000002100F0FFFC17EB00094E41201EA4F115
:100270000104DFDC484631462A464346BDE8F09F8C
:1002800000487047FC3E030810B50446FFF7F8FF2E
:100290000068005D00F0010010BD2DE9FE439946A5
:1002A00015468846074601AC022942D3002D40D0AE
:1002B00000200290A8F101004FF0FF36009022E0EC
:1002C00000FB057201FB057011464A469047002865
:1002D00005DC54F82600304444F8260013E060683A
:1002E0002A4600FB057154F8040C00FB057007E07A
:1002F0000B7890F800C001F801CB00F8013B521ECA
:10030000002AF5D1764254F8040C61688842D7DCA3
:100310004B462A463846FFF7C0FF54F8040C4B46BC
:10032000A8EB0001401C00FB05702A46491EFFF7A0
:10033000B4FFBDE8FE8300000649074A0868504341
:1003400043F23902104408604008704701490860D0
:1003500070470000B00300206D4EC64140EA010323
:100360009B0703D009E008C9121F08C0042AFAD26B
:1003700003E011F8013B00F8013B521EF9D270472F
:10038000D2B201E000F8012B491EFBD270470022D7
:10039000F6E710B513460A4604461946FFF7F0FF84
:1003A000204610BD421E12F8013F002BFBD111F870
:1003B000013B02F8013B002BF9D1704730B50546EF
:1003C0002A460B4612F8010B13F8014B08B1A04264
:1003D000F8D01CB1002802D06D1CF1E7284630BDD2
:1003E000421C10F8011B0029FBD1801A70470346FC
:1003F00011F8012B00F8012B002AF9D1184670479B
:100400000FB400B58DB010A909900B9000914FF07A
:10041000FF300A9000200C90054806900548079090
:100420006A4609A80F9900F063FC0DB05DF814FB53
:100430000D0D02082B0D02082DE9FF5F1D464FF040
:10044000FF3BD5E9014691465F464FF00008A96998
:100450007F1C01988847296A824688470028F6D180
:10046000BAF1FF3F0CD024F4C064002E19DD600601
:1004700014D5BAF12B0F09D0BAF12D0F0ED103E02C
:10048000584604B0BDE8F09F44F48064A9697F1C1D
:1004900001988847761E8246002E02DDBAF1300FA1
:1004A00003D0B9F1000F26D032E0A969761E44F4DA
:1004B00000747F1C019888478246002E05DDBAF142
:1004C000780F06D0BAF1580F03D0B9F1000F10D051
:1004D0001EE0B9F1000F02D0B9F1100F18D1A969CF
:1004E000761E24F400747F1C0198884782461020F1
:1004F00002E0082000E00A20814609E008FB090824
:10050000A969761E44F400747F1C019888478246CE
:10051000002E05DD4946504600F0D5FB0028EDDAF7
:10052000E96901988847A00502D46FF00100A8E7A7
:10053000E00725D1600613D5600502D5C8F100009B
:1005400000E0404629680A1D2A600968220501D595
:10055000087015E0220701D5088011E008600FE05F
:100560002868011D29600068210502D580F80080F7
:1005700006E0210702D5A0F8008001E0C0F8008065
:1005800038467EE72DE9FF5FD2E901A74FF000086A
:10059000916999461446DDF838B046460198884777
:1005A000054659EA0B0005D009E0A169761C0198BF
:1005B00088470546216A284688470028F5D1681CE7
:1005C00003D05FEACA7005D015E04FF0FF3004B0E9
:1005D000BDE8F09F2068011D2160D0F800800AE08E
:1005E0005FEACA7001D108F8015BA169761C7F1E21
:1005F000019888470546002F1ADD681C18D0B9F10C
:10060000000F0DD0E81705EBD060421120F01F005D
:1006100059F822102A1A012090400142E0D107E047
:10062000BBF1000FDCD1216A284688470028D7D0CB
:10063000E16901988847BBF1000F07D1002E05DD65
:100640005FEACA7002D1002188F80010A068B842A1
:1006500003DDBBF1000F03D017B16FF00100B6E767
:100660003046B4E770B5064609F048FE0468054612
:100670000A220021304600F069FB2C6070BDF0B406
:1006800080EA0102D40F4200B2EB410F02D20246CF
:10069000084611464A0042D0C30DDDB2C1F3C7522D
:1006A000AD1A202D35DAC1F3160141F4000204B170
:1006B0005242C5F1200602FA06F12A411044B3EB7A
:1006C000D05F23D0C4B1012DA0EBC35009DCF0BC36
:1006D0004FF0004202EAC352DBB200F5000000F026
:1006E00086BB400000F1807000EBC350A0F1807029
:1006F00040EAD170490009E0490841EAC071A0EB25
:10070000C35000F50000400800EBC350F0BC00F0FF
:1007100065BB6142012202EB4101001BF6E7F0BC20
:10072000704781F00041AAE780F00040A7E780EA27
:10073000010210B502F00043400022D04A001FD051
:10074000010E01EB1261C0F35600C2F3560240F4F1
:10075000000042F40002A0FB022000047F391404D0
:1007600000D0401C50EA124001D44000491EC2B2E1
:100770000C0604EBD010401C4008802A02D003E095
:10078000002010BD20F00100002900DA00201843ED
:1007900010BD30B480EA010202F0004530F00042A2
:1007A00021F0004013D090B1C30DD40DC2F3160157
:1007B000C0F31600E41A41F4000140F400027D3455
:1007C000914201D3641C00E04900002C02DA30BCE5
:1007D000002070474FF400000023914201D3891A92
:1007E000034340084FEA4101F7D151B1914202D190
:1007F0004FF0004105E002D24FF0010101E06FF03F
:10080000010103EBC450284430BC00F0E7BA2DE9E5
:10081000FE4F804681EA0300C00F0C46009021F095
:10082000004123F00045B8EB0200A94105D2404643
:10083000214690461C460B46024623F000401043DA
:1008400047D0270DC7F30A00C3F30A510290401A9C
:10085000019040286BDAC3F3130040F4801B00982A
:10086000924620B10023D2EB030A63EB0B0B0198F5
:100870005946C0F14002504600F0F4F906460D46D4
:1008800050465946019A00F00CFA10EB08006141FD
:10089000002487EA115284EAE7731A4340D0009A91
:1008A00062B3019A012A4FEA075215DC001B61EB83
:1008B00002014FF0004202EA0752CDE90042001C5B
:1008C00041F5801132462B4600F0CEFA03B0BDE868
:1008D000F08F40462146F9E7001B61EB0201001C46
:1008E00041F5801300185B412018A2F5001747EB73
:1008F000030140EAD570B6196D4111E06D084FEA69
:10090000360645EAC0754FEA0752001B61EB02014B
:10091000001C41F5801149084FEA3000001951418F
:1009200032462B4603B0BDE8F04F00F08EBA009877
:10093000012240000023D0EB020263EBE073009839
:1009400021464FEAE074B8EB000061EB0401E9E7EF
:1009500083F000435BE781F0004158E72DE9FE4F4B
:1009600081EA030404F0004421F0004100944FF0B8
:10097000000B23F0004350EA01045ED052EA030466
:100980005BD0C3F30A54C1F30A552C44A4F2F334E8
:100990000194A0FB0254C1F3130141F48011C3F38D
:1009A000130343F4801301FB024400FB034E840A4B
:1009B000970A44EA815447EA8357A4FB07680295E3
:1009C0008D0A05FB07854FEA932C04FB0C54270581
:1009D000029D4FEA065847EA1637B5EB08056EEB5D
:1009E000070C870E920E47EA811742EA8312A7FB93
:1009F0000201B6EB0B0164EB00042B0D43EA0C3350
:100A00005E1844EB1C50DA465146E7FB0201C5F381
:100A100013044FEA0B3343EA14534FEA0432019CA8
:100A200043EA0603A4F10C040294009CCDE900B44F
:100A300000F01AFA03B0BDE8F08F00200146F9E794
:100A40002DE9F04D81EA030404F0004B21F000454C
:100A500014464FF0000A23F0004150EA050220D06E
:100A600054EA01021DD0C5F30A570246C5F3130329
:100A7000C1F31300C1F30A5640F4801543F4801308
:100A8000A7EB0608101BD64608F2FD3873EB0500ED
:100A900002D308F1010801E092185B41B8F1000FA0
:100AA00003DA00200146BDE8F08D00204FF48011EC
:100AB000064684460EE0171B73EB050705D3121B91
:100AC00063EB050306434CEA010C49084FEA30008A
:100AD00092185B4150EA0107EDD152EA030012D0AF
:100AE00082EA040083EA0501084305D0101BAB41EC
:100AF00006D20122002306E000224FF0004302E06C
:100B00006FF0010253101AEB06004CEB085110EB8A
:100B10000A0041EB0B01BDE8F04D00F096B9C10FA2
:100B200080EAE0700844CA079623002100F05FB90C
:100B300096230022114600F05AB90EB5C10F80EA83
:100B4000E0700844CA07002140F233438DE80E00EC
:100B50000A460B4600F088F903B000BD0EB540F21E
:100B6000334102910021CDE900110A460B4600F005
:100B70007BF903B000BDC1F30A5210B5C1F31301F4
:100B800040F2FF3341F480119A4201DA002010BD97
:100B900040F233439A42A2F2334203DC524200F065
:100BA00070F810BD904010BD00F0004230F00040E1
:100BB0000AD0C10D01F56071C0F3160042EA01517F
:100BC000C2084007114370470020014670470000EB
:100BD00030B5041E71F1000404DB4FF000444042C4
:100BE00064EB0101141E73F1000405DB1C464FF099
:100BF0000043524263EB0403994208BF904230BD68
:100C000001F0004330B421F0004150EA010206D067
:100C10000A0DA2F56072C1F31301002A02DC30BC98
:100C200000207047440F44EAC104C100E01830BC02
:100C300000EBC25000F0D2B830B50B4601460020A0
:100C40002022012409E021FA02F59D4205D303FA8E
:100C500002F5491B04FA02F52844151EA2F101020F
:100C6000F1DC30BD202A04DB203A00FA02F100203A
:100C700070479140C2F1200320FA03F319439040DA
:100C80007047202A04DB203A21FA02F00021704745
:100C900021FA02F3D040C2F12002914008431946E4
:100CA0007047202A06DBCB17203A41FA02F043EACC
:100CB000E07306E041FA02F3D040C2F12002914015
:100CC0000843194670473A2800D2303820F02002F5
:100CD000412A01D3A2F13700884201D34FF0FF30FF
:100CE000704700000268114413780160184670478D
:100CF000D16004495161044911620021116111461A
:100D000000F06EB9E50C020889020208426842B19F
:100D1000016811F8013B23B1521EC0E900121846C8
:100D200070470121C160881E704742685AB1C3688C
:100D3000016843B983688B4205D0491E521CC0E943
:100D40000012002070474FF0FF3070472DE9F04748
:100D500091460E4680460446002514F8017B2FB1CB
:100D6000FFF78EFA0068C05DC007F6D12B2F02D0C6
:100D70002D2F1ED0641E4A463146204600F0C8FA88
:100D800026B13268A24201D1C6F800806A054FF050
:100D9000020418D50023D0EB030563EB01025D1BB1
:100DA000934109DB0023D0EB030063EB0101BDE8B5
:100DB000F08745F48065DEE709F0A0FA04600020C2
:100DC0004FF00041F3E7021E71F10002EFDA09F083
:100DD00095FA04604FF0FF304108E8E70029A8BF0A
:100DE0007047401C490008BF20F00100704710B454
:100DF000B0FA80FC00FA0CF050EA010404BF10BC09
:100E0000704749B1CCF1200421FA04F411FA0CF135
:100E100018BF012121430843A3EB0C01CB1D4FEA6E
:100E200000614FEA102042BF002010BC704700EB69
:100E3000C35010440029A4BF10BC7047401C490097
:100E400008BF20F0010010BC704710B5141E73F1EC
:100E5000000408DA401C41F1000192185B411A437A
:100E600001D120F0010010BD2DE9F04D92469B46C6
:100E700011B1B1FA81F202E0B0FA80F2203290466C
:100E8000FFF7F0FE04460F4640EA0A0041EA0B0174
:100E900053465A46084313D0114653EA010019D06D
:100EA000C8F140025046FFF7ECFE05460E4650469C
:100EB00059464246FFF7D6FE084305D0012004E01C
:100EC00020463946BDE8F08D0020054346EAE0762D
:100ED0002C4337430A986305E40AA0EB080000227C
:100EE000FD0A44EA47540A3002D500200146E9E7EA
:100EF000010510196941DDE9084500196941BDE89E
:100F0000F04DA2E72DE9F041054621F000400C46E6
:100F1000284309D0C4F30A5040F23341884205DD2A
:100F200028462146BDE8F0812846FBE740F2FE3125
:100F3000884210DC0CDB4FEA043040EA155050EADE
:100F4000053105D0104804F0004101430020E9E7D5
:100F500000200146E6E7A0F233404642C6F14002D7
:100F600028462146FFF77EFE07468846284621464A
:100F70003246FFF786FE43463A46FFF766FF3246A3
:100F8000BDE8F041FFF76EBE0000F03FC1F30A522A
:100F9000C1F3130140F2FF3341F480119A4202DAA7
:100FA00000200146704740F233439A42A2F2334296
:100FB00002DC5242FFF765BEFFF754BE064C074DF8
:100FC00006E0E06840F0010394E807009847103419
:100FD000AC42F6D3FFF7B0F8943F0308B43F0308E0
:100FE0002DE9F34F8BB04FF0000801F10C000C46D7
:100FF0004FF0010B46460DF1080A0190626901218C
:1010000001989047051E2DD0252D2CD0216A8847A8
:10101000C0B16269012101989047216A8847002880
:10102000F7D1411E62690198904700E0761CA169E2
:101030000B988847216A88470028F7D1E1690B9807
:101040008847DBE7A1690B9888470746A84201D18A
:10105000761CD3E7E1690B9888477F1C02D1B8F171
:10106000000F6FD047E1002762693D46394601987D
:1010700090472A2804D162690121019890470125EF
:10108000DFF888926269012101989047A0F1300150
:101090000A290AD24F45E5DC07EB870100EB41073F
:1010A000303FDFD445F01005ECE7E90601D46FF0DE
:1010B00000476C280AD04C2814D0682815D06A281C
:1010C0000DD074281CD07A281AD01DE06269012145
:1010D000019890476C2802D045F0040514E045F0D3
:1010E00002050DE045F020050AE062690121019842
:1010F0009047682802D045F0080505E045F40065F2
:101100006269012101989047C4E9015765283DD0E3
:1011100019DC58287AD00CDC452837D004DC252887
:1011200026D0412831D131E046282FD047282CD174
:101130002CE05B2877D0612828D063287CD06428F5
:1011400023D15AE0D1E06F2848D008DC66281DD0B2
:1011500067281BD0692821D06E2816D127E0702877
:1011600045D0732868D0752847D078280DD14DE038
:10117000A1690B988847054625283FF469AFE169C6
:101180000B9888476D1C3FF46AAFB4E023466A466B
:101190006FF001000B99AFF300809FE045F0400035
:1011A0006060A80723464FF0000236D43EE0E8070F
:1011B0007FF447AF2068011D21600068290501D533
:1011C00006701BE7290701D5068017E7A90703D595
:1011D000F117C0E9006111E706600FE745F0400034
:1011E0006060A80723464FF0080216D41EE040F6C0
:1011F0000E0125EA0100606016E045F040006060E5
:10120000A80723464FF00A0207D40FE045F040003C
:101210006060A80708D5234610226FF001000B99E3
:10122000AFF300805AE007E0234610226FF0010080
:101230000B99FFF701F951E04FF000094F464B467B
:10124000632802D05B2807D041E02079C00601D492
:101250000120A06001273AE06269012101989047CE
:101260005E2805D14FF0010962694946019890470F
:10127000216939B900210A46534643F82120491C07
:101280000829FADBB0B3216969B9C11700EBD16253
:1012900053110AEB830122F01F02821A01200B680E
:1012A000904003430B6062690121019890475D28DB
:1012B000E8D1B9F1000F09D00020514651F82020A3
:1012C000D24341F82020401C0828F7DB02AB22461D
:1012D00000976FF001000B99FFF754F900280CDA22
:1012E000401C08D1BBF1000F05D04FF0FF300DB00E
:1012F000BDE8F08FFFE74046F9E7E90701D108F1C3
:10130000010806444FF0000B78E60000CCCCCC0C72
:101310002DE9F74F4FF00009009C1546CA4614F816
:10132000010B302801D0ADB115E014F8010B4FF0DE
:101330000109782803D0582801D04DB10BE00DB138
:10134000102D08D14FF00009102514F8010B02E010
:10135000082500E00A2500273E46B8464FEAE57B0F
:1013600016E0A5FB07230BFB073105FB080005FB77
:101370000616010C571846F100061FFA80F8381EB1
:101380004FF0010976F5803000D3CA4614F8010BFE
:101390002946FFF798FC0028E3DA019838B1B9F143
:1013A000000F01D0641E00E0009C01980460BAF1B7
:1013B000000F08D008F0A2FF02210160C81E0146FC
:1013C00003B0BDE8F08F310441EA174148EA074015
:1013D000F6E770B58C1810F8015B15F0070301D122
:1013E00010F8013B2A1106D110F8012B03E010F888
:1013F000016B01F8016B5B1EF9D12B0705D40023AB
:10140000521E0DD401F8013BFAE710F8013BCB1A4C
:10141000921C03E013F8015B01F8015B521EF9D541
:10142000A142D8D3002070BD21B1826842F00102F0
:10143000826003E0826822F001028260704700004F
:1014400010B504461248844208D10121401505F028
:10145000B5FE0021601505F0B1FE17E00D4884428D
:1014600008D10121001505F0A9FE0021201505F085
:10147000A5FE0BE00848844208D10121C80305F00D
:101480009DFE00214FF4004005F098FE10BD0000C5
:101490000024014000280140003C0140014600209A
:1014A0008A6802F004020AB1012000E000207047BF
:1014B0000146C86C80B270470246002013680B409A
:1014C0000BB1012000E000207047014600208A682F
:1014D00002F008020AB1012000E00020704700007D
:1014E00030B502460020002350680F4C20400D7993
:1014F0000C6844EA05242043506090680B4C20405F
:10150000D1E902542C434D7944EA450420439060CC
:10151000D06A20F470000C7C641EE4B2234340EADD
:101520000350D06230BD0000FFFEF0FFFDF7F1FF79
:10153000F0B504460D4600200021092D11DDE068BC
:10154000A5F10A0606EB4607072606FA07F18843C7
:10155000A5F10A0606EB460603FA06F10843E06029
:101560000CE0206905EB4507072606FA07F18843DA
:1015700005EB450603FA06F108432061072A0FDA56
:10158000606B561E06EB86071F2606FA07F1884396
:10159000561E06EB860605FA06F10843606322E054
:1015A0000D2A0FDA206BD61F06EB86071F2606FAD8
:1015B00007F18843D61F06EB860605FA06F10843B5
:1015C000206310E0E06AA2F10D0606EB86071F26F5
:1015D00006FA07F18843A2F10D0606EB860605FA26
:1015E00006F10843E062F0BD816841F008018160C6
:1015F000704721B1826842F4A002826003E08268F1
:1016000022F4A00282607047816841F00401816089
:101610007047000030B10749096841F40001054AEC
:10162000116005E00349096821F40001014A1160D5
:1016300070470000082401400EB501210A4800F05F
:101640000DFD0021094800F009FD02A800214FF41A
:10165000FA730A46CDE90010084603F053F9002159
:10166000FF200DF0D7F80EBD30310102131320001A
:101670002DE9F84F04460F469046B8F1000F01D10E
:10168000BDE8F88F45463DE004F03F0ACAF1400A44
:10169000AA4501DB2E4600E05646A81B85B2B1469E
:1016A000C4F3072BE0B2009001F08AFBA02001F008
:1016B00053FB01F0DBFB584601F04EFB01F0D6FB7B
:1016C000009801F049FB01F0D1FB04200AF0ABFACD
:1016D00001F076FBA12001F03FFB01F0C7FB06E023
:1016E000012001F001FB38707F1C701E86B2002EB5
:1016F000F6D1002001F0F8FA01F088FB04200AF08E
:1017000092FA4C44002DBFD100BFB9E72DE9FF5F2D
:1017100004460E46174620212A4801F0B0F80FB9BA
:10172000BDE8FF9F3D463BE004F03F0ACAF1400A96
:10173000AA4501DBA84600E0D046A5EB080085B22B
:10174000C146C4F3072BE0B2029001F039FBA020A0
:1017500001F002FB01F08AFB584601F0FDFA01F0AE
:1017600085FB029801F0F8FA01F080FB05E0307883
:1017700001F0F2FA01F07AFB761CB8F10000A8F152
:1017800001011FFA81F8F2D101F040FB03A800210A
:101790000A230A46CDE90010084603F0B3F84C448A
:1017A000002DC1D12021074801F06BF803A80021CA
:1017B0000A230A46CDE90010084603F0A3F800BF4B
:1017C000AEE70000000C014030B58BB0054600F0DC
:1017D00063FB00F00BFBA3A008F04AFD10F01EFD18
:1017E00001200FF07BF8A2A101200FF0DFF9A4483F
:1017F000A4A1026801200FF0D9F9A948D0F803206C
:10180000A8A101200FF0D2F9ACA101200FF0CEF970
:10181000AE48AFA1026801200FF0C8F9AB48B3A1F0
:10182000426801200FF0C2F9A848B7A182680120E0
:101830000FF0BCF9A548BBA1C26801200FF0B6F9B2
:10184000A248BFA1026901200FF0B0F9C3A1012095
:101850000FF0ACF9C6480278C6A101200FF0A6F936
:10186000C348B0F80520CAA101200FF09FF9C04875
:10187000D0F80130D0F80120CCA101200FF096F96A
:10188000D3A101200FF092F9002407E0D548025DB2
:10189000D5A101200FF08AF9601CC4B20C2CF5DB35
:1018A000D3A101200FF082F9B148C27BD1A1012060
:1018B0000FF07CF9AE48D0F80B20D5A101200FF035
:1018C00075F9AB48B0F80920D8A101200FF06EF9E6
:1018D000A748B0F80720DCA101200FF067F9C14844
:1018E0000838407F00F08000802803D1DDA008F098
:1018F000BFFC02E0DEA008F0BBFCBA480838407F1D
:10190000C0F3001018B1DDA008F0B2FC02E0DFA0C7
:1019100008F0AEFCE1A101200FF048F9E44802789C
:10192000E4A101200FF042F9FFF786FE0AA802F0B9
:10193000F1FA0AA8032100220592CDE906210890B8
:10194000104680210C22E14BCDE90132CDE9031094
:1019500006200023DE4ADFA10090E24802F03CFBB3
:101960000AA8032100220592CDE90621089010461D
:1019700080210C22DC4BCDE90132CDE9031002209D
:101980000023DA4ADAA10090DE4802F025FB0AA81B
:10199000032100220592CDE90621089010464FF45C
:1019A00080616622D84BCDE90132CDE903100520D4
:1019B0000023D64AD6A10090DA4802F00DFB0AA80F
:1019C000032100220592CDE90621089010464FF42C
:1019D00000713322D44BCDE90132CDE9031003204D
:1019E0000023D24AD2A10090D64802F0F5FA0AA804
:1019F000032100220592CDE90621089010464FF4FC
:101A000080616622D04BCDE90132CDE9031005207B
:101A10000023CE4ACEA10090D14802F0DDFAD14891
:101A20000078012817D10AA8032100220592CDE9E8
:101A30000621089010464FF400713322CA4BCDE9BD
:101A40000132CDE9031003200023C84AC8A1009049
:101A5000CC4802F0C1FA0AA9CB4802F0EDFB0BB06A
:101A600030BD000041505020626567696E0A000079
:101A70000AB8B4CEBBD0C5CFA2A3BA0A00000000FA
:101A8000D40100202072657365745F7479706520DD
:101A900020202020203D203078253032780A000098
:101AA000007400202072657365745F74696D6573DE
:101AB00020202020203D2025750A00000AC8EDBC0A
:101AC000FEB0E6B1BEA3BA0A000000000C7400200C
:101AD00020626F6F745F76657220202020202020A6
:101AE000203D203078253038780A00002070745F5F
:101AF000766572202020202020202020203D2030CC
:101B000078253038780A000020617070315F766582
:101B10007220202020202020203D203078253038C1
:101B2000780A000020617070325F76657220202094
:101B300020202020203D203078253038780A0000F1
:101B400020617070335F7665722020202020202075
:101B5000203D203078253038780A00000AC9E8B1E5
:101B6000B8B3F6B3A7D0C5CFA2A3BA0A000000004D
:101B7000DC0600202050545F696E6974202020200C
:101B800020202020203D203078253032780A0000A7
:101B9000206465766963655F747970652020202014
:101BA000203D203078253034780A000020646576A6
:101BB0006963655F736E202020202020203D202552
:101BC000303130752C203078253038780A0000000C
:101BD00020757569642020202020202020202020CE
:101BE000203D2000F406002025303278200000003F
:101BF0000D0A0000207063625F766572202020204D
:101C000020202020203D203078253032780A000026
:101C1000206465766963655F706420202020202041
:101C2000203D203078253038780A00002064657621
:101C30006963655F626E202020202020203D2030D7
:101C400078253034780A0000206465766963655F22
:101C50006D66727320202020203D2030782530349E
:101C6000780A0000D6A7B3D6BDE2C2EB0A00000096
:101C7000B2BBD6A7B3D6BDE2C2EB0A00B2E5C8EB51
:101C8000BCD3C3DCC4A3BFE90A000000CEB4B2E5F4
:101C9000C8EBBCD3C3DCC4A3BFE90A000A4C6F7213
:101CA00061B2CECAFDD0C5CFA2A3BA0A000000001F
:101CB000E8010020206C6F72615F696E64657820B6
:101CC00020202020203D2025640A0000203700200D
:101CD000A52F02084C4544205441534B2048616EC7
:101CE000646C650060360020E0390020F19F020836
:101CF00055415254205441534B2048616E646C65E9
:101D0000000000002039002020560020D92F0208B2
:101D10004C4F5241205441534B2048616E646C65D6
:101D20000000000060550020A03C0020FD7002086B
:101D300050524F47205441534B2048616E646C65AC
:101D400000000000E03B002060450020616F0208B9
:101D50004F5441205441534B2048616E646C6500E0
:101D6000A0440020F8000020E066002009210208BD
:101D7000454E434F444552205441534B2048616ED9
:101D8000646C650020660020C003002008B5014691
:101D900000200090034800900098084400900098AC
:101DA000008808BD006C004008B500220092044A7B
:101DB0000092009A02440092009A116008BD00004F
:101DC000006C004070B505460C4620460FF0D2FB73
:101DD000064631462846FFF7E7FF70BD00B585B0DF
:101DE000684605F005FA019805B000BD08B507F092
:101DF0007BFF07F047FF4FF4A06001F04BF905F0BF
:101E0000E9FB08F035FF0EF0BDFE00F0D9FD0BF048
:101E1000B3FF1E4908700CF0C1FB01F07FF80FF012
:101E2000DFFB0EF09DFE00231A464FF4E131184609
:101E300011F040FA4FF480639A004FF4E131012031
:101E400011F038FA00231A464FF4E131022011F064
:101E500031FA4FF480639A004FF41651032011F0C9
:101E600029FA4FF480639A004FF41651042011F0C0
:101E700021FA03201023022205490090042000F0DB
:101E8000E5FB0221024800F0FAFC08BDF800002042
:101E90000008014000BFFEE710B500F001F810BDDA
:101EA00010B500200249086000F00AF810BD0000DB
:101EB000AC0300200149086070470000AC0300201B
:101EC00010B5FFF78BFF04462046FFF7F3FF10BD68
:101ED00001480068704700002000002070B50246ED
:101EE0000B460020002111E0555C00BF6840002433
:101EF00009E000F0010626B140104AF201067040E8
:101F000000E04010641C082CF3D3491C9942EBD329
:101F100070BD000010B502460B46002100BF04E072
:101F200052F82100034C2060491C9942F8D3014823
:101F3000006810BD00300240014800687047000092
:101F400000300240012001498860704700300240A3
:101F500010B501F0E1F94FF4005000F069F80128E4
:101F600018D1002280210D4808F09BF800210C4870
:101F700000F052F84FF4005000F040F800BF40214C
:101F8000064808F097F80028F9D04FF4807105480A
:101F900000F075FC01F0D6F910BD000000380140DA
:101FA000440002400008014010B501F0B5F94FF0BF
:101FB000007000F03DF8012817D1002280210C4864
:101FC00008F06FF800210B4800F026F84FF0007081
:101FD00000F014F800BF4021054808F06BF8002815
:101FE000F9D00221044800F04AFC01F0ABF910BD21
:101FF00000440040800002400008014000F0805191
:1020000011B10349086001E00249486070470000CF
:10201000040402400000024021B1026842F00102C3
:10202000026004E002684FF6FE731A4002607047D7
:1020300001460020002201F0805313B1054B1A68BD
:1020400001E0054B1A6802EA01030BB1012000E030
:102050000020704700040240000002402DE9F041DA
:1020600005460E460027B84606B901E04FF00408C1
:1020700000240AE025FA04F000F00107394604EBD9
:102080000802D0B200F0C2FF641C042CF2DBBDE8F1
:10209000F08100002DE9F04707460D4690460026E6
:1020A000B146042D15DCB8F1000F00D101E04FF06E
:1020B000040900240AE027FA04F000F00106314682
:1020C00004EB0902D0B200F0A1FF641CAC42F2DBC9
:1020D00013E0082D11DC01210948FFF7BFFF0024A0
:1020E00008E027FA04F000F001063146E0B200F003
:1020F0008DFF641C281FA042F3DCBDE8F0870000C0
:1021000030310102704700000EB50AF0D3FA13E037
:102110000AF016FB0CF0A2F80AF0D2F80748006AA1
:10212000401C0649086202A800210A230A46CDE99C
:102130000010084602F0E6FBEAE70000B4060020C3
:1021400010B5012000F0B4F8C8B10D480078401C6B
:102150000B4908700846807838B901224EF6602194
:102160000748163010F0C8F806E001224EF660214C
:102170000348001D10F0C0F8012000F093F810BDD6
:102180003436002010B54FF4806000F091F830B183
:1021900004200AF09DFA4FF4806000F083F84FF4B9
:1021A000805000F085F830B101200AF091FA4FF428
:1021B000805000F077F84FF4005000F079F830B11B
:1021C00003200AF085FA4FF4005000F06BF84FF44A
:1021D000804000F06DF830B105200AF079FA4FF434
:1021E000804000F05FF84FF4004000F061F830B13B
:1021F00007200AF06DFA4FF4004000F053F810BDCC
:1022000010B5022000F054F8C8B10D484078401CC9
:102210000B4948700846C07838B901224EF6602153
:1022200007481F3010F068F806E001224EF66021E2
:1022300003480D3010F060F8022000F033F810BDB4
:102240003436002010B54FF4807000F031F828B11A
:10225000012013490870000200F024F8402000F02B
:1022600027F828B100200AF033FA402000F01AF8CD
:10227000802000F01DF828B102200AF029FA802001
:1022800000F010F84FF4007000F012F830B10620A2
:102290000AF01EFA4FF4007000F004F810BD0000C0
:1022A000B501002001490860704700001404014096
:1022B000014600200022074B1B6803EA0102054B80
:1022C00014331B680B4013B10AB1012000E0002059
:1022D0007047000000040140002123498279002A50
:1022E0003AD00A46126803689A430B461A600A1DE0
:1022F000126803689A430B1D1A60027911440A6838
:1023000003681A430A60184A0832126803689A433D
:10231000154B08331A601A1D126803689A43124B52
:102320000C331A604279102A0ED11A1F1268036802
:102330001A430D4B08331A601A1D126803681A43BA
:10234000094B0C331A600DE00749427911440A68C1
:1023500003681A430A6005E0027911440A680368B9
:102360009A430A607047000000040140FEB504462D
:102370000126022C1BD1002512E03146FF200CF073
:1023800049FA0EB9012000E00020064602A800210B
:10239000C8230A46CDE90010084602F0B3FA6D1CC6
:1023A000052DEADB0021FF200CF034FA12E0012CAD
:1023B00010D10121FF200CF02DFA02A800210B46BC
:1023C0000122CDE90010084602F09CFA0021FF200E
:1023D0000CF020FAFEBD00000149C8607047000003
:1023E0000020024030B5044604250F4800F088F86C
:1023F0000546042D16D10D48006940F002000B4936
:10240000086108464461006940F0400008610648E0
:1024100000F076F805460548006941F6FD71084070
:1024200002490861284630BDFFFF0F00002002402E
:1024300004200B49C96801F0010109B101200EE037
:102440000749C96801F0040109B1022007E0044905
:10245000C96801F0100109B1032000E004207047B1
:10246000002002400348006940F0800001490861F3
:10247000704700000020024078B506460C4604254F
:10248000002000904FF6FF7000F03AF80546042D4A
:1024900026D11448006940F00100124908613480D7
:1024A0004FF6FF7000F02CF80546042D11D1B01C3A
:1024B0000090200C009908804FF6FF7000F020F883
:1024C00005460848006941F6FE7108400549086163
:1024D00006E00448006941F6FE71084001490861C0
:1024E000284678BD0020024002480349486003485E
:1024F000486070472301674500200240AB89EFCD5B
:1025000000B502460423FFF793FF034603E0FFF7FD
:102510008FFF0346521E012B01D1002AF7D102B9C9
:102520000523184600BD2DE9F04104460E46154628
:102530004FF00008374604F0030010B905F003001F
:1025400008B1BDE8F081FFF7CFFF3420FFF744FF6B
:1025500004EB050802E0206801C7241D4445FAD3B6
:10256000FFF780FF00BFECE72DE9F04104460D4680
:10257000164601274FF0000804F0030010B906F0DA
:10258000030010B10020BDE8F081FFF7ADFF34205B
:10259000FFF722FF04EB060809E020462968FFF751
:1025A0006BFF042802D12D1D241D00E000274445A7
:1025B000F3D3FFF757FF3846E5E72DE9F04104462E
:1025C0000E460025A84604F0030010B906F00300EB
:1025D00010B14046BDE8F081FFF786FF3420FFF7D9
:1025E000FBFEA019051F04E02F68781C00B102E073
:1025F0002D1FAC42F8D300BFFFF734FFAC4202D826
:10260000281DA0EB04084046E4E72DE9F04105460B
:102610000E46012700244FF0040811E0FFF764FF85
:102620003420FFF7D9FE2819FFF7DCFE8046FFF7BC
:1026300019FFB8F1040F01D0002703E004F500648E
:10264000A642EBD800BF3846BDE8F0812DE9F8433B
:1026500007460D4614461E46DDF820800121384607
:1026600004F09CFDADF800408DF803608DF8028009
:102670006946284600F026F82146284600F001F970
:10268000BDE8F88330B500228B071C0F0F2303FA37
:1026900004F20B4B8C1053F824309343084C8D10EC
:1026A00044F8253023468C1053F824308C07240F2F
:1026B00000FA04F42343024C8D1044F8253030BD59
:1026C000080001402DE9F0410246002500260020C7
:1026D00000230024002791F803C00CF00F0591F8A7
:1026E00003C00CF0100CBCF1000F03D091F802C035
:1026F0004CEA050591F800C0BCF1000F31D0146818
:1027000000202BE04FF0010C0CFA00F3B1F800C0F0
:102710000CEA03069E4220D183004FF00F0C0CFA06
:1027200003F7BC4305FA03FC4CEA040491F803C028
:10273000BCF1280F06D14FF0010C0CFA00FCC2F8D6
:1027400014C00AE091F803C0BCF1480F05D14FF066
:10275000010C0CFA00FCC2F810C0401C0828D1D3B0
:102760001460B1F800C0BCF1FF0F34DD54680020E4
:102770002EE000F1080C4FF0010808FA0CF3B1F854
:1027800000C00CEA03069E4221D183004FF00F0CDB
:102790000CFA03F7BC4305FA03FC4CEA040491F875
:1027A00003C0BCF1280F05D100F1080C08FA0CF8A1
:1027B000C2F8148091F803C0BCF1480F07D100F1B2
:1027C000080C4FF0010808FA0CF8C2F81080401C01
:1027D0000828CED35460BDE8F0810000F0B50A4669
:1027E000002300240021002500F00046B6F1004F30
:1027F00002D11D4EF16901E01B4E7168C0F3034523
:1028000083B200F44016B6F5401F08D121F0706184
:10281000154E766826F07066134F7E6012E000F465
:102820008016B6F5801F06D1032606FA05F4A143EB
:1028300041F0706106E0460D360103FA06F6B14339
:1028400041F0706122B1460D360103FA06F63143BC
:1028500000F00046B6F1004F02D1034EF16101E0F5
:10286000014E7160F0BD00000000014002460020F2
:1028700093680B400BB1012000E0002070474161DC
:102880007047016170470AB1016100E04161704722
:102890000248006800EB800080007047F4000020D0
:1028A00010B502460020002148E002EB8203254CCF
:1028B00004EB431301EB810403EB041393F82E3074
:1028C000012B0FD102EB82031E4C04EB431301EBEF
:1028D000810403EB04135B68FBB101238B400343CA
:1028E000D8B21AE002EB8203164C04EB431301EB5F
:1028F000810403EB04135B78012B0AD002EB820303
:10290000104C04EB431301EB810403EB04135B68ED
:102910001BB101238B400343D8B202EB8203094C65
:1029200004EB431301EB810403EB041393F8303001
:102930001BB101238B400343D8B2491C0229B4DBED
:1029400010BD00003893002070B500260020FFF76E
:10295000A7FF04460120FFF7A3FF054644EA051040
:10296000C6B2304670BD000070B50446002506E0D2
:1029700028466D1CB0F5FA6F01D9FF2070BD022109
:102980000E4806F033F80028F2D021460B4806F036
:1029900039F8002506E028466D1CB0F5FA6F01D91C
:1029A000FF20EBE70121054806F020F80028F2D0CF
:1029B000024806F024F8C0B2E0E700000030014011
:1029C00008B5032048233C22024900904020FFF72D
:1029D0003DFE08BD001801400246002102F00F0133
:1029E000C90001F0080008B181F0030101F01000F6
:1029F00008B181F0050101F0200008B181F0060165
:102A000001F0400008B181F0070101F07F0070473C
:102A100010B503460C4600210022194600BF01F004
:102A2000400008B182F0070201F0200008B182F0F6
:102A3000060201F0100008B182F0050201F0080062
:102A400008B182F0030201F0040008B182F0040230
:102A500001F0020008B182F0020201F0010008B1A9
:102A600082F001022270082A1DD2DFE802F004067B
:102A7000080A0E101418C91015E0C91013E0C91087
:102A800011E081F00800C1100DE0C9100BE081F0E9
:102A90001000C11007E081F02000C11003E081F0B8
:102AA0004000C11000BF00BF01F00F0010BD2DE9B4
:102AB000F84307460E4615464FF00008A94605EBB9
:102AC000D97041103046FDF762FC00240EE0381941
:102AD000694600F010F8A14604EBD9714910705412
:102AE0009DF8000008B14FF00108A41CAC42EEDBD9
:102AF0004046BDE8F883FCB507460D460026002099
:102B00000090287000240BE0385D01A9FFF780FFDA
:102B10000DF804009DF8040008B101202870641C21
:102B2000022CF1DB9DF8000006439DF8010046EA07
:102B30000010C6B23046FCBD2DE9F04107460D46F7
:102B4000164671002846FDF722FC002406E002220A
:102B500002FB0451385D00F005F8641CB442F6DB5A
:102B6000BDE8F08138B504460D460020009028806D
:102B700004F00F008DF8000020098DF801000023FB
:102B800005E01DF80300FFF727FFE8545B1C022B4C
:102B9000F7DB38BD00BFFEE7302805DB392803DC52
:102BA000A0F13001C8B210E0412805DB462803DC63
:102BB000A0F13701C8B208E0612805DB662803DC14
:102BC000A0F15701C8B200E0FF20704708B500200F
:102BD00000900121082004F0E1FA2020ADF8000067
:102BE00010208DF8030002208DF802006946154878
:102BF000FFF768FD20211348FFF743FE4020ADF8A2
:102C0000000010208DF8030003208DF80200402101
:102C10000C48FFF736FE69460A48FFF753FD80204F
:102C2000ADF8000014208DF8030003208DF8020099
:102C300080210448FFF725FE69460248FFF742FD60
:102C400008BD0000000C014010B500200F490860CD
:102C50000F48006820F070400D4908600846006881
:102C600040F0E040086000200A49C1F89C010420BF
:102C700008F0D9FF012005490860022008F0D3FFC1
:102C800000200449C1F8980110BD0000988121423C
:102C9000000C01400080214210B500200F4908605F
:102CA0000F48006820F070400D4908600846006831
:102CB00040F0E040086001200A49C1F89C0104206E
:102CC00008F0B1FF012005490860022008F0ABFFC1
:102CD00000200449C1F8980110BD000098812142EC
:102CE000000C01400080214270B5054600241748C1
:102CF000006820F07040154908600846006840F000
:102D000000400860002616E00020114908600420F9
:102D100008F089FF01200F49C1F898016006040EF0
:102D20000B487C38006808B1601CC4B2012008F070
:102D30007AFF701CC6B2082EE6DB15B9FFF7ACFFB0
:102D400001E0FFF781FF204670BD0000000C01404C
:102D5000988121420080214270B504460020154927
:102D600008601548006820F0704013490860084664
:102D7000006840F0E0400860002517E0E0090D49D8
:102D8000091D08606006040E042008F04CFF0120B5
:102D90000A49C1F89801022008F045FF00200549C2
:102DA0000860022008F03FFF681CC5B2082DE5DB73
:102DB00070BD000098812142000C0140008021423A
:102DC00010B50F48006820F070400D4908600846B3
:102DD000006840F0E040086001200A4908600A49A4
:102DE000C1F89801042008F01EFF00200549086082
:102DF000042008F018FF00200349C1F8980110BD15
:102E0000000C01409C8121420080214210B51348F2
:102E1000006820F07040114908600846006840F0E2
:102E2000E040086000200E4908600E49C1F8980192
:102E3000042008F0F8FE01200949091F0860042059
:102E400008F0F1FE01200749C1F89C01042008F0B8
:102E5000EAFE00200449087010BD0000000C01408B
:102E60009C81214200802142FC00002010B50024FA
:102E70001448006820F07040124908600846006855
:102E800040F00040086001200F49086008F0CBFEC8
:102E900001200E49C1F8980108F0C5FE07E0601C4A
:102EA000C4B2FA2C03DDFFF7B1FF012010BD0648C4
:102EB000803800680028F2D10349091F086000BF6C
:102EC000F4E70000000C01409C8121420080214277
:102ED0004AF6AA200149086070470000003000400F
:102EE0000146CA1701EB92729210A1EB820292B9CD
:102EF000642091FBF0F200FB121050B94FF4C8703F
:102F000091FBF0F200FB121008B90120704700207D
:102F1000FCE70120FAE70020F8E7000008B50320ED
:102F200010239A021B4900904020FFF78FFB4FF4BB
:102F300080411848FFF7A5FC17480078B0B9032076
:102F400010234FF47042154900902020FFF77EFBBC
:102F5000032010234FF47072114900901846FFF7B8
:102F600075FB0021FF200BF055FC10E00A480078AB
:102F700001280CD1032010234FF460520549009022
:102F80004020FFF763FB0021FF200BF043FC0BF018
:102F900071FB08BD00180140F8000020001401403A
:102FA000001001400EB516E00BF096FB0BF002FB93
:102FB00008F052FF0EF0B8FA08F0EAFE10F03AFC02
:102FC0000EF00EFD02A8002132230A46CDE90010C2
:102FD000084601F097FCE7E70EB50CF045F90BF059
:102FE0008DFE0FE00CF030FC07488069401C06495C
:102FF000886102A8002101230A46CDE90010084695
:1030000001F080FCEEE70000B406002070B5044635
:103010000D46294620460BF0FDFB70BD00BFFEE7C4
:103020007047000070B5002100230F22C47804B35C
:10303000154C246804F4E064C4F5E064210AC1F18D
:103040000403CA40447804FA03F18478144021430D
:1030500009010E4C0678A155047804F01F050124DF
:10306000AC4005786D11AD0005F1E025C5F80041D3
:1030700009E0047804F01F050124AC40044D0678F3
:10308000761145F8264070BD0CED00E000E400E04C
:1030900080E100E002490143024A116070470000EC
:1030A0000000FA050CED00E0024A0A400243024B20
:1030B0001A60704780FFFF1F08ED00E006480068B7
:1030C00000F4E06005490843001D03490860BFF3B0
:1030D0004F8F00BFFEE700000CED00E00000FA0596
:1030E0000648006800F4E06005490843001D0349F4
:1030F0000860BFF34F8F00BFFEE700000CED00E05B
:103100000000FA0515481648164817481748184889
:103110001848194819481A481A481B481B481C489F
:103120001C481D481D481E481E481F481F4820486F
:10313000204821482148224822482348234824483F
:10314000244825482548264826482748274828480F
:1031500028482948294800BF70470000083D030857
:10316000683C03086C3C0308703C0308743C03088B
:10317000783C03087C3C0308803C0308843C03083B
:10318000883C03088C3C0308903C0308943C0308EB
:10319000983C03089C3C0308A03C0308A43C03089B
:1031A000A83C0308AC3C0308B03C0308B43C03084B
:1031B000B83C0308BC3C0308C03C0308C43C0308FB
:1031C000C83C0308CC3C0308D03C0308D43C0308AB
:1031D000D83C0308DC3C0308E03C0308E43C03085B
:1031E000E83C0308EC3C0308F03C0308F43C03080B
:1031F000F83C0308FC3C0308003D0308043D0308B9
:103200007047000070B5044600F076F8002032499F
:1032100008703249087032490870324908703248E3
:1032200000680A21B0FBF1F03049086030480068BE
:1032300058B13048056845B12D48066803E0761E50
:10324000002028602D1D002EF9D102F04DFA02F069
:1032500045FB204602F03AFF208800B170BD2046B1
:1032600001F0FCFE208800B1F8E7204601F048FD9F
:10327000208800B1F2E7204603F094FC208800B1DA
:10328000ECE7204602F066FE208800B1E6E7204623
:1032900001F08CFF208800B1E0E7204601F0AEFF8E
:1032A000208800B1DAE7204602F066FA208800B1F3
:1032B000D4E7204602F076FC208800B1CEE7204615
:1032C00003F0B8FC208800B1C8E701F037FCFFF735
:1032D00019FF00BFC2E700001803002019030020F7
:1032E0004A03002050030020C83C03084C03002080
:1032F000983C0308943C03080448006804490968A2
:1033000000EB8100001F034908607047943C0308EC
:10331000983C0308A803002008480078012800D042
:10332000704707480078FA2800DBF9E7044800787E
:10333000401C0349087000BFF2E700001903002099
:103340001803002010B500242E480078012800D072
:1033500010BD00BFFCF752FF044600BF2A480078AA
:1033600028B900BF2046FCF74DFF00BFF0E7264814
:103370000078401E2449087008460078002805DDC2
:1033800000BF2046FCF73EFF00BFE1E71F48007882
:10339000002805DD00BF2046FCF734FF00BFD7E75B
:1033A00002F08EF91A4908700846007800EB4000D8
:1033B000184951F820001849086008460068174964
:1033C0000968884205D100BF2046FCF71BFF00BFFB
:1033D000BEE711480068D0F88400401C0E49096817
:1033E000C1F884000E480068401C0D4908604FF089
:1033F00080500C49086000BF2046FCF703FF00BF67
:1034000000BFA5E719030020180300204A0300208D
:1034100041030020D0BD0020A4030020A003002011
:103420007403002004ED00E02DE9FF4F83B0044653
:1034300015461F46DDE91096002000904E480078A2
:10344000002805DD45F2B960308007B0BDE8F08F97
:103450001DB945F2BB603080F7E7022F03DA45F271
:10346000BC603080F1E7B9F1040F03D245F2C160CE
:103470003080EAE74FF0030ABAF1000F0CD005EAFA
:103480000A0018B145F2BB603080DEE709EA0A00A5
:1034900010B145F2C1603080AB46A846781E80B2BC
:1034A00001900020029007E0C844CBF80080C3469A
:1034B0000298401C80B20290DDE901108842F3DBE3
:1034C0000020CBF8000000BF00BF00BFFCF796FE55
:1034D000009000BF00BF29480078401C27490870B1
:1034E00000BF00BF0098FCF78DFE00BF00BF00BF0B
:1034F000234820600498A0606560E560A782678229
:10350000A4F81090204601F03DFE1E480088401CA3
:103510001C49088000BF00BF00BFFCF76FFE009091
:1035200000BF00BF15480078401E144908700846C7
:103530000078A0B914480088002809DD00BF00BF4A
:103540000098FCF75FFE00BF00BF02F07DFA0DE0BF
:1035500000BF00BF0098FCF755FE00BF06E000BFAB
:1035600000BF0098FCF74EFE00BF00BF00BF002068
:10357000308000BF69E70000180300204A030020E4
:103580004D454D2034030020240300202DE9F04157
:1035900004460D4600272CB945F2BF602880002064
:1035A000BDE8F08100BF00BFFCF728FE074600BF62
:1035B00000BFA08A58B900BF00BF3846FCF722FE02
:1035C00000BF00BF45F2C26028800020E8E7E6683F
:1035D0003068E060A08A401EA08200BF00BF38466D
:1035E000FCF710FE00BF00BF002028803046D7E760
:1035F0002DE9F04104460E461546002724B945F250
:10360000BF602880BDE8F0811EB945F2BE60288009
:10361000F8E700BF00BFFCF7F1FD074600BF00BFA1
:10362000A08A618A88420ADB00BF00BF3846FCF7E7
:10363000E9FD00BF00BF45F2BA602880E2E7E0681C
:103640003060E660A08A401CA08200BF00BF384600
:10365000FCF7D8FD00BF00BF0020288000BFD1E7E5
:103660002DE9F04104460F4616461D464FF000086E
:1036700036480078002804DD42F6E1602880BDE885
:10368000F0811CB945F6C3502880F8E71EB946F210
:1036900094502880F3E700BF00BF00BFFCF7AEFDE9
:1036A000804600BF00BF2A480078401C28490870A7
:1036B00000BF00BF4046FCF7A5FD00BF00BF00BF34
:1036C000244820606760314604F1200001F014FEB8
:1036D00004F1080001F00EFF204602F035F81E4804
:1036E0000088401C1C49088000BF00BF00BFFCF7D9
:1036F00085FD804600BF00BF15480078401E144974
:10370000087008460078A0B914480088002809DD30
:1037100000BF00BF4046FCF775FD00BF00BF02F0D0
:1037200093F90DE000BF00BF4046FCF76BFD00BF02
:1037300006E000BF00BF4046FCF764FD00BF00BFCD
:1037400000BF0020288000BF99E700001803002078
:103750004A0300205155455548030020240300200A
:103760002DE9F04F89B00746894690461E46DDE9AF
:1037700012544FF0000B78480078002806DD46F21E
:10378000AE102080002009B0BDE8F08F27B945F6C3
:10379000C35020800020F6E726B946F2D5202080CD
:1037A0000020F0E7B8F1000F03D0B8F5004F02D1C8
:1037B00000E000BF04E045F6256020800020E2E73D
:1037C00000BF66493868884204D045F6C45020805E
:1037D0000020D8E70DB10020286000BF00BFFCF733
:1037E0000DFD834600BF00BF23462A46314607F140
:1037F000200001F04DFD8246208840B900BF00BF87
:103800005846FCF7FFFC00BF00BF5046BBE708F47A
:10381000004058B100BF00BF5846FCF7F3FC00BFA2
:1038200000BF46F2B01020800020ACE74C48007882
:1038300000280BDD00BF00BF5846FCF7E3FC00BFCB
:1038400000BF46F66350208000209CE700BF44483C
:103850000078401C4249087000BF00BF5846FCF782
:10386000D1FC00BF00BF00BF4B460522394601A86E
:1038700001F0B8FD00BF00BF00BFFCF7BFFC8346EE
:1038800000BF00BF36480078401E3549087000BFB1
:1038900000BF5846FCF7B6FC00BF00BF00BF00F0F9
:1038A00063F800BF00BFFCF7A9FC834600BF00BF60
:1038B0002C48006890F8350030B1012815D0022856
:1038C0002AD0032835D11DE026480068D0F85CA036
:1038D00024480068B0F8600030801DB121480068BD
:1038E000006C2860002020802BE04FF0000A0020B0
:1038F00030801DB11B480068006C286046F2A9109A
:1039000020801EE04FF0000A0020308005B12860C2
:1039100047F2D920208014E04FF0000A00203080C8
:103920001DB110480068006C286045F6C250208028
:1039300007E04FF0000A0020308046F62B60208020
:1039400000BF00BF00BF00BF5846FCF75BFC00BFD4
:1039500000BF504617E70000180300205155455599
:103960004A030020A003002010B50024204800785E
:10397000002800DD10BD1F480078002800DDF9E7B1
:1039800000BFFCF73BFC044600BF01F099FE1A495A
:1039900008700846007800EB4000184951F82000F4
:1039A000174908600846006816490968884205D129
:1039B00000BF2046FCF726FC00BFDBE7104800688C
:1039C000D0F88400401C0E490968C1F884000E48F4
:1039D0000068401C0C4908604FF080500B4908609B
:1039E00000BF2046FCF70EFC00BF00BFC2E700008E
:1039F000180300204A03002041030020D0BD00200E
:103A0000A4030020A00300207403002004ED00E0C4
:103A100070B50446002517480078002803DD46F6F7
:103A20006250208070BD14480078012803D045F60C
:103A300089602080F6E711480078FA2803DB45F218
:103A400009202080EEE700BF00BFFCF7D7FB05464A
:103A500000BF00BF09480078401C0849087000BF3B
:103A600000BF2846FCF7CEFB00BF00BF002020802F
:103A700000BFD7E718030020190300204A030020E5
:103A800070B5044600251F480078002803DD46F67F
:103A90006550208070BD1C480078012803D045F691
:103AA00089602080F6E71948007818B946F6645016
:103AB0002080EFE700BF00BFFCF7A0FB054600BF7A
:103AC00000BF12480078401E104908700846007870
:103AD00000280ADD00BF00BF2846FCF793FB00BFAB
:103AE00000BF46F663502080D4E700BF00BF2846E1
:103AF000FCF788FB00BF00BFFFF736FF00202080E7
:103B000000BFC7E718030020190300204A03002064
:103B10002DE9F04104460E4617461D464FF00008B9
:103B200018480078002804DD42F6E1602880BDE8EE
:103B3000F0811CB945F6C3502880F8E700BF00BFEC
:103B4000FCF75CFB804600BF00BF0F482060276287
:103B500000206062666004F1080001F0CBFC2046A2
:103B600002F008F809480088401C0849088000BF96
:103B700000BF4046FCF746FB00BF00BF0020288086
:103B800000BFD4E71803002053454D4158030020DF
:103B90002DE9F04788B00646894690461C46109DA0
:103BA0004FF0000A6E480078002806DD46F2AE109D
:103BB0002880002008B0BDE8F08726B945F6C3503C
:103BC00028800020F6E7B8F1000F03D0B8F5004FC9
:103BD00002D100E000BF04E045F625602880002007
:103BE000E8E700BF5F493068884204D045F6C4501A
:103BF00028800020DEE70CB10020206000BF00BF5D
:103C0000FCF7FCFA824600BF00BF306A88B1306A18
:103C1000401E30620CB1706A2060376A00BF00BF7E
:103C20005046FCF7EFFA00BF00BF0020288038465E
:103C3000C0E708F4004060B1376A00BF00BF5046DB
:103C4000FCF7E0FA00BF00BF46F2B010288038460B
:103C5000B0E74548007800280BDD00BF00BF5046A4
:103C6000FCF7D0FA00BF00BF46F663502880002062
:103C7000A0E700BF3C480078401C3B49087000BFEB
:103C800000BF5046FCF7BEFA00BF00BF00BF4B4666
:103C900006223146684601F0A5FB00BF00BF00BF09
:103CA000FCF7ACFA824600BF00BF2F480078401EE8
:103CB0002D49087000BF00BF5046FCF7A3FA00BFB3
:103CC00000BF00BFFFF750FE00BF00BFFCF796FA31
:103CD000824600BF00BF2548006890F8350030B12B
:103CE00001280CD002281AD0032821D110E01CB1E1
:103CF0001E480068006C20600020288024E01CB171
:103D00001A480068006C206046F2A91028801BE069
:103D10000CB10020206047F2D920288014E01CB1AB
:103D200012480068006C206045F6C25028800BE005
:103D300046F62B60288000BF00BF5046FCF762FAB1
:103D400000BF00BF002035E700BF376A00BF00BFDB
:103D50005046FCF757FA00BF00BF38462AE700007C
:103D60001803002053454D414A030020A0030020C2
:103D70002DE9FF4105460F46144635B945F6C350B7
:103D80002080002004B0BDE8F081134928688842F3
:103D900004D045F6C45020800020F3E7FEF798F8E1
:103DA00006460E48007800280CDD00200346024637
:103DB0002946CDE9017603940090074800F0D8FF2A
:103DC0000020DFE7234632463946284601F0F6FE5A
:103DD00080464046D6E7000053454D411803002079
:103DE00010B5044612480078E8B901F069FC1149A1
:103DF000087008460078104908700E48007800EBFB
:103E000040000E4951F820000D490860084600683E
:103E10000C490860012006490870FCF7A9F943F62F
:103E20009920208002E045F68A60208010BD0000C5
:103E3000190300204103002040030020D0BD0020D2
:103E4000A4030020A00300202DE9F04107464FF015
:103E5000000800202849086028490880284908608F
:103E600028490860284908602848046822E000BF03
:103E700000BFFCF7C3F9804600BF00BF002044F834
:103E8000780FE062E06060720021A161E16121626F
:103E90006162FEF71DF86061783C04F16406002061
:103EA000B081D4F8B44000BF00BF4046FCF7AAF987
:103EB00000BF00BF002CDAD102F050FD02F0B6FFC7
:103EC0001348056812E000BF00BFFCF797F9804671
:103ED00000BF00BF05F120060020B081AD6900BF22
:103EE00000BF4046FCF78EF900BF00BF002DEAD1AD
:103EF00000203880BDE8F0812C030020260300203C
:103F00006C0300208403002090030020780300202D
:103F100044030020F8B5044600266A46002102202A
:103F200000F064FCBDF8000018B1BDF8000020806E
:103F3000F8BD00BF00BFFCF761F9064600BF00BF37
:103F400000201E49086000BF00BF3046FCF75AF948
:103F500000BF00BF00251A4800681A490968884256
:103F600005D91748006817490968B0FBF1F525B96C
:103F7000134800680A21B0FBF1F56A460021284683
:103F800000F034FC00BF00BFFCF738F9064600BF64
:103F900000BF00200C490860084800680B49086011
:103FA00001200B49087000BF00BF3046FCF72AF91A
:103FB00000BF00BF0020208000BFB9E75C030020E5
:103FC000C83C0308B03C03086C03002060030020D9
:103FD00068030020704700002DE9FF4F87B00446BA
:103FE0009046DDE91BA5DDE91496179F002003909C
:103FF00087480078002805DD47F24A1028800BB07A
:10400000BDE8F08F1CB947F2AD102880F7E7B8F192
:10401000000F03D147F24F102880F0E71EB946F693
:104020002C602880EBE77B480068874203D246F685
:104030002D602880E3E71698B84203D346F62E6039
:104040002880DCE7B9F1400F03D346F273202880C3
:10405000D5E7B9F1000F06D16F48844203D046F28C
:1040600073202880CBE7B9F13F0F06D16B4884421B
:1040700003D046F273202880C1E7204602F036F8CC
:10408000002028800AF0010090B10AF0020078B107
:1040900005960020069008E000210598016005982B
:1040A000001D05900698401C06900698B842F3D370
:1040B000169806EB80000490CDE9007A324640461F
:1040C000049B0A9900F004FB0590C4F828800A9824
:1040D000E0620898206284F8379005982060049880
:1040E000A06019986065199818B94D480068A065D6
:1040F00001E01998A0651A9860606662A763A4F849
:104100003CA04FF0000B08E0002104F17C0040F8D7
:104110002B100BF101001FFA80FBBBF1000FF3D055
:1041200004F16400189901F0E7F8204600F082F8E5
:1041300000BF00BF00BFFCF761F8039000BF00BFE5
:1041400038480078401C3749087000BF00BF03980A
:10415000FCF758F800BF00BF00BF94F8370001F02B
:10416000CFFA204601F002FC204601F075FF2E48F0
:104170000088401C2C4908802C48007801282DD04C
:1041800000BF00BF00BFFCF739F8039000BF00BFBD
:1041900024480078401E2349087008460078A0B9DA
:1041A00023480088002809DD00BF00BF0398FCF702
:1041B00029F800BF00BF01F047FC0DE000BF00BFC1
:1041C0000398FCF71FF800BF06E000BF00BF03988C
:1041D000FCF718F800BF00BF00BF10E700BF00BF2A
:1041E00000BFFCF70BF8039000BF00BF0D4800783C
:1041F000401E0C49087000BF00BF0398FCF702F88E
:1042000000BF00BF00BFFFF7AFFB00BFF7E6000035
:1042100018030020C43C030810BD002050BC00203F
:104220004C0300204A0300207C03002019030020D7
:10423000240300207047000070B504460D46002698
:1042400067480078002803DD47F24E10288070BDD3
:104250006448844203D147F24C102880F7E7624853
:10426000844203D147F24D102880F0E77CB900BFAB
:1042700000BFFBF7C3FF064600BF00BF5B480468F2
:1042800000BF00BF3046FBF7BDFF00BF00BF00BF4F
:1042900000BF00BFFBF7B2FF064600BF00BF544897
:1042A0000078401C5249087000BF00BF3046FBF741
:1042B000A9FF00BF00BF00BF94F8360008282DD228
:1042C000DFE800F004090E10080A0F11204601F083
:1042D0008DFB54E053E000BF204602F023FB4EE08C
:1042E00000BF00BF00BF204602F01CFB94F8340062
:1042F000082810D2DFE800F004070508090A0B06B9
:1043000000BF00BF08E000BF00BF00BF00BF2046E5
:1043100001F028F900E000BF00BF30E000BF00BF9F
:1043200000BFFBF76BFF064600BF00BF30480078B8
:10433000401E2F49087008460078A0B92D48008813
:10434000002809DD00BF00BF3046FBF75BFF00BF60
:1043500000BF01F079FB0DE000BF00BF3046FBF766
:1043600051FF00BF06E000BF00BF3046FBF74AFF29
:1043700000BF00BF00BF46F62A60288067E700BF85
:1043800004F1640000F062FF204600F037F8204698
:1043900001F07AFE18480088401E17490880204620
:1043A00001F0A4FEFF2084F8360000BF00BF00BF6C
:1043B000FBF724FF064600BF00BF0D480078401EF3
:1043C0000B49087000BF00BF3046FBF71BFF00BF62
:1043D00000BF00BFFFF7C8FA0020288000BF36E703
:1043E0001803002050BC002010BD0020A0030020B6
:1043F0004A030020240300207C03002070477047FC
:104400002DE9F0470746884614461D464FF000093F
:1044100077480078002805DD46F2AE10288000209D
:10442000BDE8F0870CB10020206000BF00BFFBF7A3
:10443000E5FE814600BF00BF6E480068406CA8B32F
:104440006C480068406C401E6A49096848646948C5
:104450000068466C1CB167480068006C2060FDF77E
:1044600037FD64490968096C401A62490968C1F856
:10447000A00060480068D0F8A0005E490968D1F843
:10448000A410884207D95B480068D0F8A0005949B9
:104490000968C1F8A40000BF00BF4846FBF7B2FEA0
:1044A00000BF00BF002028803046B9E7FFE708F4CE
:1044B000004058B100BF00BF4846FBF7A3FE00BF55
:1044C00000BF46F2B01028800020A9E74A480078D3
:1044D00000280BDD00BF00BF4846FBF793FE00BF7E
:1044E00000BF46F663502880002099E700BF42488D
:1044F0000078401C4049087000BF00BF4846FBF7E9
:1045000081FE00BF00BF00BF3B46072200210846D6
:1045100000F068FF00BF00BF00BFFBF76FFE8146E1
:1045200000BF00BF34480078401E3349087000BF08
:1045300000BF4846FBF766FE00BF00BF00BFFFF7A5
:1045400013FA00BF00BFFBF759FE814600BF00BF52
:104550002848006890F8350020B1012826D00328AB
:1045600034D12CE0FCB123480068006C2060FDF7DA
:10457000AFFC20490968096C401A1E490968C1F856
:10458000A0001C480068D0F8A0001A490968D1F8BA
:10459000A410884207D917480068D0F8A000154930
:1045A0000968C1F8A4000020288013E01CB111485C
:1045B0000068006C206046F2A91028800AE00CB167
:1045C0000020206047F2D920288003E046F62B60C7
:1045D000288000BF00BF07480068466C00BF00BFCE
:1045E0004846FBF70FFE00BF00BF304618E700004B
:1045F00018030020A00300204A0300202DE9F04703
:1046000005460E4617461C464FF0000A2E48007815
:10461000002804DD47F258102080BDE8F0871EB95D
:1046200046F2D5202080F8E71FB946F2D520208039
:10463000F3E700BF00BFFBF7E1FD824600BF00BF0C
:104640000DB922480568286868B900BF00BF504608
:10465000FBF7D8FD00BF00BF00203060386047F294
:1046600052102080D9E795F83C0000F0010068B9AD
:1046700000BF00BF5046FBF7C5FD00BF00BF0020D4
:104680003060386047F254102080C6E700BF00BF9A
:104690005046FBF7B7FD00BF00BF4FF00008D5F84C
:1046A000249003E009F1040908F10108D9F8000099
:1046B0000028F7D0C6F80080A86BA0EB080038608F
:1046C0000020208000BFA8E718030020A0030020DE
:1046D000F0B50446DDE9055602EB85004FF0807C1D
:1046E000071F3846C7F800C0071F38463C60DFF890
:1046F0009CC0071F3846C7F800C04FF0123C071F88
:104700003846C7F800C04FF0033C071F3846C7F8CB
:1047100000C04FF0023C071F3846C7F800C0071F13
:1047200038463B60071F384639604FF0113C071F81
:104730003846C7F800C04FF0103C071F3846C7F88E
:1047400000C04FF0093C071F3846C7F800C04FF0C3
:10475000083C071F3846C7F800C04FF0073C071F4A
:104760003846C7F800C04FF0063C071F3846C7F868
:1047700000C04FF0053C071F3846C7F800C04FF097
:10478000043C071F3846C7F800C0F0BDD1630208DB
:1047900010B5FDF79DFB04461248006812490968F0
:1047A000884219D00F480068D0F88C00201A0D49B3
:1047B0000968C1F888000B48006850F8903F4068CD
:1047C00008490968D1F88810591840F10000054AD5
:1047D000126842F8901F506003480068C0F88C408F
:1047E00010BD0000A0030020A40300202DE9F0412B
:1047F00005460E46144600273F480078002804DD91
:1048000047F275202080BDE8F0813C480078002800
:1048100003DD46F663502080F5E736B1022E05D061
:10482000042E0AD0082E09D101E000BF00BF1DB937
:1048300047F27E202080E6E704E003E045F62560AD
:104840002080E0E700BF00BF00BF00BFFBF7D6FC41
:10485000074600BF00BF29480078401C2749087060
:1048600000BF00BF3846FBF7CDFC00BF00BF00BF54
:1048700001202349096881F836002346324629463B
:104880001F48006801F070FF2088A8B100BF00BF7A
:1048900000BFFBF7B3FC074600BF00BF1748007816
:1048A000401E1649087000BF00BF3846FBF7AAFC3F
:1048B00000BF00BF00BFA6E71148006801F096F8EE
:1048C00000BF00BF00BFFBF799FC074600BF00BF59
:1048D0000A480078401E0949087000BF00BF3846EA
:1048E000FBF790FC00BF00BF00BFFFF73DF80020C2
:1048F000208000BF87E70000180300204A03002043
:10490000A00300202DE9FF5F05460E461746984696
:10491000DDE90EA40020009072480078002804DD34
:1049200047F275202080BDE8FF9F6F48007800287F
:1049300003DD46F663502080F5E70AF00E0BBBF16D
:10494000000F09D0BBF1020F07D0BBF1040F10D04C
:10495000BBF1080F0ED101E000BF00BFB8F1000F9E
:1049600006D12FB926B91DB947F27E202080DAE79B
:1049700004E003E045F625602080D4E700BF2AF07C
:104980001E0008B1012000E00020039003980128D8
:1049900003D145F625602080C5E7CAF300100290D8
:1049A0000298C0B9B8F57A7F03D347F27B20208004
:1049B000B9E73B2F03DD47F27A202080B3E73B2E97
:1049C00003DD47F279202080ADE7632D12DD47F249
:1049D00078202080A7E742F20F70864203DD47F27D
:1049E000792020809FE7B5F57A7F03DB47F27820B6
:1049F000208098E73D48D0F800904FF4FA70B0FB63
:104A0000F9F0404400FB09F04FF47A71B0FBF1F18A
:104A10004FF461606843C6EB061200EB8200384435
:104A200000FB091001900198002856D000BF00BF7C
:104A300000BFFBF7E3FB009000BF00BF2A480078EF
:104A4000401C2949087000BF00BF0098FBF7DAFB43
:104A500000BF00BF00BF01202549096881F836006A
:104A600023465A4622480199006801F07DFE2088BD
:104A7000A8B100BF00BF00BFFBF7C0FB009000BFA4
:104A800000BF19480078401E1749087000BF00BFDA
:104A90000098FBF7B7FB00BF00BF00BF43E7144817
:104AA000006800F0A3FF00BF00BF00BFFBF7A6FB3C
:104AB000009000BF00BF0C480078401E0A490870F3
:104AC00000BF00BF0098FBF79DFB00BF00BF00BF09
:104AD000FEF74AFF0020208002E047F27E2020807F
:104AE00000BF20E7180300204A030020C83C030849
:104AF000A003002010B586B000F01EF8FDF7E8F91D
:104B0000044605A800210091CDE90114039007484F
:104B1000007800EB4000064A02EB800100231A46B1
:104B2000044800F025F906B010BD00004003002045
:104B3000D0BD00205449434B704700002048214815
:104B4000214822482248234823482448244825480D
:104B500025482648264827482748284828482948DD
:104B600029482A482A482B482B482C482C482D48AD
:104B70002D482E482E482F482F483048304831487D
:104B8000314832483248334833483448344835484D
:104B9000354836483648374837483848384839481D
:104BA00039483A483A483B483B483C483C483D48ED
:104BB0003D483E483E483F483F4800BF70470000E0
:104BC0000C3D0308743E03080E3D03080F3D030827
:104BD000103D0308143D0308183D0308153D030864
:104BE000483D03084A3D03084C3D03086C3D03085B
:104BF0006E3D0308703D0308723D0308743D0308D1
:104C0000763D0308783D0308A43D0308AA3D030848
:104C1000AB3D0308AC3D0308AE3D0308B03D0308BF
:104C2000B23D0308B43D0308B63D0308B83D030890
:104C3000E83D0308E93D0308EA3D0308EB3D0308AE
:104C4000EC3D0308EE3D0308F03D0308183E030861
:104C5000193E03081A3E03081B3E03081C3E0308C6
:104C60001E3E0308203E0308243E0308253E030899
:104C7000263E0308273E0308283E0308293E030872
:104C80002A3E03082B3E03082C3E03082E3E030851
:104C90002F3E0308303E0308323E0308343E03082B
:104CA000353E0308383E03086C3E03086D3E03089A
:104CB0006E3E0308703E0308723E0308002400BFE6
:104CC00019E000BF00BFFBF799FA044600BF00BF20
:104CD00009480068401C0849086008480068401CF2
:104CE0000649086000BF00BF2046FBF78BFA00BFF3
:104CF00000BFFEF785FAE4E7140300205C03002000
:104D000010B58AB0044600200E4908600320002137
:104D10000591CDE90704069108460B4909680B4A3D
:104D200012680B4B1B68CDE90132CDE903103F201F
:104D30000023084A08A100900C48FFF74DF90AB07B
:104D400010BD000014030020703C03086C3C0308F5
:104D5000683C0308BD4C020875432F4F532D494949
:104D6000492049646C65205461736B0050BC00207D
:104D70002DE9F84F04460D4616461F46DDE90BABFC
:104D8000DDF82890DDF834800020009000BF00BFDF
:104D9000FBF734FA009000BF00BF2A4800882A4978
:104DA000098888423BDA27480088401C254908804A
:104DB000264800880988884203DA22480088234967
:104DC0000880234800680460214800688560204806
:104DD0000068C6601E48006807821D480068C0F869
:104DE00014901B480068A0F818A019480068C0F883
:104DF0001CB0174800684068154908600120154933
:104E00000881154808604860002000F079FC1348CC
:104E10000078134908700020A8F8000008E0114845
:104E20000088401C0F49088044F25360A8F8000035
:104E300000BF00BF0098FBF7E5F900BF00BFBDE869
:104E4000F88F0000240300207C3C03082603002088
:104E50001C030020D0BD002010BD00204003002016
:104E600042030020280300202DE9FE4F4FF0000BE5
:104E700000BF00BFFBF7C2F9834600BF00BF444834
:104E80000068D0F8008042480068866840480068A2
:104E9000C7683F480068B0F810903D480068D0F8F7
:104EA00014A03B480068058B39480068C46938483D
:104EB000006840683649086000BF00BF5846FBF7ED
:104EC000A1F900BF00BF3349A8EB0100884525D0F8
:104ED0000ADC31484044D0B13049084460B130491F
:104EE000084400284FD123E02E49084438B32E4906
:104EF0000844002847D100E046E002A82B464A4675
:104F00003946CDE90040304600F042FC3CE002ABBF
:104F100022462946304600F051FE35E002A82B46D5
:104F20004A463946CDE90040304601F03DF92BE0D4
:104F300002AB22462946304601F056FA24E01B49CE
:104F4000097801EB41011A4A02EB810000F0AAFD49
:104F500002AB22460021174801F046FA16480068C5
:104F6000401E154908600846006858B91348006893
:104F70000860FCF7ADFF044602AB22460021104852
:104F800001F032FA00E000BF00BFBDE8FE8F000074
:104F900020030020544D5347ADBAB2BE0DF90BFAB1
:104FA000F2F8F7FF000410FC03F4FDF542030020C3
:104FB000D0BD002090C100209C0300209803002059
:104FC00050C20020002700BF40E000263CE02048FF
:104FD0000088C0B900BF00BFFBF710F9074600BF4B
:104FE00000BF00201B4908810860486000F09AFB60
:104FF00000BF00BF3846FBF705F900BF00BFFEF752
:10500000B3FC012620E0FCF763FF0546FFF72CFF09
:10501000FCF75EFF441B10480068844201D90E482B
:10502000046000BF00BFFBF7E9F8074600BF00BF00
:1050300007480088401E0649088000BF00BF384668
:10504000FBF7E0F800BF00BF002EC0D0BDE70000B6
:1050500024030020D0BD00202C030020F0B589B02F
:1050600005460020314908803148006820B944F2E3
:105070005260288009B0F0BD2E480088022803DA6B
:1050800044F254602880F5E700202B490860284846
:1050900004682646203600270CE0284820600020BF
:1050A000A060E0602082606120836660203420364A
:1050B000781C87B21F4800888742EEDB203C1C48E2
:1050C000066866601E4806601E48066000201E498D
:1050D00008801E4908801E48006818B946F62C60F2
:1050E0002880C7E71B4800681B490968884203D22B
:1050F00046F62D602880BDE7032000210591CDE90B
:105100000705069113480068144A1268104B1B6883
:10511000CDE90301CDE9013200910B46104A11A1FE
:105120001748FEF759FF00BFA4E70000280300203E
:10513000783C03087C3C03082C0300204E4F4E456E
:105140001C0300202003002024030020260300204D
:10515000843C03088C3C0308C43C0308883C0308D7
:10516000C54F020875432F4F532D494949204953D4
:1051700052205175657565205461736B0000000005
:1051800010BD0020002181610749096811B9002183
:10519000C16105E004490968C16103490968886182
:1051A0000149086070470000300300200021034AD5
:1051B0001160034A11800180704700003003002015
:1051C0003403002070B502460B46104611461031DC
:1051D0005E1EB5B2002408E001600026466006812C
:1051E000C66010301031661CB4B2AC42F4DB00264D
:1051F000066046600681C66070BD000010B50446BA
:105200000F48006818B945F21E70208010BD0D4887
:10521000008818B945F21D702080F7E70948018819
:1052200007480068FFF7CEFF054800680649086098
:105230000448008888800020C880208000BFE5E7FF
:10524000A83C0308A03C03083803002010B5014621
:1052500048894B89002B17DD0A680C4B1B681360CB
:105260000A4C4B6823602346DB884C891B1B074C88
:10527000E38023469B884C892344044CA38000236D
:105280004B818B810B604B6010BD00003803002008
:10529000F0B504460D46608940B90020288002B16F
:1052A000106046F2925018800020F0BD61684E6890
:1052B000088928800AB1C868106008686060606862
:1052C00018B900202060608102E06089401E608182
:1052D000084800680860074801608088401C054F46
:1052E000B8803846C088401EF880002018803046BC
:1052F000DBE7000038030020018100224281828127
:1053000002604260704700002DE9F0410D46DDE982
:105310000674B0F80AC0B0F80880C44505DB46F250
:10532000935CA4F800C0BDE8F081DFF8B4C0BCF81D
:1053300004C0BCF1000F04D145F21D7CA4F800C0EC
:10534000F1E7DFF89CC0DCF80010DFF89480D1F8BA
:1053500000C0C8F800C0C446BCF804C0ACF1010CE1
:10536000A8F804C0C446BCF806C00CF1010CA8F8AB
:1053700006C0B0F80AC0BCF1000F06D10160416060
:105380004FF0010CA0F80AC017E003F0100CBCF1BC
:10539000000F07D1066831604FF0000CC1F800C063
:1053A000016004E0D0F804C0C1F800C04160B0F86A
:1053B0000AC00CF1010CA0F80AC0B0F80AC0B0F89D
:1053C0000C80C44503DDB0F80AC0A0F80CC04D60E5
:1053D0000A81CF604FF0000CA4F800C000BFA2E724
:1053E000380300202DE9F04105460C4616461F46BD
:1053F0001548006880F8346000201349096881F876
:10540000350039461048006800F00AFE6CB104F11E
:105410000808EC60012229460B48006800F016F8E5
:105420002946404600F06BF806E00020064909686E
:10543000C88705490968086303480168204600F0E9
:1054400019F8BDE8F0810000A003002010B5C28764
:10545000016300230AE000244C600C600C614C6185
:105460000C83CC61886020315C1CA3B29342F2DBD8
:1054700010BD000030B548B14568C1F8B85000F122
:105480000804226893681D6AC56113E091F83450DE
:10549000022D02D0072D08D103E007A5C1F8B850AE
:1054A00007E007A5C1F8B85003E008A5C1F8B85057
:1054B00000BF00BF30BD00005461736B205100007D
:1054C0005461736B2053656D0000000020000000E4
:1054D00030B507A5C1F8B85000F1080422681AB128
:1054E00093681D6AC56101E001A5C56130BD00007A
:1054F0002000000000210160416001817047F0B58B
:105500008E6896F8375007893FB901270781002731
:105510004F600F600160416023E007897F1C0781B5
:10552000026806E0946894F83770AF4200DD02E04C
:105530005268002AF6D100BF32B900274F60436895
:105540000B60596041600CE017682FB911600027AB
:105550000F604A60016004E013680B604A605960A4
:105560001160F0BD2DE9F0410446256BE68F0AE09D
:10557000D5F80C8008F108072946384600F00AF8EB
:105580002035701E86B2002EF2DC0020E0872063FA
:10559000BDE8F08110B50489012C03D1002404601A
:1055A000446011E00C6824B94A6800241460026069
:1055B0000AE04C6824B90B6800245C60436003E097
:1055C0000B684A685A6013600489641E04810024D1
:1055D0004C600C6010BD2DE9F84306460C4617469A
:1055E0009846089D94F83600082850D2DFE800F06D
:1055F0000405080906072B2C00BF00BF00BF47E0C9
:1056000000BF94F83400032807D143463A462146A8
:105610003046009500F03FF803E0E765A4F86080AD
:10562000256436B12046FFF79DFF21463046FFF73F
:105630004FFF204600F0BEFE00203434A0706070A2
:1056400004F8340924E000BF94F83400032807D19B
:1056500043463A4621463046009500F01CF803E0E8
:10566000E765A4F860802564204601F05BF936B157
:105670002046FFF777FF21463046FFF729FF042039
:105680003434A0700020607004F8340900E000BFDA
:1056900000BFBDE8F883F0B50446059E086BCD8FCA
:1056A0000AE0C768A74204D1046142610383C6616E
:1056B00004E020306F1EBDB2002DF2DC00BFF0BD53
:1056C00070B50025074C03E005F12000C5B2241D8C
:1056D00020680028F8D02068FAF797FD2844C5B262
:1056E000284670BD0C030020002004E00021034A7E
:1056F00042F82010401C0228F8D370470C03002009
:1057000030B5420900F01F030121C3F11F04A1407D
:10571000034C54F822400C43014D45F8224030BD63
:105720000C03002030B5420900F01F030121C3F132
:105730001F04A140034C54F822408C43014D45F80E
:10574000224030BD0C03002009A1C161002141614C
:105750000849096811B90021816105E00549096816
:105760008161044909684861024908607047000086
:1057700020000000440300200021034A1160034A76
:10578000118001807047000044030020480300207E
:105790002DE9F04F85B007468A4693461C46002007
:1057A000029000BF00BF00BFFAF728FD029000BFC3
:1057B00000BF48480078401C4649087000BF00BF41
:1057C0000298FAF71FFD00BF00BF00BF07F10806EF
:1057D0003089002842D104F0100010B94FF00008C1
:1057E00001E04FF01008DDE90E0143465A46CDE9CD
:1057F0000001514607F12000FFF786FD00BF00BF02
:1058000000BFFAF7FBFC029000BF00BF31480078F0
:10581000401E3049087008460078A0B92E4800881C
:10582000002809DD00BF00BF0298FAF7EBFC00BFBB
:1058300000BF00F009F90DE000BF00BF0298FAF7C1
:10584000E1FC00BF06E000BF00BF0298FAF7DAFCF7
:1058500000BF00BF00BF05B0BDE8F08F04F40070CA
:1058600008B1358900E00125D6F8009011E0D9F89B
:1058700008000390D9F8040004900E985B46524645
:10588000009038460399FFF7A6FEDDF81090681ED9
:1058900085B2002DEBD100BF00BF00BFFAF7AEFC10
:1058A000029000BF00BF0B480078401E09490870F5
:1058B00000BF00BF0298FAF7A5FC00BF00BF00BF01
:1058C00004F4004008B9FEF74FF800210F9801805A
:1058D00000BFC0E74A0300202403002000210AE0A3
:1058E00001EB4102054B03EB8200002202810260C2
:1058F00042604A1CD1B24029F2D37047D0BD00208B
:1059000010B5044694F83700FFF7FAFE94F8370014
:1059100005490978884203D1204600F027F802E0C3
:10592000204600F003F810BD4003002010B590F8A9
:10593000373003EB43030C4C04EB83010B893BB979
:1059400001230B810023C36003610860486009E004
:105950000B895B1C0B810B68C360002303610A6821
:105960001061086010BD0000D0BD002010B590F897
:10597000373003EB43030B4C04EB83010B893BB93A
:1059800001230B810023C36003610860486008E0C5
:105990000B895B1C0B810023C3604A680261D060E5
:1059A000486010BDD0BD002010B501460C8924B15F
:1059B000012C03D0022C0CD101E000BF14E00868D8
:1059C0004A6802610024C4601461D0600A604860C3
:1059D0000AE008684A68C36800241C61C460026168
:1059E000D0600B60486000BF00BF10BD2DE9F041E2
:1059F000054695F8370000EB4000124901EB8004A2
:105A00002F69EE6887B946B9002020812060606068
:105A100095F83700FFF786FE0EE02089401E2081B2
:105A200000203061266007E02089401E2081FE6052
:105A30000EB9676000E0376100202861E860BDE8CA
:105A4000F0810000D0BD002010B5002400BFFAF79F
:105A5000D5FB044600BF00200D4908700D480E49D3
:105A6000086008460068D0F88400401C0968C1F846
:105A700084000A480068401C084908604FF08050C4
:105A80000749086000BF2046FAF7BCFB00BF10BD05
:105A90004103002010BD0020A40300207403002057
:105AA00004ED00E070B5054600262E480078012878
:105AB00000D070BD00BF00BFFAF7A0FB064600BFD4
:105AC00000BF2C683CB900BF00BF3046FAF79AFB14
:105AD00000BF00BFEDE72448844207D100BF00BFEC
:105AE0003046FAF78FFB00BF00BFE2E7A06D10B1B0
:105AF000A06D401EA065A06D38B100BF00BF30464C
:105B0000FAF780FB00BF00BFD3E72889022807DA35
:105B100000BF00BF3046FAF775FB00BF00BFC8E703
:105B200012480078002807DD00BF00BF3046FAF7B2
:105B300069FB00BF00BFBCE72846FFF735FF2C68B4
:105B4000606D18B90A480068A06501E0606DA06545
:105B500000BF00BF3046FAF755FB00BF00BF00BFD3
:105B6000A7E700005003002050BC00204A0300209B
:105B70004C03002009A1C161002141610849096865
:105B800011B90021816105E0054909688161044975
:105B90000968486102490860704700002000000061
:105BA000540300200021034A1160034A1180018040
:105BB0007047000054030020580300202DE9FF5FC8
:105BC0000446884691461D460020019000BF00BF54
:105BD000FAF714FB019000BF00BF04F108073889F1
:105BE00000284FD10420012804D0022814D0042812
:105BF00034D123E0206AFF280DD100BF00BF0198F7
:105C0000FAF700FB00BF00BF46F6C5502880002011
:105C100004B0BDE8F09F22E04FF6FF71206A884291
:105C20000BD100BF00BF0198FAF7ECFA00BF00BF2C
:105C300046F6C55028800020EAE710E0206A401CA4
:105C400058B900BF00BF0198FAF7DCFA00BF00BFE7
:105C500046F6C55028800020DAE700E000BF00BF0C
:105C6000206A401C2062D4F820A0C4F8249000BF11
:105C700000BF0198FAF7C6FA00BF00BF00202880D5
:105C80005046C5E700BF25480078401C23490870EE
:105C900000BF00BF0198FAF7B5FA00BF00BF00BF10
:105CA00008F4007008B13E8900E00126D7F800B082
:105CB00011E0DBF808000290DBF8040003900023F9
:105CC0001A46CDF8009020460299FFF784FCDDF8D3
:105CD0000CB0701E86B2002EEBD1D4F820A000BF0D
:105CE00000BF00BFFAF78AFA019000BF00BF0B485F
:105CF0000078401E0949087000BF00BF0198FAF7FC
:105D000081FA00BF00BF00BF08F4004008B9FDF7EA
:105D10002BFE0020288050467AE700004A0300202E
:105D20001CB50020009000BF06E07E4909684800CD
:105D300001AA0021FEF75AFD7B4800780128F4D122
:105D400001A8FEF781F800277848006875490968BE
:105D5000884205D97548006872490968B0FBF1F7B7
:105D600027B9724800680A21B0FBF1F7D8E0FCF7C8
:105D7000AFF8804600BF00BFFAF740FA009000BFBE
:105D800000BF6B4800686B490860002068490860E4
:105D900000BF00BF0098FAF735FA00BF00BF6648A1
:105DA000006864490968884213D96348006860B193
:105DB00060480068642148435F490968B0FBF1F01E
:105DC000C0F164005D49087006E064205B4908701A
:105DD00002E0642059490870FEF7FCF800252E46C1
:105DE0005748046851E000BF00BF00BFFAF706FA49
:105DF000009000BF00BF53480078401C5149087014
:105E000000BF00BF0098FAF7FDF900BF00BF00BF58
:105E100054F8901F6068C4E902100021216061609D
:105E2000903C00BF00BF00BFFAF7E8F9009000BF48
:105E300000BF44480078401E424908700846007878
:105E4000A0B941480088002809DD00BF00BF0098C4
:105E5000FAF7D8F900BF00BFFFF7F6FD0DE000BF6D
:105E600000BF0098FAF7CEF900BF06E000BF00BF00
:105E70000098FAF7C7F900BF00BF00BF54F8981F99
:105E800060684D194641E0690446002CABD164229C
:105E9000002328463146FAF7C2F905460E4628483F
:105EA000046821E0002185EA0100714008430ED01A
:105EB0002A463346D4E926B15846FAF7B0F900F03D
:105EC000FF0ABAF1640F04D94FF0640A01E04FF001
:105ED000000A84F881A001AB04F1A802111D20463C
:105EE000FEF78CFBD4F8B440002CDBD117480078C7
:105EF000012805D100201549087001A8FDF7A4FF6D
:105F0000FBF7E6FFA0EB080911480068814502D9BC
:105F10000F48C0F8009001AA00213846FEF766FC41
:105F200025E70000B03C030868030020C83C0308D4
:105F30005C03002064030020600300205A0300205B
:105F4000780300204A03002024030020700300206F
:105F50006C03002010B58AB0044600201F49086079
:105F60001F4908601F4908601F4908701F490870D1
:105F70001F48006820B946F62C6020800AB010BD8A
:105F80001C4800681C490968884203D246F62D6007
:105F90002080F3E7194800783F2803D346F27320A6
:105FA0002080EBE7032000210591CDE9070406914D
:105FB000084610490968124A12680D4B1B68CDE962
:105FC0000132CDE903100D48007800230D4A0EA1DF
:105FD00000901248FEF700F800BFCFE75C030020F6
:105FE0006403002060030020680300207003002089
:105FF000B43C0308BC3C0308C43C0308AC3C0308A5
:10600000B83C0308215D020875432F4F532D4949C1
:10601000492053746174205461736B00D0C0002018
:1060200038B504460D4685B16B4602222946204606
:1060300000F09AFBBDF8000018B9032084F8360080
:1060400006E0022084F8360002E0022084F83600E0
:106050002046FFF7CBFC38BD0021C0F8B01009493D
:10606000096819B90021C0F8B41007E005490968AA
:10607000C0F8B41003490968C1F8B00001490860CC
:106080007047000078030020D0F8B020D0F8B4109A
:106090004AB90D4B196011B10023C1F8B03000238B
:1060A000C0F8B4300FE029B90023C2F8B430C0F80A
:1060B000B03008E0C2F8B410C1F8B0200023C0F836
:1060C000B430C0F8B0307047780300200021044A93
:1060D0001160044A1180044A116001807047000079
:1060E000780300207C0300207403002070B5044670
:1060F00000202060A0606060E06020616061A061BD
:10610000E06126A0206200206062A062E06220635D
:10611000E0872064E065A4F86000002104F16400D9
:10612000FFF7EAF800206067A067002506E000217D
:1061300004F17C0040F82510681CC5B2002DF6D093
:10614000002034342061E0662067606084F84C00F1
:10615000A067606720814FF0004060610020A0616F
:10616000E0612062606284F84D0020656065FBF7A5
:10617000AFFE0646A6650021E1652166002020707D
:106180006070A0704020E0700020E067C4F88000DC
:1061900004A0C4F88400343C70BD00003F54617317
:1061A0006B000000200000002DE9FC4704460F466C
:1061B00090469946DDE90A654FF0000A00BF00BF2E
:1061C00000BFFAF71BF8824600BF00BF7648007890
:1061D000401C7549087000BF00BF5046FAF712F81E
:1061E00000BF00BF00BF0CB97048046800202880C1
:1061F00094F8360008287DD2DFE800F004053E3F21
:106200000607404100BF00BF00BF4B46424639462B
:1062100004F16400CDE90065FFF776F800BF00BF28
:1062200000BFF9F7EBFF824600BF00BF5E48007871
:10623000401E5D49087008460078A0B95C48008897
:10624000002809DD00BF00BF5046F9F7DBFF00BFA3
:1062500000BFFFF7F9FB0DE000BF00BF5046F9F7A4
:10626000D1FF00BF06E000BF00BF5046F9F7CAFFEC
:1062700000BF00BF00BF93E000BF00BF00BF94F8A5
:106280003400022821D143463A4621460020009698
:10629000FFF7A1F900BF00BF00BFF9F7AFFF8246CB
:1062A00000BF00BF40480078401E3F49087000BF53
:1062B00000BF5046F9F7A6FF00BF00BF00BF09F4BA
:1062C000004090BBFDF750FB38E04B464246394654
:1062D00004F16400CDE90065FFF716F800BF00BFC8
:1062E00000BFF9F78BFF824600BF00BF2E48007841
:1062F000401E00E023E02C49087008460078A8B949
:106300002B480088002809DD00BF00BF5046F9F780
:1063100079FF00BF00BFFFF797FB0EE000BF00BF93
:106320005046F9F76FFF00BF07E007E000BF00BF6E
:106330005046F9F767FF00BF00BF00BF30E000BF65
:1063400000BF00BFF9F75AFF824600BF00BF1648E2
:106350000078401E1449087008460078A0B9144817
:106360000088002809DD00BF00BF5046F9F74AFF4A
:1063700000BF00BFFFF768FB0DE000BF00BF504645
:10638000F9F740FF00BF06E000BF00BF5046F9F735
:1063900039FF00BF00BF00BF46F62A60288000BF5B
:1063A00000BFBDE8FC8700004A030020A0030020D6
:1063B0002403002010B50446204600F0B3FA94F8F8
:1063C000360000F0040010B92046FFF799FA10BD1E
:1063D00008B504480068FEF712F869460020FDF78A
:1063E0002BFF08BDA00300202DE9F8430446884692
:1063F00017461D464FF0000900BF00BF00BFF9F768
:10640000FDFE814600BF00BFCA480078401CC94954
:10641000087000BF00BF4846F9F7F4FE00BF00BF98
:1064200000BF0CB9C448046827640020288094F891
:106430003600082871D2DFE800F00405EBEC06070F
:10644000EDEE00BF00BF00BF0420012804D00228E9
:1064500039D004286FD170E0606CFF2832D100BFC2
:1064600000BF00BFF9F7CAFE814600BF00BFB148B8
:106470000078401EAF49087008460078A0B9AF48C0
:106480000088002809DD00BF00BF4846F9F7BAFEC2
:1064900000BF00BFFFF7D8FA0DE000BF00BF4846BD
:1064A000F9F7B0FE00BF06E000BF00BF4846F9F7AD
:1064B000A9FE00BF00BF00BF46F6C55028800020DF
:1064C000BDE8F88371E04FF6FF71606C884233D10C
:1064D00000BF00BF00BFF9F791FE814600BF00BFBB
:1064E00094480078401E9349087008460078A8B97F
:1064F00092480088002809DD00BF00BF4846F9F730
:1065000081FE00BF00BFFFF79FFA0EE000BF00BF93
:106510004846F9F777FE00BF07E0D5E000BF00BFAF
:106520004846F9F76FFE00BF00BF00BF46F6C550F2
:1065300028800020C4E737E037E0606C401C88BB4F
:1065400000BF00BF00BFF9F759FE814600BF00BF82
:1065500078480078401E7749087008460078A0B94E
:1065600076480088002809DD00BF00BF4846F9F7DB
:1065700049FE00BF00BFFFF767FA0DE000BF00BF94
:106580004846F9F73FFE00BF06E000BF00BF48469F
:10659000F9F738FE00BF00BF00BF46F6C55028809F
:1065A00000208DE7FFE700E000BF00BF606C401CEB
:1065B0006064666C00BF00BF00BFF9F71FFE814634
:1065C00000BF00BF5B480078401E5A49087008466B
:1065D0000078A0B959480088002809DD00BF00BF35
:1065E0004846F9F70FFE00BF00BFFFF72DFA0DE098
:1065F00000BF00BF4846F9F705FE00BF06E000BF38
:1066000000BF4846F9F7FEFD00BF00BF00BF8DE0A8
:1066100000BF00BF00BF94F83400072822D1002338
:106620001A46214618460097FEF7D5FF666C00BF54
:1066300000BF00BFF9F7E2FD814600BF00BF3D4843
:106640000078401E3B49087000BF00BF4846F9F77C
:10665000D9FD00BF00BF00BF08F4004098BBFDF7A4
:1066600083F930E0606C401C6064666C00BF00BF62
:1066700000BFF9F7C3FD814600BF00BF2D48007879
:10668000401E2C49087008460078A0B92B480088A5
:10669000002809DD00BF00BF4846F9F7B3FD00BF81
:1066A00000BFFFF7D1F90DE000BF00BF4846F9F782
:1066B000A9FD00BF06E000BF00BF4846F9F7A2FDF4
:1066C00000BF00BF00BF31E000BF00BF00BFF9F74F
:1066D00095FD814600BF00BF16480078401E154951
:1066E000087008460078A0B914480088002809DD21
:1066F00000BF00BF4846F9F785FD00BF00BFFFF7A8
:10670000A3F90DE000BF00BF4846F9F77BFD00BFCD
:1067100006E000BF00BF4846F9F774FD00BF00BFA8
:1067200000BF46F62A602880002600BF00BF304622
:10673000C6E600004A030020A00300202403002036
:10674000002108E0064A02EBC100002202608280BC
:10675000C2804A1C91B2034A12889142F2DB704710
:106760003CB90020E03C03082DE9F04F0C461646EA
:106770001D46042E1ED1DFF8A091D9F80090A4EB9D
:106780000909A9F1010313F5803F0DD94FF0000964
:10679000C0F84C90C0F85090C0F81C9047F27E2989
:1067A000A5F80090BDE8F08FC46403F10109C0F8BA
:1067B00050903FE084B3082E25D1D0F8489009EBE3
:1067C0000407DFF85491D9F80090A7EB0909A9F163
:1067D0000103A34201D2C76406E0DFF83C91D9F877
:1067E0000090A144C0F84C90DFF82CA1D0F84C9058
:1067F000DAF800A0A9EB0A09C0F85090D0F84C9044
:10680000C0F8489016E0DFF81091D9F80090A14444
:10681000C0F84C9004650DE0FFE74FF00009C0F8A8
:106820004C90C0F85090C0F81C9047F27E29A5F813
:106830000090B7E7DFF8E4A0BAF800A0D0F84C90D9
:10684000B9FBFAFB0AFB1B991FFA89F8DFF8D09015
:1068500009EBC802B2F80490B9F1000F0BD14FF068
:106860000009C0F81490C0F8189010604FF00109AA
:10687000A2F804903EE0116834E0DFF89CA0D1F863
:106880004C90DAF800A0A9EB0A09C1F85090D0F8B2
:106890005090D1F850A0D1450ED9D1F81490B9F14B
:1068A000000F01D049691DE04FF00009C0F81490B5
:1068B00081614861002115E0D1F81890B9F1000F0D
:1068C00007D14FF00009C0F818904161886110604D
:1068D00007E0D1F818C0C0F818C04161CCF8140026
:1068E000886100210029C8D1B2F8049009F101099A
:1068F000A2F80490B2F80690B2F804A0D14503DAE9
:10690000B2F80490A2F80690C2614FF00009A5F811
:10691000009000BF46E7000080030020E03C030831
:106920003CB9002010B5C269BAB1002404651468EE
:10693000844205D14169116039B100248C6104E0C1
:10694000816943694B6103B19961002444618461A9
:10695000C461C4649488641E948010BD002006E065
:10696000054A02EBC0010022CA80421C90B2034AD1
:1069700012889042F4DB70473CB90020E03C0308E9
:106980002DE9F05F4FF0000B00BF00BF00BFF9F72B
:1069900035FC834600BF00BF71480078401C704939
:1069A000087000BF00BF5846F9F72CFC00BF00BFBD
:1069B00000BFFBF78DFA05466A480068401C69492C
:1069C00008600846006868490988B0FBF1F201FBDD
:1069D00012001FFA80FA654800EBCA08D8F8004098
:1069E000002782E0002C7FD0D4F8149094F8360071
:1069F000082875D2DFE800F00408051B063D0750A3
:106A000000BF00BF00BF6CE05649E06C0968401A47
:106A100020655449E06C0968884206D1002084F85A
:106A200036002046FFF7C6FC00E0012759E04D493B
:106A3000E06C0968401A20654A49E06C09688842A0
:106A400015D10020E065A4F86000FBF741FA20644E
:106A50002046FEF787FD2046FFF7ACFC00203434CB
:106A6000A07003206070002004F8340900E00127C2
:106A700037E03C49E06C0968401A20653949E06C10
:106A80000968884206D1042084F836002046FFF7C2
:106A900049FF00E0012724E03249E06C0968401A10
:106AA00020653049E06C0968884217D10020E06514
:106AB000A4F86000FBF70CFA20642046FEF752FDB4
:106AC0002046FFF72FFF04203434A07003206070AD
:106AD000002004F8340902E006E001E0012700E0AC
:106AE00000BF00BF4C4600E00127002F3FF47AAF03
:106AF000FBF7EEF9461B1E480068864201D91C4888
:106B0000066000BF00BF00BFF9F778FB834600BFF7
:106B100000BF13480078401E1149087008460078ED
:106B2000A0B914480088002809DD00BF00BF5846FE
:106B3000F9F768FB00BF00BFFEF786FF0DE000BF5E
:106B400000BF5846F9F75EFB00BF06E000BF00BF7C
:106B50005846F9F757FB00BF00BF00BFBDE8F09FE4
:106B60004A03002080030020E03C03083CB90020D9
:106B700084030020240300201CB500BF0EE001ABFD
:106B80006A4600210846FDF73BFCBDF8040028B921
:106B900003480078012801D1FFF7F2FEEFE700007B
:106BA0001903002010B58AB004460020144908607B
:106BB00014490860FFF7C4FD134800783F2804D348
:106BC00046F2732020800AB010BD032000210591F9
:106BD000CDE9070406910D4802680D4800680D4B89
:106BE0001B68CDE90130CDE9032107480078002377
:106BF000094A0AA100900E48FDF7EEF900BFE2E74E
:106C00008003002084030020CC3C0308D83C030808
:106C1000D43C0308D03C0308796B020875432F4F1E
:106C2000532D494949205469636B205461736B00AB
:106C300090C1002070B58AB0044600203149086038
:106C40003148006840B1314800682F490968B0FBFD
:106C5000F1F02F49086006E02C4800680A21B0FBDB
:106C6000F1F02B4908602A4800682A490860002092
:106C70002949086029490860002508E0284800EBF8
:106C8000C5060020B080F0803060681C85B22548C1
:106C900000888542F2DB2448006820B947F246307C
:106CA00020800AB070BD21480068214909688842E7
:106CB00003D247F246302080F3E71E4800783F2891
:106CC00003D346F273202080EBE7032000210591D7
:106CD000CDE907040691084614490968164A126866
:106CE000114B1B68CDE90132CDE903101148007842
:106CF0000023124A12A100901748FDF76DF900BF5A
:106D0000CFE7000088030020EC3C0308C83C0308E0
:106D1000980300209C03002094030020900300208F
:106D2000C4BB0020003D0308F03C0308F83C030806
:106D3000C43C0308E83C0308F43C0308516E020815
:106D400075432F4F532D4949492054696D65722071
:106D50005461736B0000000050C20020F0B50C4677
:106D6000022680F82A60012C05D12D4F466A3F6823
:106D70003E4486610CE0066A2EB9294F466A3F6898
:106D80003E44866104E0264F066A3F683E448661C1
:106D9000244F3F888669B6FBF7FC07FB1C66B5B23B
:106DA000214E06EBC502166836B90026066146611B
:106DB0001060012696802CE0194F86693F68F61B0B
:106DC000C661116820E0164F8E693F68F61BCE61E0
:106DD000C669CF69BE4209D90E690EB1096913E0CF
:106DE000002606614161086100210DE04E692EB95F
:106DF0000026466101614861106004E04B6943610F
:106E000001611861486100210029DCD19688761C57
:106E10009680D6889788BE4201DA9688D680F0BDE3
:106E200094030020003D0308C4BB0020002006E0BE
:106E3000054A02EBC0010022CA80421C90B2034AFC
:106E400012889042F4DB7047C4BB0020003D030869
:106E50001CB500BF53E001AB6A4600210846FDF7B0
:106E6000CFFA01A8FCF7D4FDFBF732F80646244818
:106E70000068401C224908600846006821490988CA
:106E8000B0FBF1F201FB12001FFA80FA1E4800EB82
:106E9000CA08D8F800404FF0000B21E0F4B1D4F854
:106EA00010901749A0690968884214D1204600F063
:106EB0002FF8208D022804D101212046FFF74EFF34
:106EC00002E0032084F82A00A56815B12046E16895
:106ED000A8474C4604E04FF0010B01E04FF0010BD6
:106EE000BBF1000FDAD0FAF7F3FF871B01A8FCF71C
:106EF000C7FD06480068874201D904480760AAE731
:106F000094030020003D0308C4BB00209003002030
:106F1000F0B5114E36888569B5FBF6F706FB1755B7
:106F2000ACB20E4D05EBC4021568854205D101696E
:106F3000116039B100254D6104E0416903690B61BD
:106F400003B15961012580F82A500025056145618A
:106F500095886D1E9580F0BD003D0308C4BB0020E0
:106F60000EB543E0224890F82A00F8B100202049ED
:106F700081F82A000120887704201E4908701E49E4
:106F8000D1F80100F9F7E2F9F9F7D6F9462190FBBB
:106F9000F1F201FB120000F596742146012009F080
:106FA000BBF94EF66021012009F0C8F908F05CFF3A
:106FB0000F4890F8290048B100200D4981F82900B8
:106FC000012088770B49087000F01AF808F02EFFAE
:106FD0000A480069401C0949086102A800211423DD
:106FE0000A46CDE900100846FDF78CFCBAE7000020
:106FF000EC060020D1020020DC060020B4060020B0
:107000003EB5002400254FF4A1612B48F9F7BFF9E4
:107010002A49012009F05CF908F036FF012102201D
:10702000FBF7F4FF4FF40031254801F0E5FA044680
:1070300024B90121084609F04BF93EBD214621A0A3
:1070400003F016F925480079012807D100212046D0
:1070500007F0A4FF22A003F00BF913E01F4800790A
:1070600002280FD121A003F003F923488461C4F35F
:10707000CF102149088404F07F0018B10846008C25
:10708000401C088400250BE008F020F802A800212D
:107090000B460222CDE900100846FDF733FC6D1CBB
:1070A000052DF1D307F0B0FE43F69821012009F039
:1070B000D3F800BFC1E70000049F0020A0BB0D0073
:1070C0000000020873656E6420746F74616C5F6207
:1070D000797465733D25640A00000000D102002028
:1070E000B0B4BCFCB4A5B7A20A000000C3FCC1EE5A
:1070F000B4A5B7A20A0000007C9D00200EB517E0E1
:1071000003F032FE0CF0E4FA09F014FC09F0F8FD8B
:107110000CF06AFC07488068401C0649886002A899
:10712000002114230A46CDE900100846FDF7EAFBCA
:10713000E6E70000B406002001490862704700003D
:1071400000000E4201460020034A506820F44040EF
:1071500008435060704700000010024029B1064A01
:1071600052690243044B5A6104E0034A5269824364
:10717000014B5A61704700000010024029B1064AD5
:10718000D2690243044BDA6104E0034AD2698243C4
:10719000014BDA61704700000010024029B1064A35
:1071A00092690243044B9A6104E0034A9269824364
:1071B000014B9A61704700000010024029B1064A55
:1071C000D2680243044BDA6004E0034AD268824387
:1071D000014BDA6070470000001002400348406A2B
:1071E00040F0807001494862704700000010024082
:1071F00030B500210022002400232D4D6D6805F0DC
:107200000C0121B1042905D0082923D105E0294D1D
:10721000056022E0274D05601FE0254D6D6805F4EF
:107220007012234D6D6805F48034022505EB9242FF
:107230001CB9214D554305600BE01D4D6D6805F4EB
:1072400000351DB11C4D5543056002E0194D5543F5
:10725000056002E0174D056000BF00BF144D6D686A
:1072600005F0F0010909154D6B5C0568DD404560CE
:107270000F4D6D6805F4E061090A104D6B5C4568BF
:10728000DD4085600A4D6D6805F46051C90A0B4DFB
:107290006B5C4568DD40C560054D6D6805F4404197
:1072A000890B074D6B5CC568B5FBF3F5056130BD17
:1072B0000010024000127A0000093D00F802002090
:1072C0000803002010B501460022002300204A11C7
:1072D000012A02D1094C236806E0022A02D1074C98
:1072E000236A01E0054C636A01F01F020124944007
:1072F0001C400CB1012000E0002010BD0010024035
:1073000000210B4A11700A4A203A82F82010012805
:1073100002D0042808D103E00121054A117004E0DD
:107320000521034A117000E000BF00BF7047000054
:107330002010024001490860704700003C044242AE
:107340000249096A0143014A116270470010024074
:10735000024909888143014A11807047042800408E
:107360000348008840F01000014908807047000081
:1073700004280040034800884FF6EF710840014997
:10738000088070470428004070B50024002500F0F4
:1073900081F83B490860084600683A49B0FBF1F4BF
:1073A00039480088A0423CD037490C8040F2B27581
:1073B00010E02846FBF794FD40B1B4F5B77F02D347
:1073C000A4F5B77404E0681C85B206E0A4F26D145D
:1073D000681C85B2B4F5B67FEBD800BF2B4885801A
:1073E000002516E029498888FBF77AFD30B1012D88
:1073F00004D11D2C01D31D3C09E00CE02448405D64
:10740000A04203D82248405D241A00E003E0681C33
:1074100085B21C2CE6D200BF681C1C498871601C18
:10742000C871174800681749B0FBF1F201FB12045C
:107430004FF46160B4FBF0F0144908704FF46160E0
:10744000B4FBF0F100FB11403C21B0FBF1F00F491F
:1074500048704FF46160B4FBF0F100FB11403C2137
:10746000B0FBF1F201FB1200084988700B46DA7993
:107470009979988800F02AF804490872002070BDB4
:107480003000002080510100340000201C07002043
:107490003C3B0308002103480188001F008841EAA3
:1074A000004070471C28004001460020064A128810
:1074B0000A40D0B2044A121F12880A4012B108B121
:1074C000012000E00020704704280040F0B503468A
:1074D0000C461546642093FBF0F0C6B2642093FB83
:1074E000F0F700FB1730C1B2132E02DD01F164008A
:1074F000C1B20846CF1701EB977701EBA707BAB2E5
:10750000072092FBF0F700FB172082B25719601E8C
:10751000DFF82CC01CF80000384482B2CF1701EB12
:107520009777BF10A1EB87071FB9032C01DA501E14
:1075300082B2072092FBF0F700FB1720C0B2F0BD2B
:10754000303B03080EB50120FFF7AEFF08B1FFF78F
:107550001BFF0220FFF7A8FFA0B10220FFF7F8FEF3
:10756000FFF712FF0A48807809494978084A1278DB
:10757000CDE9002102900648C3798279818805A06F
:1075800002F076FE0520FFF7E3FE00F023F90EBDC2
:107590001C070020416C61726D2054696D653A25AD
:1075A000642D25642D25642025643A25643A2564DC
:1075B0000A00000029B1064A12880243044B1A80CF
:1075C00004E0034A12888243014B1A80704700008E
:1075D000002800401CB5002401214FF0C050FFF7E7
:1075E000CDFD0120FFF7A8FD0420FAF7CFFB45F2FF
:1075F000510188423ED00120FFF782FE04E0601C6A
:10760000C4B20A2004F006FB4120FFF75BFE08B974
:10761000FA2CF4DBFA2C01DB01201CBD4FF4807046
:10762000FFF78EFE0120FFF785FE00F0D3F800F093
:10763000DBF801210846FFF7BDFF00F0CBF8FFF7AC
:107640008FFE47F6FF7000F0A5F800F0C3F80020A9
:10765000102117231A22CDE90010042140F2E57011
:1076600000F026F8FFF786FE45F251010420FAF7F4
:107670009BFB07E000F0B8F801210846FFF79AFFEE
:1076800000F0A8F800F004F8FFF77EFE0020C4E741
:1076900008B503208DF8000000208DF801008DF85A
:1076A000020001208DF803006846FBF7BBFC08BD13
:1076B0002DE9F05F06460F4690469946DDE90AAB94
:1076C000002440F2B270864203DB40F6330086426B
:1076D00002DD0120BDE8F09F40F2B2750AE02846C5
:1076E000FBF7FEFB10B12048044401E01F480444AE
:1076F000681C85B2B542F2DB781EC7B2002510E0E7
:107700001B48405D40F2A321484304EBC0143046BF
:10771000FBF7E6FB18B1012D01D116480444681CA3
:1077200085B2BD42ECDBA8F1010040F2A321484341
:1077300004EBC014C9EB4910C0EB092004EB0014A2
:10774000CAEB0A1004EB80045C4401214FF0C050E6
:10775000FFF714FD0120FFF7EFFC204600F00CF8C6
:1077600000F038F80020B5E70085E2018033E10140
:107770003C3B03088051010000B50246FFF7F0FDD5
:10778000100C03490880091D0A80FFF7F3FD00BDB6
:107790001828004000B50246FFF7E2FDC2F303409F
:1077A00003490880091D0A80FFF7E4FD00BD0000C1
:1077B0000828004010B5044601214FF0C050FFF7E3
:1077C000DDFC0120FFF7B8FC2046FFF7D5FF00F0F5
:1077D00001F810BD00BF0348008800F02000002819
:1077E000F9D0704704280040074800884FF6F77129
:1077F00008400549088000BF0348008800F00800E1
:107800000028F9D0704700000428004001460120FC
:107810007047000002460AB91F207047002111E09E
:107820000A4850F8310090420AD8084B481C53F8D7
:107830003000904204D9481C03EBC0000079ECE70B
:10784000481CC1B21529EBD300BFFEE7B43B0308C7
:107850002DE9F04107468C46DDE906450021032667
:107860000BB9082000E0002000EBC2001830012D09
:1078700002D14FF0020801E04FF00008A04400EBF5
:10788000C800BDE8F0810000014600200B2922D28B
:10789000DFE801F0060C12181B1D1F21090F15004F
:1078A00041F6846017E042F6B10014E043F6095057
:1078B00011E045F261100EE047F612200BE04AF2AB
:1078C000C32008E04FF2244005E0044803E00448E8
:1078D00001E0044800BF00BF7047000048E8010015
:1078E00090D0030020A107002DE9F04F0446164672
:1078F000DDE909C806F104094FF0000A0025002758
:10790000052901D0062902D10C2B00DA0C231CB961
:107910000B2905D00C2903D0012C03D10C2901D14E
:107920004FF0010A0B9808B1102000E0002000EB96
:10793000C8004FF0040B0BFB1100BCF1000F02D08C
:107940004FF0000B01E04FF0140B00EB0B05062984
:1079500001D88A0007E00835BAF1010F02D1881E6C
:10796000820000E08A00002D00DA0025A818401EE1
:1079700090FBF2F000FB093000F10C07062900D85B
:10798000BF1CB800401CA1F1020B4FF0010E0EFA13
:107990000BFE00FB0EF0BDE8F08F00B501F00AF918
:1079A000042804D0052804D0072806D103E00220CB
:1079B00000BD0120FCE70320FAE70020F8E700B54E
:1079C00001F0E6F8C01C00BD10B504461048046084
:1079D00001F0D0F90F4801F0B9F9002001F0B6FE2E
:1079E000012001F010FE0021084601F045FC0421B1
:1079F000002001F0EBFE00231A464FF6FF71084607
:107A000001F0A4FC01F052FF00200349087010BDF2
:107A1000B80100208D7C0208B501002038B5002493
:107A200072480078012804D071480AF02BFC002825
:107A30007ED06E480078012802D100206B49087082
:107A400001F0AAF80446204601F053F804F00100C2
:107A500078B101F07BFF012001F030FD654800683E
:107A600038B164480068006818B16249096808685C
:107A7000804704F0020002284AD104F04000402868
:107A800012D15D48007810B9012001F017FD594866
:107A9000006800283CD0574800680069C0B35549C9
:107AA00009680869804733E001F0D4FB5248007848
:107AB00090B9012001F002FD002140F6021001F012
:107AC000D0FF40F6441001F056FB40F00205294675
:107AD00040F6441001F0C5FFFF226946474801F017
:107AE000BBF8474801F06CF84248006878B141485B
:107AF0000068806858B1424890F90D3090F90C2028
:107B00003C4800689DF8001085683C48A84700BFC5
:107B100004F08000802811D1012001F0CFFC35480D
:107B2000006858B133480068806938B1314800E0D6
:107B30005BE000688169C4F30020884704F40070AA
:107B4000B0F5007F28D101F035F8042810D101F0FC
:107B5000FDFE012001F0B2FC26480068E0B1254896
:107B600000684068C0B1234909684868804713E04D
:107B700001F020F805280FD101F06CFB012001F085
:107B80009DFC1C48006838B11A480068C06818B1EC
:107B900018490968C868804704F00400042804D123
:107BA00001201449096881F8240004F0100010280D
:107BB00004D101200F49096881F8250004F0200054
:107BC000202812D101F046FB0B48007810B90120A3
:107BD00001F074FC0748006838B106480068C068C6
:107BE00018B104490968C868804738BDB50100204C
:107BF0001D020020B8010020B4010020F83400204C
:107C0000E43400202DE9F0478AB080460C46154642
:107C10001E464FF001094FF0000A0027002000F037
:107C20000DF9404600F0E8F8012000210691079187
:107C3000CDE9081002910391049103200B464FF403
:107C40001672CDE9004005912146002000F03AF976
:107C5000002000F067F8012000F094FF00BF0CE066
:107C6000002000F059F88246AA4502DD4FF00009D5
:107C700005E0012000F086FF7F1CB742F0D300BF73
:107C800000F038FB48460AB0BDE8F0870121014A00
:107C900011707047B501002010B504460548006812
:107CA00038B104480068C06818B102490968C8685A
:107CB000804710BDB801002010B504460548006893
:107CC00038B104480068406818B10249096848683A
:107CD000804710BDB801002010B50024012000F03D
:107CE000ADF800231A461946184601F02FFB00F0A4
:107CF000CAFF0446204610BD10B50446A0B201F0EC
:107D00003AFA10BD70B504460D461646A0B232468A
:107D1000294601F03AFA70BD10B5044600F0E7FFBD
:107D200010BD000010B5044600231A464FF6FF713F
:107D3000084601F00BFB24B1204601F0E1FC01F004
:107D40007DFA07480078012804D16FF07F4001F0E8
:107D50008CFC04E003490968880101F086FC10BD31
:107D6000B4010020B001002010B5044600231A46DB
:107D70004FF6FF71084601F0E9FA24B1204601F000
:107D8000BFFC01F05BFA07480078012804D16FF0CE
:107D90007F4001F07EFC04E003490968880101F09E
:107DA00078FC10BDB4010020B001002070B505467C
:107DB0000C4600231A4640F20121084601F0C6FA9B
:107DC00000F044FF012802D10948C47301E00848CB
:107DD0000472074801F08CFB00222146284601F07E
:107DE0003FFA0448006801F037FD01F0A3FD70BDC3
:107DF000F8350020AC01002010B50446204601F003
:107E000009FC10BD70B505460C46012D06D1094888
:107E100004700948C47301F06BFB09E00648C0799F
:107E2000012805D1034804700348047201F060FB87
:107E300070BD0000A8010020F835002010B50446F0
:107E400014B1012C07D000BF002001F0C5FB0020B9
:107E50000A49487010E0012001F0BEFB0748407855
:107E600006490978884206D00448007803494870DA
:107E7000487800F005F800BF00BF10BDB601002033
:107E800010B504460E48047044700120FFF7D6FF79
:107E9000012C0AD134214FF4E86001F0E2FD4421C5
:107EA00040F2417001F0DDFD09E014214FF4E8607B
:107EB00001F0D7FD242140F2417001F0D2FD10BD48
:107EC000B60100202DE9FE4F80460D461446994626
:107ED000DDF844B0DDE90EA70D9E7AA103C9CDE916
:107EE00001017A49159808701598012801D14FF0C1
:107EF000000A012F03D176491098087002E0FF2094
:107F000073490870B8F1000F03D0B8F1010F57D1D1
:107F100057E0002001F02BFC00206E4981F828007A
:107F20000846C4620B2180F834106800FFF772FC29
:107F30000146684880F835100020664908704FF601
:107F4000FF7000EAC60048800421624801711821D0
:107F500041710021817187F00101C1715C48017894
:107F60005C480172BBF1010F02D1F221417202E0C3
:107F700001215848417201215648817200F0CAF926
:107F8000544991F8281009B1012100E00021084668
:107F9000FFF754FF4F48283001F028FA4D4801F010
:107FA000A7FA01A801F0EAFB40F2FF1001F05AFC29
:107FB0004FF4FA500AFB00F0B0FBF4F046490860B9
:107FC0007DE0002001F0D3FB0120424981F8280028
:107FD000084680F838404148415D3E4880F83910F5
:107FE00080F83A901DB90B2C05D00C2C03D0012D34
:107FF00006D10C2C04D10121364880F83B1003E057
:108000000021344880F83B100120324908700846AE
:1080100090F83800052804D0084690F83800062863
:1080200008D10C2E03DA0C212A48818104E029486A
:10803000868101E027488681264887732448017895
:108040002448C17380F810B01499417400F062F9AB
:10805000204991F8281009B1012100E000210846CB
:10806000FFF7ECFE1B48283001F0C0F9194801F079
:108070003FFA0AF0FF0001F08EF91648407C012813
:108080000CD140F2367001F076F820F00400014681
:10809000009040F2367001F0E4FC0BE040F23670E4
:1080A00001F069F840F004000146009040F236709B
:1080B00001F0D7FC4FF6FF700749086000BF00BF12
:1080C000BDE8FE8FC194C10000000000B401002093
:1080D000A8010020F8350020B0010020643C03080E
:1080E00070B504460D462946204601F0EBFA70BDF6
:1080F0002DE9FE4F0746884691461C46DDE90FAB49
:108100000E9E0C9D69A103C9CDE9010117B1012F94
:108110004AD14AE00020674981F828000846C56234
:108120000B2180F834106000FFF774FB01466148B2
:1081300080F83510C0F8309000205E4908704FF686
:10814000FF7000EAC600488004215A4801711821D6
:108150004171002181718AF00101C171BBF1010FF0
:1081600002D1F221417202E0012152484172012103
:108170005048817200F0CEF84E4991F8281009B1AC
:10818000012100E000210846FFF758FE4948283049
:1081900001F02CF9474801F0ABF901A801F0EEFA23
:1081A00040F2FF1001F05EFB57E00120414981F8E9
:1081B0002800084680F838503F48015D3D4880F867
:1081C00039100D9980F83A101CB90B2D05D00C2DE3
:1081D00003D0012C06D10C2D04D10121354880F8A3
:1081E0003B1003E00021334880F83B100120314967
:1081F0000870084690F83800052804D0084690F822
:108200003800062808D10C2E03DA0C212948818178
:1082100004E02848868101E026488681254880F8C8
:108220000EA0264801782348C17380F810B0139936
:10823000417400F06FF81F4991F8281009B101212D
:1082400000E000210846FFF7F9FD1A48283001F048
:10825000CDF8184801F04CF900BF00BF012F11D133
:10826000144890F8390006280CD140F6890000F037
:1082700082FF20F004000146009040F6890001F0E2
:10828000F0FB0BE040F6890000F075FF40F00400C1
:108290000146009040F6890001F0E3FB404601F002
:1082A000DDF9074914980860BDE8FE8FC194C1004C
:1082B00000000000F8350020643C0308A8010020FD
:1082C000AC0100202DE9F04106460C4615464FF45E
:1082D0007A7005FB00F7304601F09CF9204601F06A
:1082E000BDF901F069FA384601F0B6FA01F022FB57
:1082F000BDE8F08108B5002000909DF8000020F056
:108300000400001D0090009801F000FA022000F027
:1083100039FC08BD10B5002001F018FA10BD10B5E9
:1083200000231A464FF4C071084601F00FF800F020
:10833000B0FF10BD2DE9FE4F81460E4615461F4683
:10834000DDE90EAB4FF000080124B9F1000F03D0B6
:10835000B9F1010F21D10DE0CDE900AB3946284636
:10836000DDE90C23FFF774FA4FF47A7100FB01F892
:108370002C4612E00D988DE8010C3A46294630460D
:108380000C9BFFF7B1FA4FF47A7100FB01F8074933
:10839000885DFFF779FA044600BF00BF08EB0400D0
:1083A000401EB0FBF4F0BDE8FE8F0000643C030803
:1083B0002DE9F34F91B000201090119810B10128D1
:1083C00053D153E07B49C86AF8F7C8FBCDE90A01ED
:1083D0001298F8F7C3FBCDE9060176494A88497936
:1083E00002EBE100F8F7A9FBCDE904017148C0797F
:1083F00010B90020034601E000206F4B0246CDE992
:108400000203DDE90401F8F702FA8046DDE90623FC
:10841000F8F7FDF9CDE908016648407A022803D152
:1084200000204FF0804101E0002001468046424696
:108430000B46DDE90801F8F7EAF9824600225F4BB6
:10844000F8F78CFA0646DDE90A23F8F7F9FA002274
:108450005B4BCDE90C01F8F781FACDE90E0109F08B
:1084600061F80446F8F787FB10909DE0514890F8BA
:108470003900001F00EB4000524901EB00114D484C
:1084800090F83800C0F10C0001EBC00003C8CDE942
:108490000E0148498889F8F761FB044600224A4BDF
:1084A000F8F7B5F90646DDE90E23F8F757FACDE9F6
:1084B0000C01404991F83A10CA17059101EB9271ED
:1084C0008A100599A1EB8201081DF8F736FBCDE96A
:1084D0000201384991F8382091F83B10002901DD5C
:1084E000022100E00021511A8800F8F726FB064619
:1084F0000F461299CA002F4991F83810042303FB44
:1085000011221C322B49097C102303FB012229492B
:10851000897B012901D1142100E00021501AF8F7CC
:108520000CFB32463B46CDE90001F8F789FA82465A
:1085300002F0B2FE0446DDE90223F8F70FFA8046A6
:1085400089460022134640464946F8F741FB02D2CD
:108550004046494601E000200146044622460B46BB
:1085600000201649F8F753F9CDE90A01DDE90E2399
:10857000DDE90A01F8F7F2F9CDE90801DDE90823A0
:10858000DDE90C01F8F743F9CDE906010F4A104B7C
:10859000DDE90601F8F73BF9044604F095F90646D3
:1085A000F8F7E9FA109000BF00BF109813B0BDE8CB
:1085B000F08F0000F83500200000F03F0000204060
:1085C00000408F4018010020000011402B8716D971
:1085D000CEF7EF3F70B504460D46A0B2294601F034
:1085E00040FA70BD70B504460D461646A0B232463C
:1085F000294601F03EFA70BD2DE9F34F8BB00546D8
:108600000024182105A8F7F7C2FE0020049003906B
:1086100029465BA001F02CFE28460C99F9F7CDFF06
:108620000446281950F8147C3B462246214657A0A0
:10863000009701F01DFEB4F5003F05D921465CA06E
:1086400001F016FE002497E029464DA001F010FE2F
:10865000281950F8049C281950F808AC281950F82B
:108660000C6C281950F8147C281950F810BC3346AB
:108670005246494654A0CDE9007B01F0F9FD62481D
:1086800082453ED1614883453BD161A001F0F0FDB8
:1086900007F11400844205D063A001F0E9FD012038
:1086A000039030E065480068B0420BD064A001F050
:1086B000DFFD62483146026865A001F0D9FD012066
:1086C000039020E001214020FEF748FDF9F73AFC35
:1086D000201F81082846F9F71DFCF9F72DFC80467C
:1086E00000214020FEF73AFD424649465EA001F0D7
:1086F000BFFDC14507D064A001F0BAFD0120039081
:1087000001E0012003900398002835D005943F48EC
:1087100006904A48006807903B48089028191022A4
:1087200005A9F9F721FF04905AA0049901F0A0FDD2
:10873000143401214020FEF711FDF9F703FC201F3E
:1087400081082846F9F7E6FBF9F7F6FB8046002199
:108750004020FEF703FDCDF8148053A0059901F0E9
:1087600087FD2919081F042205A9F9F7FDFE0490C9
:1087700050A0049901F07CFD20460DB0BDE8F08FBB
:10878000616464723D253038780A00006461746168
:108790006C656E3D253038782C25753B2066696CFC
:1087A000656C656E3D253038782C25750A00000013
:1087B000C9FDBCB6B0FCB3A4B6C8B3ACB9FD313288
:1087C000384B3A2025640A00637263566C3D2530AD
:1087D00038782C666978436861723D253038782C8A
:1087E00066696C655665723D253038782C66696C13
:1087F000656C656E3D253038782C745F61646472F9
:108800003D253038780A0000574A425700000208D8
:10881000C9FDBCB6B0FCB0FCBAACC1CBBAF33230C7
:10882000D7D6BDDA0A000000C9FDBCB6B0FCB3A4BF
:10883000B6C8D0A3D1E9B4EDCEF30A00EC0600200F
:10884000B9CCBCFED0C5CFA2B4EDCEF30A00000077
:1088500066696C657665723D253038782C6170707C
:108860003D253038780A0000726561645F63726389
:108870003A253038782C206765745F6372633A2537
:108880003038780A0000000063726320B4EDCEF344
:108890000A000000666972737420666C6167203D8F
:1088A0002025640A000000006372633D253038789B
:1088B0000A0000007365636F6E6420666C61672058
:1088C0003D2025640A00000070B500240025082022
:1088D000F9F75CFA044621461DA001F0C9FC2046C8
:1088E0000AF08CFF40B3E0B282280BD100210820AF
:1088F000F9F75AFA2A200AF08DFF0120184981F869
:108900002A0023E0E0B283280BD100210820F9F7E8
:108910004BFA2B200AF07EFF0120114981F82A0032
:1089200014E000210820F9F73FFA0C20F9F72EFA9D
:1089300005460C490D7009E000210820F9F734FACA
:108940000C20F9F723FA054606490D7070BD0000AA
:108950000A424B505F4452323A253034780A0000C4
:10896000EC060020D00200202DE9F043002600276D
:10897000B046B146002009F0CBF90746012009F0C6
:10898000C7F98046002414E000250EE004EB8400C3
:108990000F4901EB401005EB850100EB0110007859
:1089A000012800D18146681CC5B2022DEEDB601C97
:1089B000C4B2022CE8DB3FB9B8F1000F04D1B9F121
:1089C000000F01D1002600E001263046BDE8F0830B
:1089D0003893002021B1028842F04002028004E076
:1089E00002884FF6BF731A4002807047024600208B
:1089F00013890B400BB1012000E0002070470146B5
:108A0000888970478181704710B50022028802F47E
:108A100041520B884C8823438C882343CC882343C2
:108A20000C8923434C8923438C892343CC892343DA
:108A30001A430280838B4FF2FF74234083830B8A97
:108A4000038210BD704770477047000038B5044678
:108A50001B48844206D9E1208DF80000E9208DF8FA
:108A6000010026E01748844206D9D7208DF800007F
:108A7000DB208DF801001CE01348844206D9C12098
:108A80008DF80000C5208DF8010012E00F488442E7
:108A900006D975208DF8000081208DF8010008E0CE
:108AA0000B48844205D96B208DF800006F208DF8AB
:108AB000010002226946982000F0B3FF38BD000093
:108AC00000E9A43580F8A9328044E52D000B6B1B2A
:108AD00040FC541910B500F06DF818B100F06AF8B8
:108AE000062803D100F05CFFFFF7AEFF00F034FF73
:108AF00010BD38B50446200A8DF80000E0B28DF8AC
:108B0000010002226946104600F08BFF38BD0000CC
:108B10002DE9FF4F81B081468A461C4600231A4644
:108B20004FF4C071084600F011FC4FF47A7104FB59
:108B300001F0F8F713F807460022084BF7F780FF1B
:108B40000546F8F718F80023009051464846039A66
:108B500000F0A9FB05B0BDE8F08F000000402F40F9
:108B600010B5014643F60950B1FBF0F202FB1013B9
:108B7000401000EB833043F60954B0FBF4F000EBF7
:108B8000823010BD10B50446A0B203F043F810BD0A
:108B9000002070470220704708B502226946122063
:108BA00000F0C3FA9DF801009DF8001040EA012092
:108BB00008BD00000148007870470000BC0100209B
:108BC00038B5044603226946142000F0AEFA00F0DE
:108BD0003DF82070207820B1012814D00F2828D12A
:108BE00028E09DF8000020719DF8010040424010EF
:108BF00041B2A1719DF802004042401041B2617142
:108C00000021A1601DE09DF800004042401041B2EB
:108C100021739DF8010040B2801C811061739DF8A2
:108C200002004042401041B2A1730748016821612F
:108C300007E000BF14212046F7F7A9FB0F202070A2
:108C400000BF00BF38BD00000C01002001480078C3
:108C50007047000008010020F8B505460C4616468E
:108C6000002000906946204600F050F82078B0427D
:108C700001DD0120F8BD227829469DF8000000F0B2
:108C80002FFA0020F6E738B50020009000240025D8
:108C900040F6E20000F06FFA044624F0010140F6CD
:108CA000E20000F0DEFE40F6E50000F064FA054662
:108CB00025F0800140F6E50000F0D3FE6FF07F4024
:108CC00000F0D3FC0422694640F6190000F05DFA7A
:108CD000002000F03BFD214640F6E20000F0C1FE1E
:108CE000294640F6E50000F0BCFE009838BD38B5D6
:108CF000002401226946152000F017FA9DF80000B3
:108D00004042401044B2204638BD000038B5044609
:108D10000D4602226946132000F007FAFFF796FF7E
:108D2000012809D108480078012805D140F20270D5
:108D300000F021FA207002E09DF8000020709DF8FC
:108D40000100287038BD00000901002010B504465C
:108D500000F044FA204600F06BF800F021FE0020FD
:108D600000F0F4FC00F0A9F800F0A2F8012000F0F7
:108D7000A5FB10BD38B5FF2401215820FEF70EFADF
:108D800003208DF8020048208DF803001020ADF874
:108D9000000069461748F9F795FC04208DF8030098
:108DA0000220ADF8000069461348F9F78BFC4FF438
:108DB0000070ADF8000069461048F9F783FC4FF4E5
:108DC0008060ADF8000069460C48F9F77BFC202074
:108DD000ADF8000069460748F9F774FC00F0E2FEC0
:108DE00004461CB106A001F043FA02E009A001F01C
:108DF0003FFA38BD00100140000C0140001801404E
:108E00007370693120696E6974206572726F720DBA
:108E10000A000000535831323678496F496E697440
:108E200020696E6974207375636573730D0A0000A1
:108E30001FB5044601214820FEF7B0F903208DF844
:108E40000E0028208DF80F004FF48070ADF80C0054
:108E500003A91648F9F736FC01210846FEF79EF9EA
:108E600008210420F9F70EFC4FF4807001900020D7
:108E70008DF8080008208DF8090001208DF80A00FF
:108E800001A8F9F729FA17208DF8000000208DF8C5
:108E9000010001208DF802008DF803006846FAF702
:108EA000C1F84FF48070F9F7FDF91FBD00180140BB
:108EB00010B5012000F043FA10BD704770B50446AC
:108EC0000020234908702349086B8047214622A0CF
:108ED00001F0CEF99CB30020234908702348807F1D
:108EE000012830D122480078022813D12048407848
:108EF00008280FD1F7F720FA462190FBF1F201FB89
:108F0000120000F5FA752946012007F0B7F9022092
:108F100006F04AF916480078042814D1F7F70CFA3D
:108F2000462190FBF1F201FB120000F5FA7529468B
:108F3000012007F0F1F9022006F036F903E0FFE71F
:108F400001200949087008200A49087070BD000016
:108F5000E4010020483B0308636164446F6E6520B0
:108F600025640D0A0000000038020020EC060020F5
:108F7000D1020020E00100202DE9F84305460C460F
:108F80001746984600263B46224617A10020CDF8FA
:108F9000008007F00BFE1D49086B804723462A46D8
:108FA0001BA1002002F028FE012006F003FA06466D
:108FB00086B154B1224629463046F7F7CFF922460A
:108FC0003146012006F0B8F908E03146012006F0EC
:108FD00025FA03E03146012006F020FA00200F496F
:108FE0000870BDE8F88300005278446F6E65207306
:108FF000697A653A2564203C727373693A25642C5A
:1090000020736E723A25643E200D0A00483B030827
:109010006C6F72612072637600000000E001002036
:1090200010B505A001F024F90949086B804700201C
:109030000849087010BD000052784572726F7220A6
:109040007265747279207265636976650D0A000035
:10905000483B0308E001002010B505A001F008F925
:109060000A49086B804700200949087010BD0000BC
:10907000527854696D656F757420726574727920C9
:109080007265636976650D0A00000000483B0308BD
:10909000E001002010B50449086B80470020034917
:1090A00008700349087010BD483B0308E001002028
:1090B000E501002010B505A001F0DAF80649086BBB
:1090C000804700200549087010BD0000547854699D
:1090D0006D656F75740D0A00483B0308E0010020C0
:1090E0002DE9F04107460D4616460024FFF7F2FC35
:1090F000002000F0D3F91E2000F0D1FB384600F02C
:10910000CEFB002000F0CBFB00BF05E0002000F00C
:10911000C6FB2855601C84B2B442F7DB012000F086
:10912000BDF900F019FCBDE8F0812DE9F0410746DA
:109130000D4616464FF000080024FFF7CBFC002038
:1091400000F0ACF9384600F0AAFB002000F0A7FBC5
:10915000804600BF05E0002000F0A1FB2855601C00
:1091600084B2B442F7DB012000F098F900F0F4FB80
:109170004046BDE8F08138B50446012269462046E4
:1091800000F003F89DF8000038BD2DE9F0410446D9
:109190000E4617460025FFF79DFC002000F07EF9E3
:1091A0001D2000F07CFB200A00F079FBE0B200F00B
:1091B00076FB002000F073FB00BF05E0002000F00C
:1091C0006EFB7055681C85B2BD42F7DB012000F0D4
:1091D00065F900F0C1FBBDE8F081000008B50A2088
:1091E000FFF7D0FC01210820FDF7D8FF03208DF800
:1091F000020010208DF803000120ADF80000694640
:109200000D48F9F75FFA002201210B48F9F73BFB03
:109210001420FFF7B7FC012211460748F9F733FB8A
:1092200048208DF8030069460348F9F74BFA0A20F5
:10923000FFF7A8FC08BD0000000C014003480068CF
:109240000349886001200870704700000401002075
:10925000D83400200020014908707047D83400201D
:1092600070B505460E4614463146284600F0C2F950
:10927000204600F08DFA70BD38B505460C468DF8D5
:1092800000508DF80140022269468F2000F0C9FB92
:1092900038BD10B500221146C52000F0C2FB0720E2
:1092A00000F00CF910BD2DE9FC4105460E46904634
:1092B0001F46089C8DF800508DF801608DF80280E3
:1092C0008DF80370200C8DF80400200A8DF805003D
:1092D000E0B28DF8060007226946882000F0A1FB65
:1092E000072000F0EBF8BDE8FC8138B50446200A01
:1092F0008DF80000E0B28DF80100FFF7A7FC30B94F
:109300000222694640F2BE6000F0B3FB00E000BFFD
:1093100000BF38BD38B50446200A8DF80000E0B221
:109320008DF80100FFF792FC30B90222694640F245
:10933000BC6000F09EFB00E000BF00BF38BD01B57F
:10934000012269469D2000F06CFB08BD2DE9FC411F
:1093500007460C4615461E46380A8DF80000F8B23E
:109360008DF80100200A8DF80200E0B28DF80300AC
:10937000280A8DF80400E8B28DF80500300A8DF84F
:109380000600F0B28DF8070008226946104600F08A
:1093900048FBBDE8FC81F8B50646F82E01DDF82053
:1093A00000E03046401C441000250020009003E0FF
:1093B000E01C8410681CC5B21F2CF9DC6800401C3E
:1093C00004FA00F0C0B2009001226946A02000F02B
:1093D00028FB4EB105EBC400C0B200909DF8001010
:1093E00040F2067000F03DFBF8BD00007CB504467D
:1093F00000250020009001902078264909788842B5
:1094000002D0207800F0E8F8207820B1012829D097
:109410000F283AD13AE008261F496068B1FBF0F501
:10942000280C8DF80000280A8DF80100E8B28DF8AC
:109430000200207B8DF80300607B8DF80400A0689B
:10944000FFF78EFB0546280C8DF80500280A8DF8DD
:109450000600E8B28DF80700324669468B2000F01E
:10946000E0FA14E00426207C8DF80000607C8DF882
:109470000100A07C8DF80200E07C8DF803003246EC
:1094800069468B2000F0CDFA01E000BF7CBD00BF33
:1094900000BFFBE7080100200000093D10B50446AD
:1094A00024B110210448F9F7ECF903E01021024837
:1094B000F9F7E5F910BD0000000801400149087006
:1094C00070470000BC010020F8B504460D46164662
:1094D0001F468DF800408DF801508DF802608DF820
:1094E000037004226946952000F09BFAF8BD000045
:1094F000FEB50446002600200090019002902078DE
:1095000033490978884202D0207800F065F8207845
:1095100020B101283AD00F284FD14FE0607AF128CE
:1095200009D14FF6FF70FFF7F5FE48F20500FFF78F
:10953000DCFE02260DE0607AF22809D141F60F50D8
:10954000FFF7E8FE41F22100FFF7CFFE062600E01C
:10955000667A09256088000A8DF80000A0788DF8E9
:10956000010020798DF8020060798DF80300A07960
:109570008DF80400E0798DF80500207A8DF806005A
:109580008DF80760A07A8DF8080018E00625A089FC
:10959000000A8DF80000207B8DF80100A07B0D49AA
:1095A00008708DF80200E07B8DF80300207C8DF8B8
:1095B0000400607C8DF8050001E000BFFEBD00BF27
:1095C0002A4669468C2000F02CFA00BFF6E700001E
:1095D000080100200901002001B59DF800000449A0
:1095E0000870012269468A2000F01BFA08BD0000BD
:1095F0000801002070B504460D462A462146002089
:1096000000F0EEF970BD01B501226946962000F028
:1096100008FA08BD38B5054600240F48007828B977
:109620002846FFF713FA01200B4908702846FFF778
:1096300097FA0446200E8DF80000200C8DF80100EA
:10964000200A8DF80200E0B28DF80300042269467A
:10965000862000F0E6F938BD1001002010B5044660
:109660000221204600F0B2F810BD38B504460520AE
:10967000FFF724FF200C8DF80000200A8DF8010070
:10968000E0B28DF8020003226946822000F0C9F999
:1096900038BD38B504460520FFF710FF962140F687
:1096A000AC0000F0DEF9200C8DF80000200A8DF8E7
:1096B0000100E0B28DF8020003226946822000F02A
:1096C000B0F938BD7CB505460C46280C8DF8000075
:1096D000280A8DF80100E8B28DF80200200C8DF800
:1096E0000300200A8DF80400E0B28DF80500062280
:1096F0006946942000F095F90620FFF7DFFE7CBD57
:109700000149486070470000D834002001B582B09C
:1097100000200190FFF797F99DF80800C0F3800042
:1097200080009DF80810C1F3400140EA41009DF817
:10973000081001F0010108430190012201A98420D1
:1097400000F06FF90020FFF7B9FE0EBD01B5012250
:109750006946802000F065F99DF8000018B90120E5
:10976000FFF7ACFE02E00220FFF7A8FE08BD01B53E
:10977000012269469F2000F054F908BD10B5044647
:10978000082221464FF4D86000F073F9002010BD84
:1097900038B504460420FFF791FE200C8DF8000038
:1097A000200A8DF80100E0B28DF80200032269461C
:1097B000832000F036F938BD10B500221146D120C3
:1097C00000F02FF90420FFF779FE10BDF8B504462C
:1097D0000D46FFF7DFF9012818D10F2C06D1012320
:1097E0001A4600210620FFF76FFE05E001231A4606
:1097F00000210420FFF768FE0E2C01DB0E241FE081
:1098000014F1110F1CDA6FF0100419E040F6D800C3
:10981000FFF7B1FC40F01E06314640F6D80000F0DC
:1098200020F90123002207210420FFF74DFE162C0A
:1098300001DD162404E014F1090F01DA6FF00804C9
:10984000E0B28DF800008DF80150022269468E20AA
:1098500000F0E7F8F8BD00000149486070470000DB
:10986000CC34002070B504460025FFF7EFF998B915
:109870004FF4D760FFF77FFC00F0FE05C4F3002033
:10988000054329464FF4D76000F0EBF8E1B240F20F
:10989000B96000F0E6F800E000BF00BF70BD10B591
:1098A00004462046F9F760F810BD00001FB50121FD
:1098B0000220FDF763FC1D208DF8000003208DF8C9
:1098C00001008DF8020001208DF803006846F9F7C9
:1098D000A9FB0A20ADF808001248006842F2107196
:1098E000B0FBF1F080B2ADF804000020ADF80A0042
:1098F000ADF8060001A90C4800F0C0FA00200B49A1
:1099000008700B4908700121074800F090FA012106
:10991000054800F089FA01221146034800F0A4FA34
:109920001FBD0000E402002000040040CC340020F1
:10993000D83400200348006803498860012008707B
:109940007047000004010020CC34002000200149B1
:1099500008707047CC34002010B500240BE020467E
:10996000641CB0F57A7F03D906A000F081FC0024C6
:109970000120FFF707F910210848F8F777FF0128C1
:10998000EDD010BD776169742062757379207069BC
:109990006E2074696D656F75740D0A0000100140CA
:1099A00010B50020FFF77AFDC020FFF778FF0446CE
:1099B000214607A000F05CFC0020FFF770FF0120AB
:1099C000FFF76CFDFFF7C8FF0120FFF777FD10BD23
:1099D000737461747573203D2025640D0A000000C6
:1099E0002DE9F04107460D4616460024FFF772F8B0
:1099F0000020FFF753FD0E20FFF751FF3846FFF719
:109A00004EFF00BF04E0285DFFF749FF601C84B2F1
:109A1000B442F8DB0120FFF741FDFFF79DFFBDE8F1
:109A2000F0812DE9F04105460E4617460024FFF768
:109A300051F80020FFF732FD2846FFF730FF00BF46
:109A400004E0305DFFF72BFF601C84B2BC42F8DB02
:109A50000120FFF723FD842D01D0FFF77DFFBDE836
:109A6000F08113B50446012201A9204600F001F857
:109A70001CBD2DE9F04104460E4617460025FFF7B0
:109A800029F80020FFF70AFD0D20FFF708FF200A44
:109A9000FFF705FFE0B2FFF702FF00BF04E0705DD3
:109AA000FFF7FDFE681C85B2BD42F8DB0120FFF721
:109AB000F5FCFFF751FFBDE8F08110B500F002F8AA
:109AC00010BD00000CB500200190009033480068E4
:109AD00040F480303149086000BF3048006800F42D
:109AE000003000900198401C0190009820B94FF67A
:109AF000FF7101988842F0D12848006800F40030D6
:109B000010B10120009001E0002000900098012891
:109B100043D12348006840F01000214908600846FE
:109B2000006820F0030008600846006840F002006A
:109B300008601A484068194948600846406848600B
:109B40000846406840F4806048600846406820F459
:109B50007C1048600846406840F4E81048600846B9
:109B6000006840F08070086000BF0C48006800F09A
:109B700000700028F9D00948406820F00300074928
:109B800048600846406840F00200486000BF034853
:109B9000406800F00C000828F9D10CBD001002400C
:109BA0000020024000B587B001210803FDF7F6FA56
:109BB00001210420FDF7F2FA03208DF81A00182085
:109BC0008DF81B00E020ADF8180006A91E48F8F734
:109BD00079FD0020ADF804004FF48270ADF8060066
:109BE0000020ADF80800ADF80A00ADF80C004FF405
:109BF0000070ADF80E002020ADF810000020ADF888
:109C000012000720ADF8140001A91048FEF7FCFE71
:109C100001210E48FEF7DEFE01210420FDF7BEFA09
:109C200003208DF81A0010208DF81B00ADF81800E5
:109C300006A90548F8F746FD10210348F8F721FE6C
:109C4000002007B000BD00000008014000300140C6
:109C500010B5F9F761FBFAF74DFFF9F773FB074809
:109C60000068401C05490860054802684068521CAD
:109C700040F1000002490A60486010BD2000002049
:109C80002800002030B585B06846FDF7B1FA4FF4E2
:109C90007A720098B0FBF2F1B1F1807F00D31DE041
:109CA00021F07F40401E4FF0E022506150170F22FC
:109CB000002807DA13071D0E094B00F00F04241FBC
:109CC0001D5503E013071C0E064B1C5400BF00205B
:109CD0004FF0E02290610720106100BF05B030BD59
:109CE00018ED00E000E400E010B51148006840F015
:109CF00001000F490860084640680E4908400C49B9
:109D00004860084600680C49084009490860084650
:109D1000006820F4802008600846406820F4FE00B7
:109D200048604FF41F008860FFF7C7FE10BD0000B9
:109D3000001002400000FFF8FFFFF6FE10B50024FF
:109D400001212A4800F07FF800284ED028480068FA
:109D5000401C274908600121244800F065F8254887
:109D60000078F8B12348806821490968884205D8FD
:109D7000204880681E4909680C1A06E01D48806862
:109D8000C0F1FF301A49096844181A484068A042D7
:109D900008D2FFF7DBFD16480068164988600020EE
:109DA000FDF78AFF14480078F8B11348806810491D
:109DB0000968884205D8104880680D4909680C1A5E
:109DC00006E00D488068C0F1FF3009490968441871
:109DD00009484068A04208D2FFF73CFA04480068EE
:109DE000054988600020FDF757FF10BD00040040C2
:109DF00004010020CC340020D834002010B501210B
:109E0000074800F020F850B106480068401C05499A
:109E1000086006F0E7FF0121014800F005F810BDD9
:109E200000080040F4000020CA430282704721B1BC
:109E3000028842F00102028004E002884FF6FE73BD
:109E40001A400280704730B50246002000230024EB
:109E5000158A05EA0103958905EA010413B10CB1DD
:109E6000012000E0002030BD1AB183890B438381BB
:109E700002E083898B4383817047000000220288BF
:109E80001D4B98420ED01D4B98420BD0B0F1804F25
:109E900008D01B4B984205D01A4B984202D01A4B5F
:109EA000984204D14FF68F731A404B881A43174BD0
:109EB000984207D0164B984204D04FF6FF431A4001
:109EC000CB881A4302808B8883850B8803850A4BD5
:109ED00098420BD0094B984208D00E4B984205D0BF
:109EE0000D4B984202D00D4B984201D10B7A03865C
:109EF0000123838270470000002C014000340140A0
:109F00000004004000080040000C00400010004029
:109F1000001400400040014000440140004801405E
:109F200010B500F00BF803490860084600680249C4
:109F3000486210BD10000020EC0600202DE9F0471B
:109F4000F8F744FE104800F023F80F49497808114B
:109F5000F6F7E5FD04462046F6F726FE0746002202
:109F60000A4BF6F76DFD0546F6F74AFE044606492C
:109F70000878F6F7DDFD05462146F6F780FB8146B9
:109F80004846BDE8F0870000FD000020000030409A
:109F900070B504460225F8F713FF9020F8F7DCFEB1
:109FA000F8F764FF0020F8F7D7FEF8F75FFF04200A
:109FB00001F039FEF8F704FF9120F8F7CDFEF8F72D
:109FC00055FF06E00120F8F78FFE2070641C681E24
:109FD00085B2002DF6D1F8F719FF70BD10B503203A
:109FE00009F0D6F910BD10B5042009F0D1F910BD63
:109FF0000EB5002405E00021204609F03FFB601C5F
:10A00000C4B2052CF7DB16E0002404E0204609F07A
:10A010008FFA601CC4B2052CF8DB07480068401CAE
:10A020000549086002A8002114230A46CDE9001062
:10A030000846FAF767FCE7E7B406002010B50020F1
:10A0400009F0A6F910BD10B5012009F0A1F910BD65
:10A0500010B5022009F09CF910BD01F40072B2F5B0
:10A06000007F00D100BFCA430280704710B50022B4
:10A07000002340F66A14A14200D100BF0A12012455
:10A080009440A3B2DC43048010BD21B1828942F424
:10A090000052828104E082894DF6FF731A4082816A
:10A0A00070471AB1838A0B43838202E0838A8B4311
:10A0B0008382704702460020B1F5007F00D100BFC7
:10A0C00013880B400BB1012000E00020704770B5F1
:10A0D0000246002400230025002040F66A16B14203
:10A0E00000D100BFC1F3421501F01F03012606FA9B
:10A0F00003F3012D02D19689334006E0022D02D1EF
:10A10000168A334001E0968A33400C12012606FA83
:10A1100004F41688344013B10CB1012000E0002093
:10A1200070BDF0B50346002400260025002040F64F
:10A130006A17B94200D100BF1846C1F3421401F0BA
:10A140001F06012707FA06F5012C01D10C3004E0A7
:10A15000022C01D1103000E014301AB107682F43EF
:10A16000076002E00768AF430760F0BD2DE9F047E4
:10A1700086B005460E460024A24600BFA146002731
:10A18000B08900B100BF2F462C8A4CF6FF70044006
:10A19000F08804432C82AC894EF6F3100440B0885A
:10A1A00031890843718908430443AC81AC8A4FF676
:10A1B000FF400440B0890443AC8201A8FDF718F8C1
:10A1C0001F48874202D1DDF810A001E0DDF80CA0A5
:10A1D000A88900F4004040B10AEBCA0000EB0A1065
:10A1E00031684900B0FBF1F807E00AEBCA0000EB68
:10A1F0000A1031688900B0FBF1F86420B8FBF0F078
:10A2000004012009642101FB1089A88900F40040A1
:10A2100040B1322000EBC900B0FBF1F000F00700C4
:10A22000044308E0322000EB09106421B0FBF1F098
:10A2300000F00F0004432C8106B0BDE8F087000059
:10A240000038014001468888C0F30800704700BF0D
:10A25000FEE7000010B500F0C7FC0349086008469F
:10A2600000680249086210BD0C000020EC060020C6
:10A270000FB4054B10B503A9044A029800F020F969
:10A2800010BC5DF814FB0000A5C90208B40300204F
:10A290000FB47CB50C0009AD01D0611E00E00021B7
:10A2A000CDE90001064B6A462946089800F008F9F6
:10A2B000002C02D0009A002111707CBC5DF814FBC8
:10A2C000C7AB02080FB4084B10B504A902AA039843
:10A2D00000F0F6F8044602A9002000F07FFC2046BA
:10A2E00010BC5DF814FB0000DDAB0208014B024A14
:10A2F00000F0E6B8A5C90208B40300200048704782
:10A30000B803002002E008C8121F08C1002AFAD1D1
:10A3100070477047002001E001C1121F002AFBD1E5
:10A32000704710B502460B460020002103E0545C44
:10A3300060404C1CE1B29942F9DB10BD2DE9FF5F92
:10A3400082B00021DDE90430020DDDF840B00343A6
:10A3500018D044F61050A2F2FF324243151411985F
:10A3600001281FD0A5EB0B00401C5FEA000A4FF04C
:10A3700000064E4FDFF83891B046504615D5CAF169
:10A38000000413E0119801244AA3012801D16FEAC7
:10A390000B010298119AC0E90031C0E9024206B0EF
:10A3A000BDE8F09FCBF10000DFE704460021404A02
:10A3B000491842EB0450CDE9001012E0E00707D045
:10A3C00032463B4640464946F6F7C8FA804689463B
:10A3D00032463B4610461946F6F7C0FA06460F4687
:10A3E0006410002CEAD1DDE90401DDE90023BAF1B3
:10A3F000000F06DAF6F7B2FA42464B46F6F7AEFA27
:10A4000005E0F6F71DFB42464B46F6F719FB0446FE
:10A410000E460022284BF6F7DBFB03D84FF0FF3047
:10A42000014607E00022254B20463146F6F7EFF9BA
:10A43000F6F7ACFD102409E0002C0ADB0A22002309
:10A44000F5F7EDFE039B30321A55641E50EA010207
:10A45000F2D1641C039AC4F111031444119A012A25
:10A4600003D0012208430DD10AE0084304D00020A4
:10A470004FF0110B119072E7A3EB0B056D1E0DE071
:10A480005B4504DD4FF0000205F1010504E003DA4D
:10A490004FF00002A5F10105002AECD002981199B5
:10A4A000C0E90231C0E9004579E70000000014402E
:10A4B0000000F03F300000000000F0430000E03FEB
:10A4C0002DE9FF4F95B09A46884606460025EEE1F5
:10A4D000252877D100242746F94A0121039400E07A
:10A4E000044316F8013F203B01FA03F01042F7D174
:10A4F00030782A2811D06FF02F033078A0F1300285
:10A50000092A16D8039A44F0020402EB820203EBF4
:10A5100042021044761C0390EFE758F8042B039294
:10A52000002A03DA504244F40054039044F0020439
:10A53000761C30782E2816D116F8010F44F004044A
:10A540002A280DD06FF02F023078A0F13003092BAC
:10A5500009D807EB870302EB4303C718761CF3E720
:10A5600058F8047B761C30786C280FD006DC4C2819
:10A5700017D068280DD06A2814D104E0742810D0B0
:10A580007A280FD10DE044F400140AE044F480145A
:10A5900001E044F440147278824202D104F5801440
:10A5A000761C761C307866280BD013DC582877D0C0
:10A5B00009DC002875D04528F6D04628F4D0472875
:10A5C0001AD193E118E0632835D0642879D0652842
:10A5D00012D18BE1702873D008DC6728F1D069288C
:10A5E0006FD06E280DD06F2806D1ACE073282CD028
:10A5F000752874D0782853D05246179990476D1C0F
:10A6000054E1C4F30250022809D003280DD0D8F831
:10A61000001004280DD00D6008F1040846E1D8F8B8
:10A620000010EA17C1E90052F6E7D8F800100D80D3
:10A63000F2E70D70F0E718F8041B8DF80010002009
:10A640008DF80100EB46012003E058F804BB4FF001
:10A65000FF3061074FF0000102D40DE009F1010164
:10A660008946B9420FDA8145F8DB1BF80910002949
:10A67000F4D108E009F1010189468142FADB1BF8B7
:10A6800009100029F6D103985346A0EB090721468B
:10A690003846179A00F080FA284400EB090507E0D5
:10A6A00044E008E10DE01BF8010B52461799904772
:10A6B000B9F10109F7D2534621463846179AF2E01C
:10A6C00039E00A21C4F302524FF0000B0091022A34
:10A6D00006D058F8040BC117032A09D00AE023E07A
:10A6E00008F1070020F00702F2E80201904605E0B9
:10A6F00000B2C117042A01D140B2C117002906DAFD
:10A700000A460021404261EB02012D2202E02205AF
:10A7100004D52B228DF80420012203E0E20701D0AA
:10A720002022F7E7914657E00A2100E010214FF080
:10A73000000B00910BE010214FF0000B44F00404DB
:10A740000827009103E008204FF0000B0090C4F3AD
:10A750000252022A05D058F8040B0021032A08D01F
:10A7600008E008F1070020F00702F2E80201904635
:10A7700003E080B2042A00D1C0B24FF000092207E2
:10A780002AD53278702A07D0DDF800C08CF0100C82
:10A790005CEA0B0C05D00EE040228DF8042001226B
:10A7A00008E050EA010306D030238DF804308DF81C
:10A7B000052002229146009B83F0080353EA0B0315
:10A7C0000AD150EA010201D1620705D530228DF885
:10A7D00004204FF001097F1E3278582A04D039A294
:10A7E0000C920CAA02920BE03BA2F9E75B46009A9E
:10A7F000F5F715FD0C9B9B5C029A521E029213709A
:10A8000050EA0102F2D1029804A9081A00F1200BC3
:10A81000600702D524F4803400E001275F4502DDA3
:10A82000A7EB0B0000E0002000EB0B010090039869
:10A830004944401A0390E00306D453462146179A30
:10A84000039800F0A9F90544002706E001A8524644
:10A85000C05D179990476D1C7F1C4F45F6DBE003E8
:10A860000CD553462146179A039800F095F90544F4
:10A8700004E030205246179990476D1C0099481EFD
:10A8800000900029F5DC08E0029802995246007811
:10A89000491C0291179990476D1CBBF10001ABF167
:10A8A000010BF1DC5BE100F065F90544761C3078C2
:10A8B00000287FF40DAE19B02846BDE8F08F0000E7
:10A8C0000928010030313233343536373839616286
:10A8D000636465660000000030313233343536374A
:10A8E000383941424344454600000000600700D427
:10A8F000062708F1070020F00700F0E80223804651
:10A9000003F0004C5FEA0C0001D097A009E020059D
:10A9100001D596A005E0E00701D095A001E0AFF2D7
:10A920004C001390307823F0004365280CD006DCEF
:10A93000452809D046281DD047287FD13BE066280E
:10A9400018D067287AD136E00021112F01DB1120C1
:10A9500000E0781CCDE9000104A90CA8FFF7EEFC8B
:10A96000DDE90D010C9A4FF0000B07F1010910927F
:10A9700000914EE04FF000400097CDE9011004A98E
:10A980000CA8FFF7DBFCDDE90D020C9B0F994FF0E3
:10A99000000B91461093009211B9791C00EB01094C
:10A9A000B7EB090003D4C0F1FF3B07F10109A9EBA4
:10A9B0000700019042E0012F00DA01270021112F4A
:10A9C00001DD112000E03846CDE9000104A90CA802
:10A9D000FFF7B4FCDDE90D010C9A00914FF0000B7C
:10A9E000B946109221070FD4009A4A4503DA9146DE
:10A9F00001E0A9F10109B9F1010F05DD109AA9F1F2
:10AA00000101515C3029F4D0B84202DA10F1040F90
:10AA100003DA0121CDE9011010E0002803DC8344B2
:10AA2000A9EB000102E0411C494500DD8946A0EB8D
:10AA30000B00401C01904FF000400290200705D40D
:10AA40000198484502DB4FF0FF30019000208DF85F
:10AA50004B0002980DF14B07B0F1004F25D00220BA
:10AA60000C902B200D90029800280CDA40420290A6
:10AA70002D200D9007E00A210298F6F7DDF830311D
:10AA8000029007F8011D0C99481E0C900029F2DC79
:10AA900002980028EFD1791E0D980870307800F0E8
:10AAA000200040F0450007F8020D11A8C01BC01D92
:10AAB00002901398007800B1012000EB0901019881
:10AAC00001EBE071029801440398401A401E039084
:10AAD000E00306D453462146179A039800F05CF829
:10AAE00005441398007818B15246179990476D1C89
:10AAF000E00323D553462146179A039800F04CF8FB
:10AB000005441BE0BBF1000F07DB0098584504DD4E
:10AB10001098179910F80B0001E017993020524651
:10AB2000904701980BF1010B401E05F101050190C2
:10AB300004D12E205246179990476D1CB9F100019F
:10AB4000A9F10109DEDC05E017F8010B524617995F
:10AB500090476D1C0299481E02900029F4DC534670
:10AB60002146179A03989EE62D0000002B00000056
:10AB7000200000002DE9F041044600251E4617463E
:10AB8000880404D405E039462020B0476D1C641EBB
:10AB9000F9D52846BDE8F0812DE9F04104460025AD
:10ABA0001E469046C80301D5302700E020278804C0
:10ABB00004D505E041463846B0476D1C641EF9D502
:10ABC0002846BDE8F0814A68002A06D00A68531C6E
:10ABD0000B6010704868401E486070470A68531C3C
:10ABE0000B601070704700002DE9FE430025002621
:10ABF0000027032720E007220121002003F0DEF8D0
:10AC000006463046F5F794FF81461649F5F78FFD65
:10AC100080464FF08B41F5F7BCFD0446214628469F
:10AC2000F5F72DFD054602A800210A230A46CDE9C5
:10AC300000100846F9F766FE381EA7F101018FB231
:10AC4000D9D109492846F5F7A4FD0446074920460D
:10AC5000F5F79FFD04464FF080412046F5F767FD6C
:10AC6000BDE8FE8300404E450000404000007A44AD
:10AC700000B587B001210420FCF790FA01214802B9
:10AC8000FCF78CFA4FF40040FCF75CFA0120ADF8B9
:10AC9000180000208DF81B0006A91A48F7F712FDCE
:10ACA0001948F6F7CDFB002001908DF808008DF8CB
:10ACB00009004FF4602003900020049001208DF8DB
:10ACC000140001A91048F6F70BFC01210E48F6F715
:10ACD000ABFB0D48F6F788FC00BF0B48F6F7F5FB19
:10ACE0000028FAD10848F6F78FFC00BF0648F6F7AF
:10ACF000D5FB0028FAD101210348F6F77AFC07B00A
:10AD000000BD000000080140002401402DE9F04191
:10AD100003460E461746002400220DE0985CF7F724
:10AD20003BFF8046511C585CF7F736FF054645EA65
:10AD300008103055641C921CBA42EFDB2046BDE877
:10AD4000F08170B503460C460020002107E05D5CF1
:10AD5000665CB54201D0012003E04D1CA9B29142CE
:10AD6000F5DB00BF70BD000030B5A1B0802101A8A7
:10AD7000F5F70DFB002494E1E01CC1B20122FB4871
:10AD800007F0DCFBFA4908800846008800287CD0E0
:10AD900008460088F7490880E21CD1B2F34AF54B17
:10ADA0001B88D018322207F0C9FBF14908800846F9
:10ADB0000088F04909880844ED490880211DEEA06B
:10ADC000FFF756FAEA480288E849EEA000F0CCFE08
:10ADD000E7480088802804DDEDA0FFF749FA21B09C
:10ADE00030BDE2488078FF285BD0E01C00EB80108B
:10ADF000EC4911F8200068B90021E01C00EB80103C
:10AE0000E84A02EB800041800121E01C00EB801049
:10AE100002F82010E01C00EB8010E24901EB8000FA
:10AE20004088D3490988084480280DDD0021E01CB2
:10AE300000EB8010DB4A02F82010E01C00EB8010D1
:10AE400002EB80004180CAE7E11C01EB8111D54A89
:10AE500002EB8101091DE21C02EB8212D14B03EBD4
:10AE6000820252888818C2490A88C049F5F776FAE2
:10AE7000E01C00EB8010CB4901EB80004088BC490E
:10AE80000988084481B2E01C00E05CE000EB80101F
:10AE9000C44A02EB80004180B4488078012800D089
:10AEA0009DE7E01C00EB8010BE4911F8200018B3AC
:10AEB0000021E01C00EB8010BA4A02F82010E01CD0
:10AEC00000EB8010134603EB80004288E01C00EB8F
:10AED000801003EB8000011DA448F5F73FFAE01C49
:10AEE00000EB8010AF4901EB80004088A04908804A
:10AEF000E11CC8B208F0BEF9ABA0FFF7B9F9AD4844
:10AF00008078032820D1AB4890F82010E01C8142C3
:10AF100019D1A848C0790128FAD1A648008941F280
:10AF200052018842F4D1A44807F006FAE11CC8B2E5
:10AF3000002106F0D0FE8E4802888C49012007F0DF
:10AF4000C1FA04F095FEAAE09C4803789C48027B75
:10AF5000017A9CA0FFF78CF99948017AE01C8142A4
:10AF6000F1D1954807F0E8F9E11CC8B2002106F0DC
:10AF7000B2FE67259148007801287AD18F48807900
:10AF8000572820D18D48407803281CD19D4801685E
:10AF90000191416802910089ADF80C007448028863
:10AFA00072490DF10E00F5F7D9F9714800780A30B1
:10AFB000C3B201AA0121284602F090FA07F0C4F8B2
:10AFC00004F04EFE54E07D488079572822D17B481A
:10AFD000407802281ED17948C078702814D164487E
:10AFE000028862490DF10E00F5F7B8F96048007863
:10AFF0000A30C3B201AA0121284602F06FFA07F015
:10B00000A3F804F02DFE33E059480188574807F0B3
:10B0100007F82DE069488079562824D167484078A0
:10B02000012803D06548407804281CD15048018885
:10B030004E4806F0F5FF74480078022809D1002038
:10B040007149087007F080F800F0A6FC04F008FED3
:10B05000C5E602206C49087007F076F8042006F077
:10B0600011F9BCE605E042480188404806F0D8FFE7
:10B07000B5E65348007B012808D13D490B7850497B
:10B08000087B3A4A012100F041FD06E03848037888
:10B09000364A0121284602F021FA04F0E1FD601C45
:10B0A000C4B2022CFFF668AE01220221574807F015
:10B0B00045FA5749088008460088002855D00846B8
:10B0C00000882C4908805149514A12888818322238
:10B0D000022107F033FA4E490880084600882549C6
:10B0E000098808444A49088008460288474949A017
:10B0F00000F03AFD46480088E52803DD24A0FFF76C
:10B10000B7F86CE64748807F01280DD146480078A3
:10B11000052809D145484078022805D13C480188D6
:10B120003A4808F0F5FB5AE62248807803287FD198
:10B13000204890F82000022817D11F4807F0FCF89B
:10B14000052003F033FD1B48C07901280DD11948B3
:10B15000008941F25201884207D12D4802882B49CB
:10B16000012007F0AFF904F083FD89E0F8870020A3
:10B170004C0200204E020020554152543A25640AE8
:10B180000000000075617274207263760000000098
:10B19000756172742072637620746F6F206C6F6EAD
:10B1A000670A0000848C0020626567696E207072F7
:10B1B0006F630A0028A400200C8C0020E0A6002069
:10B1C000F88B00206D73675F706172612E7561721C
:10B1D00074203D2025642C6D73675F706172612E51
:10B1E00066697273745F747970653A25642C746152
:10B1F000785F73656E645F73746172743A25640A74
:10B200000000000099A80020500200209891002022
:10B21000560200207561727433207263762070725A
:10B220006F740000EC060020D10200204AA4002028
:10B23000FFE714488078FF280ED1134807F07CF808
:10B24000052003F0B3FC114802881149022004F0E4
:10B2500073F804F00DFD13E00E48007A02280FD1B8
:10B26000094807F069F8052003F0A0FC64250748A9
:10B270000378074A0121284602F030F904F0F0FC77
:10B2800000BFACE528A400200C8C00205602002052
:10B2900098910020F88B00202DE9F041C1F30A526B
:10B2A000A2F2FF362F4A304B0D460446142E2FDAF9
:10B2B000002E12DAF5F7ABFA00221346F5F788FCF8
:10B2C0004CD2002DBCBF4FF00045002446DB55EAB0
:10B2D000040018BF254D19D140E0DFF894C02CFAC6
:10B2E00006F705EA070C5CEA040C08BFBDE8F0812C
:10B2F000F5F78DFA00221346F5F76AFC2ED2002DE1
:10B3000003DD4FF48010F0400544BD43002425E0E8
:10B31000332EC8BFBDE8F081A6F1140C4FF0FF3703
:10B3200027FA0CF73C4208BFBDE8F081F5F713FBA4
:10B3300000221346F5F74CFC10D2002D0DDD142E23
:10B3400008BF6D1C09D0C6F13400012101FA00F0DC
:10B350002044A04238BF6D1C0446BC432946204609
:10B36000BDE8F0819C7500883CE4377E0000F03F2A
:10B37000FFFF0F000248002101604160018170471A
:10B38000158C002010B5064806F07CFF38B105A0EA
:10B39000FEF76EFF002005F0A1FAFFF7EBFF10BDEE
:10B3A000168C0020BCD3C3DCC4A3BFE9CBC0C1CB87
:10B3B0000000000010B50748407F022808D1064869
:10B3C000407828B9012205490348401C06F094FF43
:10B3D00010BD0000EC060020158C002080EE360029
:10B3E00010B5002009498874487281F82400C87695
:10B3F00081F82D0081F8360081F83F0081F848007F
:10B400000021FF2003F006FA10BD00006734002081
:10B410002DE9F04185B00646B4463A4801903A48D5
:10B4200002903A4803903A48049031200870322044
:10B430004870332088703420C87000235CE00024FA
:10B4400003E000200DF80400641C042CF9D31CF860
:10B45000030091F8008080EA080505F08000A8B19B
:10B460009DF8000080F0A0008DF800009DF801001C
:10B470008DF801009DF8020080F001008DF80200B7
:10B480009DF8030080F094008DF803006806070E15
:10B49000012219E007F0800098B19DF800000DF13D
:10B4A000040818F8028080EA08008DF800009DF872
:10B4B00003000DF10C0818F8028080EA08008DF8EE
:10B4C00003007806070E521C082AE3D348789DF83B
:10B4D000008080EA0800087088789DF8018080EA82
:10B4E00008004870C8789DF8028080EA08008870DB
:10B4F0009DF80300C8705B1C042BA0D3002005B08E
:10B50000BDE8F081A0502898C060301894CA653317
:10B51000180C0603024610680B68984201D90120F6
:10B5200070474FF0FF30FBE730B5C1B0054604ACC3
:10B530002848D0F80100206027480079207140F2A7
:10B540000170A4F805002448407AE0712572012DAD
:10B5500003D00020A4F809002AE0E079401EC0EBE7
:10B56000C00000EB80001D490844B0F80100A4F8B9
:10B570000900E079401EC0EBC00000EB80000B46E4
:10B580001844B0F80120E079401EC0EBC00000EB89
:10B5900080001844C11C04F10B00F4F7DFFE002109
:10B5A000E079401EC0EBC00000EB80000B4A115454
:10B5B000B4F809000B3082B2622101A802F064FBEA
:10B5C000BDF80E000C3082B201A905A000F0CCFA43
:10B5D00041B030BDDC060020F88B00202B8C002011
:10B5E000636D643733000000F0B5A1B005460E4628
:10B5F0001446802101A8F4F7CAFE0027124806F07D
:10B600009BFE00201049C91E08700CB1012C07D107
:10B6100001AB22463146284600F018F807460AE0FA
:10B62000022C01D0032C06D101AB2246314628461C
:10B6300000F0B4F807463B4601AA01216C2001F056
:10B640004DFF21B0F0BD0000228C00202DE9F84F05
:10B6500006460F4690461C464FF0000A0020009018
:10B660008146254685F80080F7F71AF968700120B1
:10B67000F7F716F9A8703E484670F7F765F93C49A8
:10B6800088700120087001224FF4FA613848C01C0C
:10B6900006F032FE7A1ED1B2721ED0B243466A461E
:10B6A00005F022FE81464B469DF8002031A1012085
:10B6B00005F07CFA85F80390701E00EB0010354908
:10B6C00001EB4011781E00EB001001EB00109DF81B
:10B6D000001001EB0111084400686860701E00EB67
:10B6E00000102C4901EB4011781E00EB001001EB1B
:10B6F00000109DF8001001EB01110844007940F0A2
:10B7000080002872701E00EB0010224901EB4011EE
:10B71000781E00EB001001EB00109DF8001001EB0B
:10B7200001110844D0F80500C5F80900701E00EBAF
:10B730000010184901EB4011781E00EB001001EBDE
:10B7400000109DF8001001EB01110844D0F8090029
:10B75000C5F80D00701E104901EBC001781E51F8AC
:10B760002000C5F811004FF0150A5046BDE8F88FCB
:10B770001F8C0020726561642067726F75703A25B6
:10B78000642C206E65772070756C73653A25640AA9
:10B790000000000098940020D89800202DE9F04F78
:10B7A00089B0054691461F460020089007900690F4
:10B7B00082468346142101A8F4F7E9FD3E460DF1C7
:10B7C000040886F800900020F7F76AF870700120EE
:10B7D000F7F766F8B07048484570F7F7B5F846498E
:10B7E00088700120087001224FF4FA614248C01CA1
:10B7F00006F082FD00246FE0691EC8B24B4607AA1E
:10B80000214605F071FD0690069828B10120A04060
:10B8100040EA0A0000F0FF0A681E00EB00103749FA
:10B8200001EB401004EB041100EB01109DF81C101B
:10B8300001EB011108440068C8F80000681E00EB25
:10B8400000102E4901EB401004EB041100EB011035
:10B850009DF81C1001EB01110844D0F80500C8F850
:10B860000400681E00EB0010244901EB401004EBBB
:10B87000041100EB01109DF81C1001EB01110844AC
:10B88000D0F80900C8F80800681E1D4901EBC00087
:10B8900050F82400C8F80C00681E00EB001017498F
:10B8A00001EB401004EB041100EB01109DF81C109B
:10B8B00001EB01110844007928B10120A04040EAC1
:10B8C0000B0000F0FF0BB11D01EB0410102201A9C9
:10B8D000F4F744FD601CC4B2022C8DDB86F803A093
:10B8E0004BF080003071022070712620089008987B
:10B8F00009B0BDE8F08F00001F8C00209894002054
:10B90000D898002010B5C0B003AC1E48D0F8010094
:10B9100020601D48007920711C484068C4F805006B
:10B920001A480068C4F8090018488069C4F80D0076
:10B930001648007F60744FF47A7200231449086837
:10B940004968F4F76CFCC4F812001048006AC4F8A7
:10B9500016000E48406AC4F81A000E480078A07716
:10B960000A488168C4F81F10C168C4F82310006930
:10B97000C4F827002B226821684602F085F940B000
:10B9800010BD0000DC060020F88B0020EC06002033
:10B9900028000020D002002010B5C0B003AC0C4835
:10B9A000D0F8010020600B48007920710A48407FE0
:10B9B000607106226621684602F066F9BDF80A0049
:10B9C0000C3082B2694605A000F0CEF840B010BD40
:10B9D000DC060020F88B0020EC0600206865617210
:10B9E00074626561740000002DE9F04104460F4661
:10B9F000154600264FF6FE6020800120A0701948F1
:10BA00000068C4F8030017480068401C1549086026
:10BA1000E77100202081A81C608104F10C0000EB7C
:10BA20000508608900F10A012046F6F757FAA8F8E0
:10BA30000000022003F0BEFC064666B105F10E02CE
:10BA400021463046F4F78AFC05F10E023146022009
:10BA500003F072FC03E03146022003F0DFFCBDE896
:10BA6000F0810000DC0200202DE9F04104460E4682
:10BA700015464FF6FE6020800220A0701148006835
:10BA8000C4F803000F480068401C0E4908600420F9
:10BA9000E0712681A81C6081608900F10A012046BE
:10BAA000F6F71CFA074604F10C0047553A0A691CE0
:10BAB000425405F10E022146022007F0FFFCBDE8CA
:10BAC000F0810000E002002070B504460D462646D5
:10BAD000F079012804D12946204603F0A3FE00E0B6
:10BAE00000BF00BF70BD70B504460E462546E8791C
:10BAF000012809D1288941F20701884203D1314642
:10BB0000204605F063F800BF00BF70BD2DE9F0418D
:10BB1000C0B007460D4690461E4603AC104800696B
:10BB200020601048D0F8010060600D48407A207213
:10BB30006572012D07D166813246414604F10C0041
:10BB4000F4F70CFC01E00020608160890C3082B2C7
:10BB50003946684602F098F840B0BDE8F081000030
:10BB6000F88B0020DC0600202DE9F04105460E464A
:10BB700017460024294614A0FEF77AFB00BF1BE0FD
:10BB8000E11704EB91718910A4EB810179B974B1CB
:10BB9000E11704EB11710911A4EB011121B91CB1DA
:10BBA0000FA0FEF765FB02E00FA0FEF761FB315D21
:10BBB0000EA0FEF75DFB641CBC42E1DB0DA0FEF7AE
:10BBC00057FBBDE8F08100002573204461746120BB
:10BBD000496E666F3A200D0A2020202000000000E8
:10BBE0000D0A20202020000020000000253032789F
:10BBF000200000000D0A00002DE9F04107460C4628
:10BC000015461E4627B1324629462046FFF7ACFFAF
:10BC1000BDE8F08110B504464FF47A7104FB01F0E1
:10BC200000F001F810BD0021002200BF05E0002255
:10BC300000E0521C092AFCD3491C8142F7D370470B
:10BC40000A480B4908600B48006848600A480088A9
:10BC500088820A48D0F8030088610948007808778C
:10BC60000846084B0ECB08300EC070473031010239
:10BC7000EC0600200C740020CA0100200074002093
:10BC8000D4010020F473002010B510210448F4F70B
:10BC90007EFB102202490D20F5F7EAFC10BD0000E2
:10BCA000DC06002010B511480078012803D10020DF
:10BCB0000F4988770AE003200D498877001F0B4958
:10BCC000C1F8010040F20120A1F805000948806890
:10BCD0000949884207D0084606498860042208318D
:10BCE0002920F5F713FDFFF7ABFF10BDDC060020A0
:10BCF000EC0600200C7400203031010210B5102237
:10BD000002490D20F5F702FD10BD0000DC06002001
:10BD10001CB504460320009000208DF804000C2080
:10BD20008DF805008DF806406846F6F7D5FA0F48FD
:10BD3000007801280DD14FF2C060009000208DF8EE
:10BD4000040010208DF805008DF806406846F6F7CF
:10BD5000C3FA074804700078012803D105A0FEF754
:10BD600087FA02E006A0FEF783FA1CBDF800002067
:10BD70001400002069727120656E61626C650A00B2
:10BD80006972712064697361626C650A0000000069
:10BD900010B5FFF7F7FA1B4806F074FA40B101211D
:10BDA000194806F0BFFA19A0FEF762FA02F0A6FFE2
:10BDB000154806F067FA60B11AA0FEF759FAFCF7C9
:10BDC000D3FD20B101201F4981F82B0001E0F7F7D6
:10BDD00075F91C4890F82B0058B1FCF7C5FD40B927
:10BDE00019A0FEF745FA0020164981F82B00F7F755
:10BDF00065F9184806F046FA18B100201549C91E21
:10BE0000087010BD260200202F0200206C6F7261A6
:10BE1000D2BBD0A1CAB1CEB4CAD5B5BDCAFDBEDDB4
:10BE20000A0000006C6F7261B8B4CEBB35B7D6D6CD
:10BE3000D3BAF3BBB9CEB4CAD5B5BDCAFDBEDD0A0F
:10BE400000000000EC060020B2C9BCAFC6F7B8B4D1
:10BE5000CEBB0A00228C002010B5044806F012FA6E
:10BE600018B1FEF75DF8FEF7F5F910BD15000020DA
:10BE70000246002040F201239A4208D1084BD3F831
:10BE800001308B4201D04B1C43B9012006E04FF634
:10BE9000FF739A4202D14B1C03B901207047000086
:10BEA000DC06002002460020054BB3F80530934223
:10BEB00005D1034BD3F801308B4200D101207047EC
:10BEC000DC06002010B50246002000234FF6FF7468
:10BED00004EA12438B4200D1012010BD00B58FB09F
:10BEE000382101A8F4F753FA352201A90020F5F70B
:10BEF000BFFB0B2201A92148F4F730FA10220DF103
:10BF000011011F48F4F72AFA14220DF125011D48EA
:10BF1000F4F724FA022201A94020F5F7A9FB9DF8C5
:10BF200004009DF80510C943C9B288420ED0002014
:10BF30008DF804009DF80400C043C0B28DF80500E0
:10BF4000022201A94020F5F7E1FB11E09DF8040071
:10BF500003280DDD00208DF804009DF80400C04387
:10BF6000C0B28DF80500022201A94020F5F7CEFBF2
:10BF70009DF80400044908700FB000BD0074002053
:10BF8000DC0600200C740020E801002070B5044697
:10BF90000D461646324629462046F5F7B7FB70BDDA
:10BFA00010B550210548F4F7F2F918210448F4F7C8
:10BFB000EEF9044800210160416010BD3893002073
:10BFC000D8920020789400202DE9F047A6B04FF0D9
:10BFD000000A20211EA8F4F7DAF9202116A8F4F7A8
:10BFE000D6F9002012901390149015900E900F9097
:10BFF000109011900A900B900C900D900690079065
:10C0000008900990049005900290039000BF2022B0
:10C010001EA98020F5F72CFB202216A9D000F5F7E9
:10C0200027FB20231EAA7EA10020FFF7E5FD202389
:10C0300016AA80A10020FFF7DFFD10220AA95001F7
:10C04000F5F716FB102206A94FF41070F5F710FB58
:10C05000202212A91EA8F6F72AFD804620220EA94A
:10C0600016A8F6F724FD8146102204A90AA8F6F7BF
:10C070001EFD0746102202A906A8F6F718FD06467F
:10C08000B8F1000F05D1B9F1000F02D10FB9002EA0
:10C0900047D00AF1010000F0FF0A6BA0FEF7E8F8B4
:10C0A000BAF1030F00DAB2E7B8F1000F0DD020218A
:10C0B0001EA8F4F76CF900201290139014901590BC
:10C0C00020221EA98020F5F721FBB9F1000F0DD029
:10C0D000202116A8F4F75BF900200E900F90109025
:10C0E0001190202216A9D000F5F710FB5FB10020B7
:10C0F0000A900B900C900D900490059010220AA9C4
:10C100005001F5F703FB66B10020069007900890F8
:10C11000099002900390102206A94FF41070F5F7D1
:10C12000F5FA102312AA4DA10020FFF765FD102398
:10C130000EAA4DA10020FFF75FFD00256AE0002454
:10C1400065E00DBB4B4800EB051000EBC40012A9E5
:10C1500001EBC40206CA06C0474800EBC50004A9AB
:10C1600051F8241040F82410434800EBC50050F863
:10C17000240005EB8501414A02EB411104EB8402E6
:10C1800001EB0211486222E0012D20D1394800EB79
:10C19000051000EBC4000EA901EBC40206CA06C0DC
:10C1A000354800EBC50002A951F8241040F82410CE
:10C1B000314800EBC50050F8240005EB85012F4AFB
:10C1C00002EB411104EB840201EB021148622948A1
:10C1D00000EB051000EBC4004068264901EB051197
:10C1E00051F83410631C6A1CCDE9001024A1012011
:10C1F00004F0DCFC204800EBC50050F82400631C70
:10C200006A1C28A10090012004F0D0FC641C022CC0
:10C2100097DB6D1C022D92DB26B0BDE8F087000095
:10C2200074617831207265616420656570726F6D2C
:10C2300000000000746178322072656164206565D9
:10C2400070726F6D00000000656E636F6465722030
:10C2500064617461206572720A0000007461783153
:10C26000206465636F64650074617832206465637F
:10C270006F64650078940020D898002038930020DF
:10C280007461783A25642C67756E3A25642C69646C
:10C290003D25752C746F74616C2070756C73653DF1
:10C2A00025750A007461783A25642C67756E3A2505
:10C2B000642C67756E206E756D3D25750A00000053
:10C2C00030B589B000200790089003900490059045
:10C2D0000690002400258E4805F0D4FF002873D076
:10C2E0008C48007800EB80008B4901EB40108B49B3
:10C2F000097801EB810100EB01100078002877D06C
:10C3000087488449097800EB01108449097850F87E
:10C31000315083487F49097800EB01107F49097843
:10C3200000EBC10103C9CDE90701082203A907A851
:10C33000F6F702FC7748007828B978480078802121
:10C3400001EB001409E073480078012805D1734817
:10C3500000784FF4807101EB0014102203A92046ED
:10C36000F5F7D4F96B48007800EB80006A4901EBDF
:10C3700040106A49097801EB810100EB0110C560AA
:10C38000102303AA67A10020FFF736FC6448614927
:10C39000097800EB01106149097800EBC1004068A1
:10C3A0005F495C4A127801EB02115C4A127851F83D
:10C3B00032105A4A1278521CCDE900210290554899
:10C3C00003785B1C224600E09FE05AA1002004F0A5
:10C3D000EDFB00204F49097801EB81014E4A02EB49
:10C3E00041114E4A127802EB820201EB02110870F1
:10C3F0004848007800EB8000474901EB401047496E
:10C40000097801EB810100EB011090F82800002869
:10C4100064D04048007800EB80003F4901EB4010B9
:10C420003E49097801EB810100EB0110406A504957
:10C43000384A127801EBC201384A127841F82200DA
:10C440004B483449097800EBC1003449097850F869
:10C4500021000790042203A907A8F6F76DFB2D48D9
:10C46000007830B92D4800784FF4007101EBC0041A
:10C4700009E028480078012805D1284800784FF4C1
:10C48000107101EBC004082203A92046F5F73EF91C
:10C4900037482049097800EBC1002049097850F855
:10C4A00021001E490978491CCDE90010194803787C
:10C4B0005B1C22462FA1012004F078FB00211548C7
:10C4C000007800EB8000144A02EB4010134A127807
:10C4D00002EB820200EB021080F828100F49097865
:10C4E000481C00EBD0714910A0EB41010B4A1170C0
:10C4F0001046007848B907490978481C00EBD0710C
:10C500004910A0EB4101034A117009B030BD000091
:10C51000C0020020C902002038930020CA02002077
:10C5200078940020777269746520656570726F6D0C
:10C5300000000000D0B4656570726F6DA3BA6164CD
:10C5400064723D307825782C207461783D25642C08
:10C550002067756E3D25642C2069643D25752C206F
:10C56000746F74616C2070756C73653D25750A007D
:10C57000D8980020D0B467756E206E756DA3BA612F
:10C580006464723D307825782C207461783D256490
:10C590002C2067756E3D25642C2067756E206E75A6
:10C5A0006D3D25750A0000001FB501213820FAF7FE
:10C5B000F5FD01213B48F6F711F903208DF80E0037
:10C5C00048208DF80F004FF48060ADF80C0003A9EF
:10C5D0003548F6F777F803208DF80E0048208DF8DF
:10C5E0000F004FF43070ADF80C0003A92F48F6F798
:10C5F00069F803208DF80E0048208DF80F004FF4E5
:10C600007040ADF80C0003A92948F6F75BF801214A
:10C610000846FAF7C3FD0A210120F6F733F8062190
:10C620000220F6F72FF807210220F6F72BF8092150
:10C630000220F6F727F80C210320F6F723F80D2146
:10C640000320F6F71FF80E210320F6F71BF80F2141
:10C650000320F6F717F84FF2C060019000208DF824
:10C66000080010208DF8090001208DF80A0001A8AB
:10C67000F5F732FE28208DF8000000208DF801002B
:10C680008DF8020001208DF803006846F6F7CAFC19
:10C690004FF47440F5F706FE4FF43070F5F702FEE4
:10C6A0001FBD000000023000000C014000100140DE
:10C6B0000014014010B5FFF773FCFFF775FF01F0A0
:10C6C0009FFC00F09FF801F051FDFFF77DFC10BDCD
:10C6D00070B50446184810F8345000EBC400467892
:10C6E000154800EBC400807878B905EB8501134A42
:10C6F00002EB411106EB860201EB021101F1300061
:10C700000122642105F0F8FD15E00B4800EBC400A0
:10C71000807801280FD105EB8501084A02EB411111
:10C7200006EB860201EB021101F13D0001224FF4FC
:10C730007A7105F0EBFD70BD9892002038930020CF
:10C7400070B5002448E0002542E004EB8401244A4F
:10C7500002EB411105EB850201EB021101F14600EC
:10C7600005F090FDA8B100222946204604F07CFB8C
:10C77000012104EB84001A4A02EB401005EB85020C
:10C7800000EB021080F82E106A1C611C15A0FDF74A
:10C790006FFD04EB8400124901EB401005EB8501AD
:10C7A00000EB011090F82F0080B1002104EB840011
:10C7B0000B4A02EB401005EB850200EB021080F8FB
:10C7C0002F1001222946204604F04EFB681CC5B2FA
:10C7D000022DBADB601CC4B2022CB4DB70BD0000B9
:10C7E000389300207461783A25642C67756E3A2579
:10C7F000642C70756C73652074696D656F75740A4F
:10C800000000000030B5002055E000214FE000227C
:10C8100048E001EB4103294C04EB031302EB420413
:10C8200003EBC4035B6900EB4004254D05EB840476
:10C83000A468A34210D1234B03F8301003EBC003CC
:10C840005A7000231F4C04EBC004A37064231D4CDA
:10C8500004EBC004636027E001EB4103174C04EBD9
:10C86000031302EB420403EBC4039B6800EB400498
:10C87000134D05EB8404A468A34211D1114B03F8B6
:10C88000301003EBC0035A7001230E4C04EBC004BC
:10C89000A3704FF47A730B4C04EBC004636003E0A5
:10C8A000531CDAB2022AB4DB00BF4B1CD9B20229F6
:10C8B000ADDB431CD8B20828A7DB30BDD8920020DE
:10C8C00058020020989200202DE9F041C1F30A524D
:10C8D000A2F2FF362F4A304B0D460446142E2FDAB3
:10C8E000002E12DAF3F793FF00221346F4F770F9E3
:10C8F0004CD2002DA4BF0024254647DA25F0004085
:10C90000204318BF254D41D018E0DFF894C02CFA21
:10C9100006F705EA070C5CEA040C08BFBDE8F081E5
:10C92000F3F775FF00221346F4F752F92ED2002DCB
:10C9300003DA4FF48010F0400544BD43002425E0A5
:10C94000332EC8BFBDE8F081A6F1140C4FF0FF37BD
:10C9500027FA0CF73C4208BFBDE8F081F3F7FBFF74
:10C9600000221346F4F734F910D2002D0DDA142EFC
:10C9700008BF6D1C09D0C6F13400012101FA00F096
:10C980002044A04238BF6D1C0446BC4329462046C3
:10C99000BDE8F0819C7500883CE4377E0000F0BF64
:10C9A000FFFF0F002DE9F04105460F464FF47A7660
:10C9B0000E4884690E480078A8B901E0701E86B25E
:10C9C000002E01DD012000E00020218820EA9110E6
:10C9D0000028F3D1E8B2A08000BF80212046FDF7F7
:10C9E00069FB0128F9D12846BDE8F0813C00002010
:10C9F000289900202DE9FE4305460027B846002669
:10CA000005F10C04E87952380C287DD2DFE800F0FB
:10CA1000067C1F3A55F6EEEDECEBEAE92068E649B4
:10CA2000D1F80110884211D12079E44908712268B7
:10CA30001146E3A0FDF71CFCE979E8A0FDF718FC1E
:10CA4000072002F0B3F8284600F0D0FDB1E12068DD
:10CA5000D949D1F80110884213D12079D7490871FA
:10CA600023681A46D6A1012004F0A0F8EA79DBA1D8
:10CA7000012004F09BF8072002F098F8284600F007
:10CA800013FB96E12068CC49D1F80110884213D1FC
:10CA90002079CA49087123681A46C9A1012004F007
:10CAA00085F8EA79CDA1012004F080F8072002F092
:10CAB0007DF8284600F0F8FA7BE12068BE49D1F8FD
:10CAC000011088423CD12079BC490871D5F8030097
:10CAD000086022681146BAA0FDF7CAFBE979BFA039
:10CAE000FDF7C6FB072002F061F8688907286CDDB6
:10CAF000697CBDA0FDF7BCFB687C012812D1BE4853
:10CB0000407F00F0030000E052E130B90220BB4951
:10CB10000870032004F0B6FB04E01420FFF77AF855
:10CB2000FEF73AFF687C022811D1B348407F00F03D
:10CB30000C0030B90220B1490870042004F0A2FBB7
:10CB40005BE01420FFF766F8FEF726FF55E0687CEF
:10CB5000032852D1A848407F00F0030050B1A648F6
:10CB6000407F00F00C0028B11420FFF753F8FEF7C7
:10CB700013FF42E0A048407F00F0030010B90127F6
:10CB8000701CC6B29C48407F00F00C0018B94FF0F2
:10CB90000108701CC6B2012E0ED11FB1032004F093
:10CBA00071FB05E0B8F1000F02D0042004F06AFB2D
:10CBB00002209249087020E0022E1ED1032004F0CA
:10CBC00061FB01208D49087017E08B48407F00F021
:10CBD000030068B9022089490870032004F052FB61
:10CBE0000BE0C7E0A7E06AE087E048E021E005E06D
:10CBF0001420FFF70FF8FEF7CFFEDAE020686E4949
:10CC0000D1F80110884213D120796C49087123684A
:10CC10001A466BA1012003F0C9FFEA796FA1012038
:10CC200003F0C4FF072001F0C1FF284600F03CFAE2
:10CC3000BFE020686049D1F8011088421ED12079F8
:10CC40005E490871D5F80300086023681A465CA1A4
:10CC5000012003F0ABFFEA7960A1012003F0A6FFF9
:10CC6000072001F0A3FF02A8002114230A46CDE902
:10CC700000100846F7F746FEFEF744FE99E02068EC
:10CC80004D49D1F80110884202D02068401CA8B953
:10CC900020794A490871D5F80300086023681A46CC
:10CCA00047A1012003F082FFEA794CA1012003F0A3
:10CCB0007DFF072001F07AFFF6F712FA79E020688D
:10CCC0003D49D1F80110884216D120793B490871BD
:10CCD000D5F80300086023681A4639A1012003F043
:10CCE00065FFEA793DA1012003F060FF072001F014
:10CCF0005DFF284600F08CF85BE020682E49D1F8F3
:10CD00000110884216D120792C490871D5F803000A
:10CD1000086023681A462AA1012003F047FFEA7938
:10CD20002EA1012003F042FF072001F03FFF28461B
:10CD300000F00AF93DE032480078012819D1206856
:10CD40001D49D1F80110884213D120791B4908717F
:10CD500023681A461AA1012003F028FFEA791FA1CF
:10CD6000012003F023FF072001F020FF284600F0F8
:10CD70009BF91EE020681049D1F80110884216D1B5
:10CD800020790E490871D5F80300086023681A4617
:10CD90000BA1012003F00AFFEA791AA1012003F098
:10CDA00005FF072001F002FF284600F07FF800E0B1
:10CDB00000BF00BFBDE8FE83DC060020F88B00202A
:10CDC0006465766963655F736E3D25303130753C0F
:10CDD0003078253038783E0A00000000747970659C
:10CDE0003A25780A0000000074617820696E646555
:10CDF000783A25640A000000EC060020500200206A
:10CE0000F8000020747970653A253034780A000003
:10CE100038B505460020009005F10C04A2791448AD
:10CE2000017814A0FDF724FAA07904281EDAA0796D
:10CE30000F490978884219D0A0790D49087001F08E
:10CE40005DFF0B4800788DF800009DF80000C0439E
:10CE5000C0B28DF80100022269464020F4F756FC6A
:10CE6000034802780DA1012003F0A0FE38BD0000A8
:10CE7000E8010020636F6C6C5F6C6F72615F6772BA
:10CE80006F75703A25642C20676174655F6C6F72F2
:10CE9000615F67726F75703A25640A006C6F72612A
:10CEA0002063686F6963653A25640A0070B50546BA
:10CEB00005F10C04E079012802D0022829D11BE0F9
:10CEC000B4F8050040F20121884204D112A0FDF718
:10CED000CFF9F6F705F9B4F8050040F20161884290
:10CEE00009D11048407F022805D1002003F0F6FC4C
:10CEF0000DA0FDF7BDF90CE0B4F8050040F20121EA
:10CF0000884205D1032005F04FF90CA0FDF7B0F9D8
:10CF100000BF00BF70BD000063707520726573654F
:10CF2000740A0000EC06002063697068657274651D
:10CF300078742072657365740A000000706F732046
:10CF400072657365740A000070B5044604F10C053F
:10CF5000D5F80500FAF72EFC70BD000070B5054647
:10CF600005F10C04D5F803003D490860E879087321
:10CF70002889C881207A487220680861207A0128AF
:10CF80000FD0207A02280CD0364805F0D5F9344964
:10CF9000087B00231A460421FEF7B8FD02F060FE6C
:10CFA00070BDF5F7D1FC064666B12E4805F0C4F910
:10CFB0002B49087B00231A460621FEF7A7FD02F045
:10CFC0004FFEEDE72648407A012803D1002001F00A
:10CFD000EDFD05E02248407A022801D101F0E6FD8E
:10CFE0002148407F01280FD11D48407A012803D1F4
:10CFF00003201B4908720EE01948407A02280AD122
:10D0000004201749087206E01748407F022802D121
:10D0100001201349087201224FF47A71114805F07A
:10D020006BF96089802803DD10A0FDF721F9B7E7CF
:10D0300062890B49087A04F10C0106F03FFA0848AE
:10D04000437A007A421C10A1012003F0AFFD6389EE
:10D0500004F10C0211A10120FEF7CEFD00BF9FE7F5
:10D06000F88B00200C8C0020EC0600207561727497
:10D070002073656E64206461746120746F6F206C2E
:10D080006F6E670A00000000756172743A25642CA7
:10D09000207461783A25640A0000000074617820E9
:10D0A00073656E64000000002DE9F84305464FF0FB
:10D0B000000805F10C04D5F80300DF490860B4F856
:10D0C0000500C880E0794872207A8872607AC87258
:10D0D000B4F80520D9A1002003F068FDE8795728AD
:10D0E00073D1D548C08840F2012188420CD0D9487C
:10D0F00005F022F900231A460321672000F0EEF91B
:10D1000002F0AEFDBDE8F883CB48407A01280FD08D
:10D11000C948407A02280BD0CE4805F00DF900230B
:10D120001A460421672000F0D9F902F099FDE9E7D9
:10D13000F5F70AFC07465FB1C64805F0FDF8002385
:10D140001A460621672000F0C9F902F089FDD9E7E7
:10D15000C148007878B1C0488078B8420BD0BD484B
:10D1600005F0EAF800231A460621672000F0B6F918
:10D1700002F076FDC6E7B048407A012804D1B748EE
:10D18000407F00F0030809E0AB48407A022805D14F
:10D19000B248407F00F00C084FEAA808A648C07AC1
:10D1A00000F00F00404511D0A348C07A00F00F00F6
:10D1B00060B1A84805F0C0F800231A460321672093
:10D1C00000F08CF902F04CFD9CE77BE008F00100D8
:10D1D00048B19948407A801C97490872087A012121
:10D1E00004F079FD44E09D48407F00F080008028F5
:10D1F00030D19148407A801C8F4908720846407AA5
:10D20000801C974948718C48807A401E0871207CA8
:10D21000C870B4F80B2004F10D0191480830F3F701
:10D220009DF8E07A8E49C8718348807A00908248E0
:10D23000437A007A421C8BA1012003F0B7FC884896
:10D24000C27900F108018DA0FEF78EFC572004F092
:10D2500093FF57E70320784908728B480078401CF9
:10D260008949087008460078052801DDFEF7A2F814
:10D2700001224FF47A71774805F03EF8B4F80B00BC
:10D28000802803DD81A0FCF7F3FF3BE7B4F80B2017
:10D290006949087A04F10D0106F010F96648807AB0
:10D2A00000906548437A007A421C6EA1012003F089
:10D2B0007DFCB4F80B3004F10D027BA10120FEF7D8
:10D2C0009BFCB7E0E879542841D15B48C08840F620
:10D2D000041188420BD05F4805F02EF800231A464F
:10D2E0000321642000F0FAF802F0BAFC0AE70220F9
:10D2F00051490872042001F059FC01224FF47A715F
:10D30000544804F0F9FFB4F80B00E52803DD5FA0F2
:10D31000FCF7AEFFF6E6B4F80B204749087A04F1B3
:10D320000D0106F0CBF84448807A00904248437AD9
:10D33000007A421C4BA1012003F038FCB4F80B30FA
:10D3400004F10D025BA10120FEF756FC72E0E879C2
:10D350005C286FD1667B0096237AE27958A1012080
:10D3600003F024FCB4F8050040F20151884208D0D3
:10D3700000231A4603216C2000F0B0F802F070FC84
:10D38000C0E62D48407A01280CD02B48407A02286C
:10D3900008D000231A4604216C2000F09FF802F008
:10D3A0005FFCAFE6032E08DD00231A4605216C2042
:10D3B00000F094F802F054FCA4E6012E30DC1E4884
:10D3C000807A18B11C48807A042808DD00231A46A8
:10D3D00004216C2000F082F802F042FC92E616482C
:10D3E000807A022815DD1448407A012808D00023ED
:10D3F0001A4604216C2000F071F802F031FC81E63D
:10D400000D48807A801EC1B232460120FEF7ECF84A
:10D410000EE0094A917A507A3246FEF7E5F807E0C5
:10D42000032E05DC044A917A507A3246FEF7DCF886
:10D4300002F016FC00BF65E6F88B0020705F6D738C
:10D44000675F6465765F747970653A253034780A71
:10D45000000000000C8C00201F8C0020EC06002037
:10D46000E0A60020756172743A25642C20746178FE
:10D470003A25642067756E3A25640A00CAD5B5BDA1
:10D48000D6B8C1EE20000000158C002075617274C2
:10D490002073656E64206461746120746F6F206C0A
:10D4A0006F6E670A000000007461782073656E6417
:10D4B000000000007873702073656E640000000047
:10D4C000706F72743A25642C2067756E3A25642C4F
:10D4D000206F726465723A25640A00002DE9F041FC
:10D4E000C0B006460D4690461F4603AC3148D0F802
:10D4F000010020603048007920712F48C088A4F8CE
:10D5000005002D48407AE0712B48807A20722A4825
:10D51000C07A6072A572012D08D1A4F80B703A464A
:10D52000414604F10D00F2F719FF02E00020A4F8D3
:10D530000B00672E0FD1042D0DD0E079401EC0EBFB
:10D54000C00000EB80001D49085C012803D140F2B7
:10D550000170A4F80500B4F80B000D3082B231461A
:10D56000684600F091FB012D17D19DF807006C284B
:10D5700009D1BDF80A000C3083B26A4610A101201F
:10D58000FEF73AFB12E0BDF80A000C3083B26A469F
:10D590000FA10120FEF730FB08E0BDF80A000C30B7
:10D5A00083B26A460EA10120FEF726FB40B0BDE81B
:10D5B000F0810000DC060020F88B00202B8C00207E
:10D5C000656E636F6465722072657475726E0000BB
:10D5D000627573696E6573732072657475726E001F
:10D5E0006572722072657475726E000070B50546C2
:10D5F00005F10C04D5F803000C490860B4F80500E7
:10D60000C880E0794872E079012808D0E0790228E2
:10D6100005D00420FDF788FF02F022FB70BD012039
:10D62000FDF782FF02F01CFB00BFF7E7F88B00203C
:10D630002DE9FC5F06464FF00009CA46002700248A
:10D64000A046F848807F01280ED00120F549887750
:10D650000020F5490870F549D1F80100F2F776FE8F
:10D66000F348002101600171F1480078032809D1D5
:10D67000F179F0A0FCF7FCFD42F21071012002F0FC
:10D68000C1FDDDE2F079132806D0142874D01528E6
:10D6900073D0162872D18DE206F10C07F179E5A05E
:10D6A000FCF7E6FDD7F802103888FEF7E1FB00280A
:10D6B00077D0F888F968B0EB114F72D10220DC49BD
:10D6C00008703869B0F5003F0CD9262006F0A2F8A2
:10D6D00042F21071012002F095FDDAA0FCF7C8FDBE
:10D6E000BDE8FC9FD248C07828BB0120D049C87053
:10D6F0000020FEF70DFB4FF40031D548F4F785FF0D
:10D7000081464946D3A0FCF7B3FD4FF4C471D54818
:10D71000F2F73DFED449012002F0ECFD212006F095
:10D7200079F800211020F4F74DFB02F0ADFB012148
:10D730000846F5F76BFC0620BD4948703946C948D4
:10D7400001F00CFDC748008CC649B1F85811484398
:10D7500000F6B830C549086008460068C2498842EA
:10D7600016D9C3A0FCF784FDC04800684FF47A7155
:10D77000B0FBF1FB594602E02BE0F4E050E2C3A01D
:10D78000FCF776FD42F21071012002F03BFDA7E7A5
:10D79000B6480168012002F01DFDB248028C816983
:10D7A00000E010E0BFA0FCF763FDB04800684FF454
:10D7B0007A71B0FBF1FBAB48B0F858115A46C3A0E0
:10D7C000FCF756FD04E042F21071012002F01AFD50
:10D7D00035E206F10C04D4F802102088FEF748FB6D
:10D7E00000287CD092484078072879D102209049BF
:10D7F0000870207C802800DD72E7E0899949898CD7
:10D80000884200DA6CE7A0899649098C884268D181
:10D810009448008DE189CDE90010A389D4F8022055
:10D820002188B4A0FCF724FD227CE189491E884BA5
:10D8300003EBC11004F11101F4F796FE8948858CC1
:10D840001CE08848008D401C864908850846C28C2B
:10D85000C08C401C0B46D88401F12A0020F81250DD
:10D860002A38008D962808D142F21071012002F06A
:10D87000C9FC222005F0CEFF32E76D1CE089A842EA
:10D88000DFD8E089401C77498884E089098C884288
:10D8900028D17448008D40B9092065494870A3A07B
:10D8A000FCF7E6FC02F0ECF93AE0F2F745FD462120
:10D8B00090FBF1F201FB120000F5967B5946012026
:10D8C00002F0DCFC42F21071012002F0E9FC0021C0
:10D8D000084602F07FFC99A0FCF7CAFC20E037E084
:10D8E00028E03FE05F48008CE189401A5D49B1F8CB
:10D8F0005811484300F6B8305C4908600846016892
:10D90000012002F067FC594800684FF47A71B0FBBF
:10D91000F1FB5448B0F858115A466CA0FCF7A8FC2B
:10D920005048008CE189A0EB010A01215046F4F730
:10D9300095FB17E0202005F06DFF42F210710120E9
:10D9400002F060FC49480168002002F043FC09E055
:10D9500042F21071012002F055FC44480168002099
:10D9600002F038FC6BE106F10C04D4F802102088B8
:10D97000FEF77EFA002853D02D484078082850D171
:10D9800002202B490870207C802800DDA8E6A089B1
:10D990003449098C88423DD1002520E031482A30A5
:10D9A00030F81500E189884218D12E48008D401EBC
:10D9B0002C49088500212B482A3020F81510227C9C
:10D9C000E189491E224B03EBC11004F11101F4F768
:10D9D000CBFDE1895EA0FCF74BFC04E06D1C214807
:10D9E000C08CA842DAD800BFE2891E48018D5FA032
:10D9F000FCF73EFC1B48008D28B909200C494870F3
:10DA000002F03EF96CE61748B0F828A00121504614
:10DA1000F4F724FB42F21071012002F041FCC8E04F
:10DA2000C2E0BBE0EC060020D0020020DC060020B3
:10DA3000D1020020705F6D73672D3E747970653A76
:10DA400025780A00D7DCB3A4B6C8CCABB4F30A007F
:10DA500000000608666C61736820666C61673D258E
:10DA6000640A0000F49B0020A0BB0D00D802002037
:10DA7000636F6E74696E756F75732074696D652060
:10DA8000746F206C6F6E670A000000006F74612075
:10DA9000636F6E74696E756F75732074696D653A26
:10DAA00025750A006F74615F746F746C655F6279CD
:10DAB00074653A25642C206F74615F746F746C65B3
:10DAC0005F706B673A25640A0000000073656E643E
:10DAD00020696E74657276616C3A25642C20636FE0
:10DAE0006E74696E756F75732074696D653A25641F
:10DAF0000A00000075706461746520636F6E74695C
:10DB00006E7565733A2074797065203D20307825F4
:10DB1000782C206964203D20307825782C207B25C6
:10DB2000642F25642F25647D0D0A000063686563FA
:10DB30006B20626567696E0A00000000726574728E
:10DB4000616E736D697420626567696E0A0000001A
:10DB50007263762072657472616E736D6974207081
:10DB60006B6769643A25640A000000006F74615FA6
:10DB7000696E666F2E6C6F7373506B67436F756E53
:10DB8000746572203D2025642C206C6F7373506B7C
:10DB90006749643A25640D0A0000000042F21071E2
:10DBA000012002F02FFB04E042F21071012002F08C
:10DBB00029FB44E02348007828BB06F10C08B8F89C
:10DBC000000040F2012188421ED1D8F802001E490F
:10DBD000D1F80110884217D101201A490870404637
:10DBE00001F0BAF90120194981F8290002201549EC
:10DBF000087117A0FCF73CFBD8F80E20D8F80810E5
:10DC000019A0FCF735FB0AE00F480078012803D182
:10DC100000200E49887702E003200C4988770EE047
:10DC20000848007850B908480078012803D100203E
:10DC30000649887702E003200449887700BF00BFC7
:10DC400000BF4DE5D1020020DC060020EC060020DC
:10DC5000CDF8B9D8CFC2B7A2BFAACABCC0EBCFDF3C
:10DC6000C9FDBCB60A000000736C61766520736E56
:10DC70003A25303130752C2064657320736E3A2557
:10DC8000303130750A0000002DE9F04104460E469F
:10DC9000154600274FF6FE6020800120A07019482D
:10DCA0000068C4F80300E671012E03D142F252006D
:10DCB000208101E000202081A81C608104F10C007B
:10DCC00000EB0508608900F10A012046F4F706F927
:10DCD000A8F80000022001F06DFB074667B105F1CE
:10DCE0000E0221463846F2F739FB05F10E0239469D
:10DCF000022001F021FB03E03946022001F08EFBF7
:10DD0000BDE8F081F88B00202DE9F04704460E466F
:10DD100017469846DDE908A54FF6FE602080A670FC
:10DD2000C4F8037084F80780A4F808A0A81C6081D8
:10DD3000608900F10A012046F4F7D0F8814604F129
:10DD40000C0000F805904FEA1922691C425405F1B5
:10DD50000E022146022001F0EFFA05F10E0082B218
:10DD6000214602A0FDF700FFBDE8F0876C6F7261ED
:10DD70002073656E6400000010B5002404210E4875
:10DD8000F4F774FD08B144F0010408210A48F4F7DF
:10DD90006DFD08B144F0020410210748F4F766FD58
:10DDA00008B144F0040420210348F4F75FFD08B1F2
:10DDB00044F01004204610BD0018014070B5044620
:10DDC0000D46164633462A4621460A48F3F7B0FB6D
:10DDD00001210848F3F70DFC0120F3F71BFC00BFFD
:10DDE00002210448F3F768FB0028F9D00148F3F753
:10DDF0005FFB70BD002401402DE9F04104460D4653
:10DE000016460027BEB904EB4402184B03EB02127E
:10DE100005EB450302EBC302118A04EB4402134BEA
:10DE200003EB021205EB450302EBC302D068F4F7E3
:10DE30001DFD074617E0012E15D104EB44020B4BE4
:10DE400003EB021205EB450302EBC302918804EBDE
:10DE50004402064B03EB021205EB450352F8330074
:10DE6000F4F704FD07463846BDE8F081D89200205B
:10DE700070B504460025012C05D101020348F4F7D2
:10DE8000F5FC054600E00125284670BD000801406C
:10DE900000EB8001174A02EB41010968164A116044
:10DEA00000EB8001134A02EB41010979134A11701A
:10DEB00000EB80010F4A02EB41014979104A1170D1
:10DEC00000EB80010B4A02EB410189790D4A117088
:10DED00000EB8001074A02EB4101C9790A4A11703F
:10DEE00000EB8001034A02EB4101097A074A1170F5
:10DEF00070470000F5010020EC010020F001002037
:10DF0000F1010020F2010020F3010020F4010020C3
:10DF1000002002490868024A10807047002004E08F
:10DF2000CA01002006480068064908600448001D30
:10DF30000068486002480830006888607047000048
:10DF4000E8F7FF1FF473002010B502460B460020CF
:10DF5000002103E0545C60404C1CA1B29942F9DB03
:10DF600010BD000070B504460D4604EB8401214A43
:10DF700002EB411105EB850201EB021101F14600B4
:10DF800004F0DAF904EB84001A4901EB401005EBC8
:10DF9000850100EB011090F82F00401CC1B204EB8A
:10DFA0008400144A02EB401005EB850200EB0210DE
:10DFB00080F82F10002104EB84000E4A02EB401081
:10DFC00005EB850200EB021080F82E10002004EB18
:10DFD0008401084A02EB411105EB850201EB0211B5
:10DFE000487005480068054901EB441101EB051133
:10DFF000886070BD3893002020000020E898002041
:10E0000070B500206CE0002166E001EB4004364D65
:10E010002B5D01EB4004354D2A5D02EB4204344D8B
:10E0200055F8244000EB4005324E06EB051501EB98
:10E03000410605EBC605EC6002EB42042C4D05EBF6
:10E040008404A58800EB40042A4E06EB041401EB7F
:10E05000410604EBC604258202EB4204244D05EB85
:10E060008404A56800EB4004224E06EB041401EB87
:10E07000410604EBC604656103EB43041C4D55F8EF
:10E08000244000EB40051B4E06EB051501EB410655
:10E0900045F8364003EB4304154D05EB8404A48892
:10E0A00000EB4005134E06EB051501EB410605EBB1
:10E0B000C605AC8003EB43040D4D05EB8404A46856
:10E0C00000EB40050B4E06EB051501EB410605EB99
:10E0D000C605AC604C1CE1B2022996DB441CE0B2E0
:10E0E000022890DB70BD0000B8020020BC020020B6
:10E0F00058020020D892002070B504460D46002139
:10E1000004EB8400154A02EB401005EB850200EB9E
:10E11000021080F82E10012004EB84010F4A02EB5C
:10E12000411105EB850201EB0211487004EB8401FB
:10E130000A4A02EB411105EB850201EB021101F1E4
:10E1400046000122064904F0D7F80648006806494F
:10E1500001EB441101EB0511486070BD38930020BC
:10E16000E093040020000020E898002070B500240F
:10E1700058E0002553E0E9B2E0B20022FFF73CFE90
:10E1800004EB8401294A02EB411105EB850201EB06
:10E19000021181F82C00E9B2E0B20122FFF72CFE57
:10E1A00004EB8401214A02EB411105EB850201EBEE
:10E1B000021181F8390004EB84001C4901EB401086
:10E1C00005EB850100EB011090F82C0000BB01204D
:10E1D00004EB8401154A02EB411105EB850201EBCA
:10E1E0000211487004EB8401104A02EB411105EB67
:10E1F000850201EB021101F1460001220C4904F0F5
:10E200007BF86B1C621C0BA1012002F0CFFC05E027
:10E210006B1C621C0CA1012002F0C8FC6D1C022DBD
:10E22000A9DB641C022CA4DB70BD00003893002025
:10E23000E09304007461783A25642C67756E3A2582
:10E24000642CCCA7C7B90A007461783A25642C679E
:10E25000756E3A25642CB9D2C7B90A0070B500248E
:10E260004AE0002544E004EB8401254A02EB411119
:10E2700005EB850201EB021101F1300004F002F818
:10E28000002833D0002229462046FFF7B5FD064678
:10E2900004EB84001A4901EB401005EB850100EB0B
:10E2A000011090F82C00B04215D056B129462046F6
:10E2B000FFF758FE6B1C621C12A1012002F076FCD5
:10E2C00009E029462046FFF717FF6B1C621C13A1CB
:10E2D000012002F06BFC04EB8400094901EB4010C3
:10E2E00005EB850100EB011080F82C60681CC5B2BD
:10E2F000022DB8DB601CC4B2022CB2DB70BD000082
:10E3000038930020743D25642C20673D25642C67DC
:10E31000756E20646F776E0A00000000743D2564FE
:10E320002C20673D25642C67756E2075700A0000EF
:10E330002DE9F04706460F4690464FF000090025AC
:10E34000BA464FF4A0710B48F2F721F800240BE015
:10E3500016F80490074948194B4607A24FF4A071DC
:10E36000FBF796FF0544641C5445F1DBA8F8005008
:10E37000BDE8F08732990020253032780000000097
:10E380002DE9F04104460F4615461E46601E00EB7F
:10E39000401077490844007920B101284AD002286A
:10E3A0007ED1B6E02046FFF763FD002841D1601E14
:10E3B00000EB40106E4908444079022822D1611ECA
:10E3C00001EB41116A4A114401F10F0003F05AFFB9
:10E3D00080B10121601E00EB4010654A10440171BC
:10E3E000611E01EB41111144881D0122394603F0E1
:10E3F00083FF17E00221601E00EB40105C4A1044CE
:10E4000001710FE00121601E00EB4010584A1044DA
:10E410000171611E01EB41111144881D0122394631
:10E4200003F06AFF0021601E00EB4010504A1044C8
:10E43000417199E02046FFF71BFD00285BD10121C7
:10E44000601E00EB40104A4A10444171611E01EB0E
:10E4500041111144881D03F015FF002858D0601E9B
:10E4600000EB401042490844407880B90121601E09
:10E4700000EB40103E4A10444170611E01EB411117
:10E48000114401F118000122314603F035FF601EEE
:10E4900000EB4010364908448078401CC1B200E0CF
:10E4A00054E0601E00EB4010314A10448170601E41
:10E4B00000EB401011460844C078401CC1B2601EF9
:10E4C00000EB40101044C170601E00EB401011467C
:10E4D0000844C378601E00EB40100844827821464F
:10E4E00024A0FBF7C5FE0221601E00EB4010204A6D
:10E4F000104401710CE00021601E00EB40101C4A2A
:10E50000104401710121601E00EB40101044417164
:10E510002AE02046FFF7ACFCB8B10021601E00EBFA
:10E520004010134A10440171611E01EB4111114466
:10E5300001F10F000122294603F0DEFE0221601ED8
:10E5400000EB40100A4A104441710DE00021601EAA
:10E5500000EB4010064A104401710321601E00EBDD
:10E5600040101044417100BF00BFBDE8F0810000C1
:10E57000043400206B65793A25642C206B65792082
:10E580006E756D3A25642C206B657920746F74610B
:10E590006C206E756D3A25750A00000008B50320E1
:10E5A00004239A01024900901846F4F74FF808BD79
:10E5B0000008014070B56424642541F28836334672
:10E5C0002A4621460120FFF7DBFE0C48407898B12F
:10E5D0000A48183003F056FE70B10948807F18B120
:10E5E0000748807F032803D10449887800F00AF89F
:10E5F000002002494870887070BD0000043400207B
:10E60000EC06002010B50446062C24D2DFE804F006
:10E610002303191A1B1C012010490870012240F61F
:10E62000B8310F4803F068FEFCF7DAFE012204213E
:10E630000C480078401CF3F72DFD01200A490870B2
:10E640000AE009E008E007E00120084981F8290014
:10E650000749087100E000BF00BF10BDFB000020AB
:10E66000C1340020E801002004340020EC06002022
:10E67000D102002010B563211548F1F788FEFF2074
:10E68000134908704FF4FA70C1F805004FF4967101
:10E690000F48C0F81710C0F80E10C0F8291001621A
:10E6A000C0F83210C0F83B100A48807F032808D118
:10E6B000FF20074981F851004FF496710448C0F8D3
:10E6C00056104FF4967102484164C0F84D1010BDC9
:10E6D00067340020EC06002010B54848007818B1D7
:10E6E000474803F029FE15E04648807F032809D1FA
:10E6F0004348513890F8510060B9FF21404803F079
:10E7000011FE07E03E48513890F8510010B13C48E6
:10E7100003F012FE3A48513803F0B4FD38B13A48DC
:10E72000006808B9012000E000203749086034483B
:10E7300003F0A8FD60B135480178FF20F4F766FCCE
:10E740003248007808B9012000E000202F49087005
:10E750002B483F3803F096FD18B101210846F4F725
:10E7600055FC2748483803F08DFD18B101210020E1
:10E77000F4F74CFC22482D3803F084FD18B1012138
:10E780000320F4F743FC1E48363803F07BFD18B134
:10E7900001210220F4F73AFC1948243803F072FDF5
:10E7A00018B101210720F4F731FC15481B3803F09C
:10E7B00069FD18B101210620F4F728FC1048123831
:10E7C00003F060FD18B101210520F4F71FFC0C488F
:10E7D000093803F057FD18B101210420F4F716FCA5
:10E7E0000748093003F04EFD38B100200849087091
:10E7F000FCF7F6FD00200149087010BD043400202C
:10E80000B8340020EC060020B8012342FA000020B2
:10E81000FB00002070B505460C46BC480078002877
:10E8200073D1042D49D007DC7DB1012D1BD0022D01
:10E8300027D0032D6AD132E0052D4BD0062D56D0BE
:10E84000072D64D0FF2DF5D16FE0012C04D12103F9
:10E85000AF48F4F714F805E024B94FF48051AC4800
:10E86000F4F70FF87BE0012C04D16103A848F4F71A
:10E8700006F805E024B94FF40051A548F4F701F873
:10E880006DE0012C04D1A103A148F3F7F8FF05E0E6
:10E8900024B94FF480419E48F3F7F3FF5FE0012C69
:10E8A00004D1E1039A48F3F7EAFF05E024B94FF4F5
:10E8B00000419748F3F7E5FF51E0012C04D14021D6
:10E8C0009448F3F7DCFF04E01CB940219148F3F7CA
:10E8D000D8FF44E0012C04D180218E48F3F7CFFF0C
:10E8E00004E01CB980218B48F3F7CBFF37E0012C03
:10E8F00004D121028748F3F7C2FF05E024B94FF4A1
:10E9000080718448F3F7BDFF29E029E026E0012C5F
:10E9100004D161027F48F3F7B2FF05E024B94FF458
:10E9200000717C48F3F7ADFF19E0012C0AD14FF4D8
:10E9300070417748F3F7A3FF4FF470717548F3F710
:10E940009EFF0AE04CB94FF470417148F3F799FF0C
:10E950004FF470716F48F3F794FF00E000BFD4E00C
:10E960006A4800780128FAD1042D65D007DC7DB112
:10E97000012D22D0022D35D0032D72D147E0052D77
:10E9800073D0062D6FD0072D6ED0FF2DF5D1ABE0E3
:10E99000012C06D16048007820F001005E49087023
:10E9A00006E02CB95C48007840F001005A49087034
:10E9B0005948007800F0B2F8A6E0012C06D156487C
:10E9C000007820F002005449087006E02CB9524843
:10E9D000007840F00200504908704F48007800F07D
:10E9E0009DF891E0012C06D14B48007820F00400FE
:10E9F0004949087006E02CB94748007840F0040007
:10EA0000454908704448007800F088F87CE0012C03
:10EA100006D14148007820F008003F49087006E020
:10EA20002CB93D48007840F008003B4908703A484E
:10EA3000007800F073F867E0012C06D136480078C2
:10EA400020F010003449087006E02CB932480078F4
:10EA500040F01000304908702F48007800F05EF850
:10EA600052E050E001E015E029E0012C06D12A48EF
:10EA7000007820F020002849087006E02CB92648CC
:10EA8000007840F02000244908702348007800F006
:10EA900045F839E0012C06D11F48007820F04000ED
:10EAA0001D49087006E02CB91B48007840F0400072
:10EAB000194908701848007800F030F824E0012C5B
:10EAC00006D11548007820F080001349087006E050
:10EAD0002CB91148007840F080000F4908700E48AA
:10EAE000007800F01BF80FE0012C03D100200A4948
:10EAF000087003E014B9FF20074908700648007841
:10EB000000F00CF800E000BF00BF70BDF80000206E
:10EB10000014014000100140F900002070B50446C7
:10EB20004FF480512048F3F7AAFE0220FDF77BF84E
:10EB30004FF400511C48F3F7A4FE0420FDF773F8CE
:10EB4000002521E004F0800028B14FF40061164850
:10EB5000F3F797FE04E04FF400611348F3F78FFEDC
:10EB60006006040E4FF400510F48F3F788FE0420AE
:10EB7000FDF759F84FF400510B48F3F782FE0420DB
:10EB8000FDF751F8681CC5B2082DDBDB4FF480514E
:10EB90000548F3F776FE0420FDF745F84FF4805161
:10EBA0000148F3F76CFE70BD0018014010B5044633
:10EBB0003048807F00285CD12F480078002858D149
:10EBC000082C54D2DFE804F00D042117493F352BFF
:10EBD00001212A4803F0A6FB00210120F4F716FAD0
:10EBE00046E001212548093803F09CFB0021084636
:10EBF000F4F70CFA3CE001212048123003F092FBBC
:10EC000000210320F4F702FA32E001211B48093009
:10EC100003F088FB00210220F4F7F8F928E0012135
:10EC200016481B3003F07EFB00210720F4F7EEF9B5
:10EC30001EE001211148243003F074FB002106205E
:10EC4000F4F7E4F914E001210C482D3003F06AFBDD
:10EC500000210520F4F7DAF90AE0012107483630EF
:10EC600003F060FB00210420F4F7D0F900E000BFBE
:10EC700000BF10BDEC060020FB000020793400200E
:10EC80003EB50446012C04D140211B48F3F7F9FDA1
:10EC900010E0022C04D180211748F3F7F2FD09E0BF
:10ECA000032C07D140211448F3F7EBFD80211248D3
:10ECB000F3F7E7FD02A8002164230A46CDE900101E
:10ECC0000846F5F71FFE012C04D140210A48F3F74E
:10ECD000D6FD10E0022C04D180210748F3F7CFFDC8
:10ECE00009E0032C07D140210348F3F7C8FD802138
:10ECF0000148F3F7C4FD3EBD0018014010B58AB0CD
:10ED000031483249086032488860324848603248A9
:10ED1000C86032480861324888610220FFF7B0FFBE
:10ED200030480078FFF7B4F82F4801682748884733
:10ED30002D48C1682D48006888474FF47A7000213B
:10ED400005910691CDE9071001210022284800789D
:10ED5000284B1B78CDE90130CDE903212648007806
:10ED600000902148C469254803782548007841B2BD
:10ED70000120A047002006900790089009900120EC
:10ED8000002102910391CDE9041019480078CDE9E2
:10ED90000010154884691748037817480278174807
:10EDA00001780120A0474FF4FA630A2216210120BE
:10EDB000F9F7AEFE0C48416B00208847012011494D
:10EDC00008700AB010BD000095900208D08700209E
:10EDD000798F0208B5900208599002082190020824
:10EDE000BD8E0208E8010020483B0308EC0100202A
:10EDF000F4010020F3010020F2010020F1010020C5
:10EE0000F0010020E001002030B5E3B026AC002581
:10EE1000802102A8F1F7BBFA33A0FBF729FA3848A2
:10EE2000008CA0818020207435480088E080344820
:10EE30004068A0603248C068C4F8020030480089C9
:10EE400020808C210120F9F7B3FA0546B5F5967FAD
:10EE500001D9284601E04FF496700546294629A0BD
:10EE6000FBF706FA2648018C2AA0FBF701FA32E0EC
:10EE70002348428C018C2FA0FBF7FAF92048408CE4
:10EE8000E0811F48408C401C1D494884E189491E8F
:10EE9000304A02EBC110802202A9F3F744FB802222
:10EEA00002A904F11100F1F759FA9122142123A8C3
:10EEB000FCF79AFD1249098C114A528C881A0121DB
:10EEC000F3F7CCF822A800212B460A46CDE9001022
:10EED0000846F5F717FD0A48408C0949098C884215
:10EEE000C6DD63B030BD00006C6F72615F67775F35
:10EEF0006F74615F636F6E74696E7565730D0A0080
:10EF00007C9D002074696D6572203D2025640D0A8A
:10EF1000000000006C6F72615F7570646174652041
:10EF2000746F74616C5F706B6773203D2025640D96
:10EF30000A0000006C6F72615F67775F6F74615FDA
:10EF4000636F6E74696E756573207B25642F25640D
:10EF50007D0D0A000000020810B504464FF4C4718C
:10EF60000C48F1F714FAA0890A490880D4F80E0079
:10EF70004860E0880881A068C86007480068486168
:10EF800000208861C86108840120888448840020AA
:10EF900010BD00007C9D0020EC06002070B50446EA
:10EFA0000D464FF4C4711348F1F7F1F91248B0F867
:10EFB0000500104908804FF0FF304860C8600E48D7
:10EFC000B0F8050008810D48006848610846846172
:10EFD000C561C4F3CF1008840120888404F07F0049
:10EFE00018B10846008C401C08840120014948845F
:10EFF000002070BD7C9D0020DC060020EC06002077
:10F0000070B50446002515480078032805D142F262
:10F010001071012001F0F6F870BDE07921280FD0C1
:10F02000222802D0232815D10BE004F10C05284634
:10F0300000F016F843F69821012001F00DF90AE0DE
:10F0400009E043F69821012001F006F9204600F07E
:10F0500075FD00E000BF00BF00BFDDE7D10200206A
:10F0600030B5E1B0054624AC802101A8F1F78FF955
:10F070001448008CA081E888E08180202074114829
:10F080000088E0800F484068A0600E48C068C4F85F
:10F0900002000C4800892080E988491E0A4A02EBD8
:10F0A000C110802201A9F3F73EFA802201A904F1E0
:10F0B0001100F1F753F99122152121A8FCF794FCD6
:10F0C00061B030BD7C9D00200000020830B5C1B0A9
:10F0D000002504AC16480088E08015484068A06010
:10F0E0001348008920801248C068C4F80200104804
:10F0F0004069E0600E48806920618C210120F9F7A9
:10F1000057F90546B5F5967F01D9284601E04FF439
:10F1100096700546A58221692A4606A0FBF7A8F845
:10F120001622132101A8FCF75FFC41B030BD00009E
:10F130007C9D0020746F74616C5F627974657320CC
:10F140003D2025642C2073656E6420696E746572A1
:10F1500076616C203D2025640A0000000246088884
:10F160001081D1F80200D060C88810808868506093
:10F17000C8685061086990610869C0F3CF101084B5
:10F180000020D08401209084087C00F07F0010B122
:10F19000108C401C10840020108501205084888A27
:10F1A000A2F85801002070477FB50546012D28D1EF
:10F1B00021E003A800231A46194600902648F4F7D8
:10F1C000E7FC03A8002102AB4FF40042CDE9001098
:10F1D00021483038F4F7C4FA044603AA4FF400710A
:10F1E0001D48F4F7C5FD34B1BDF8080018B121463B
:10F1F000012000F013F91948B0F82A080028D8D1E6
:10F2000029E0022D27D121E003A800231A46194640
:10F2100000901348F4F7BCFC03A8002102AB4FF4A4
:10F220000042CDE900100E483038F4F799FA044650
:10F2300003AA4FF400710A48F4F79AFD34B1BDF8FF
:10F24000080018B12146022000F0E8F80548B0F89F
:10F250002A080028D8D17FBD807D0020507500206D
:10F260002C860020FC7D00200EB502AB012218A1E7
:10F270001A48F4F74DFC02AB082219A117483038A0
:10F28000F4F7EEF902A84FF480710823184ACDE98B
:10F29000001018A102F65800F4F7C6F802AB0122DC
:10F2A00018A11B48F4F734FC02AB082219A1184836
:10F2B0003038F4F7D5F902A84FF480710823194AC1
:10F2C000CDE9001018A102F65800F4F7ADF80EBD14
:10F2D0006C6F72615F73656D5F727800807D002076
:10F2E0006C6F72615F71756575655F7278000000A3
:10F2F000507500206C6F72615F6D656D6F72795F24
:10F30000727800006C6F72615F73656D5F74780076
:10F310002C8600206C6F72615F71756575655F7416
:10F3200078000000FC7D00206C6F72615F6D656D80
:10F330006F72795F74780000FEB504460E4615467C
:10F34000012C18D102A800231A461946009017482C
:10F35000F4F71EFC02A80021AAB20B46CDE900106A
:10F36000314612483038F6F713FA02AA61020F4804
:10F37000F4F7FEFC19E0022C17D102A800231A466C
:10F38000194600900A48F4F703FC02A80021AAB22B
:10F390000B46CDE90010314605483038F6F7F8F94C
:10F3A00002AA21020248F4F7E3FCFEBD807D0020A2
:10F3B0002C8600207CB504460025012C13D101A821
:10F3C00000231A46194600901248F4F7E1FB01A900
:10F3D00010482830F4F7DAF8054601AA61020D4812
:10F3E000F4F7C6FC14E0022C12D101A800231A463F
:10F3F000194600900848F4F7CBFB01A906482830CD
:10F40000F4F7C4F8054601AA21020348F4F7B0FC5A
:10F4100028467CBD807D00202C8600207CB50446DB
:10F420000D46012C13D101A800231A46194600905D
:10F430001348F4F7ADFB01AA294611482830F4F728
:10F44000D7F801AA61020E48F4F792FC14E0022CEE
:10F4500012D101A800231A46194600900948F4F772
:10F4600097FB01AA294607482830F4F7C1F801AAFA
:10F4700021020448F4F77CFCBDF804007CBD0000C8
:10F48000807D00202C8600202DE9FF4100240026ED
:10F4900003A800231A46194600906548F4F778FB44
:10F4A00003A8002102AB4FF40042CDE900106048F0
:10F4B0003038F4F755F9044603AA4FF400715C485C
:10F4C000F4F756FC002C73D0BDF808000028FAD0E1
:10F4D00020884FF6FE61884208D056A0FAF7C8FE91
:10F4E00021460120FFF79AFFBDE8FF8160890C30BB
:10F4F000BDF80810884207DD52A0FAF7B9FE214690
:10F500000120FFF78BFFEFE76089801E04F10C01FB
:10F510000F5A608900F10A012046F2F7DFFC054628
:10F520004C48807F02287DD0A078012863D1E07903
:10F5300000F0F000502811D1AF4207D046A0FAF7F2
:10F5400097FE21460120FFF769FFCDE74148807F04
:10F55000002867D12046FDF74DFA63E0E07900F01E
:10F56000F00010280DD100F027FA3E48007801285D
:10F5700058D03848807F042854D02046FEF758F8E9
:10F5800050E0E07900F0F000202812D100F014FAE9
:10F590003048807F012845D132480078012803D0C7
:10F5A0003048007803283DD12046FFF729FD39E097
:10F5B0003CE0E079012835D104F10C0670682A4955
:10F5C000D1F8011088422DD1208941F252018842A0
:10F5D00028D173681A4625A1012001F0E7FA228993
:10F5E000E17929A0FAF744FE0720FFF7DFFA204669
:10F5F000FDF7B4FC16E0A078032808D11548807FF9
:10F6000080B9BDF808102046FCF75EFA0AE0A07841
:10F61000FF2807D10F48807F20B9BDF80810204689
:10F62000FCF761FA21460120FFF7F8FE00BF5BE717
:10F63000807D0020686561646572206572726F72FA
:10F640000A000000646174616C656E206572720A64
:10F6500000000000EC060020637263206572720AED
:10F6600000000000D1020020DC06002064657669FD
:10F6700063655F736E3D25303130753C30782530E1
:10F6800038783E0A0000000066697273742074794D
:10F6900070653A25782C207365636F6E64207479E9
:10F6A00070653A25780A00007FB503A800231A4642
:10F6B000194600903948F4F76BFA03A8002102AB11
:10F6C0004FF40042CDE9001034483038F4F748F8E0
:10F6D0000446002C61D0BDF8080000285DD0BDF8BC
:10F6E0000800C1B22E48826A20469047BDF8083013
:10F6F00022462CA10020FCF77FFA0620FFF756FADD
:10F7000000F05AF92948807F01283CD12848007828
:10F71000022810D12648407808280CD1F0F70CFEBA
:10F72000462190FBF1F201FB120000F59675294687
:10F73000012000F0A3FD1E480078042823D11D48B5
:10F740000078401C1B490870084601781AA0FAF797
:10F750008FFDBDF8082021461BA0FCF705FA1548CF
:10F76000007805280DDAF0F7E7FD462190FBF1F26D
:10F7700001FB120000F596752946012000F0CCFD32
:10F7800001E001F005FF03AA4FF400710348F4F70C
:10F79000EFFA21460220FFF741FE7FBD2C860020B4
:10F7A000483B03084C4F524120547800EC0600209F
:10F7B000D10200200CA40020736C61766520736573
:10F7C0006E6420256420000074696D65730000007C
:10F7D00030B5C1B0054604AC1048B0F80500208033
:10F7E0000E48D0F80100C4F802000C48B0F805003B
:10F7F000E0800A48D0F80100A06009484068E06055
:10F8000007480068206125750020C4F815001922FA
:10F81000232101A8FCF7E8F841B030BDDC06002048
:10F82000EC06002070B504460D4626463089A0F54A
:10F830008050523820B92946204602F081FD00E070
:10F8400000BF00BF70BD000010B55148007851499D
:10F850000978884207D04F48007820B14E480068A8
:10F860004E49C1F801004B480078494908704B489F
:10F8700002F008FD10B10020464908704848B0F871
:10F880002A0808B1FFF700FE42480078092876D21E
:10F89000DFE800F005757575254D4E4F5000414964
:10F8A000086B80474048B0F82A0850B13D49886B42
:10F8B000804706203749087000203C4981F826001F
:10F8C00006E03848416B0020884704203149087021
:10F8D0000020364981F8250081F8260053E033489E
:10F8E00090F82600A8B1324802F0CCFCF0B100201C
:10F8F0002E4981F82600084690F82500B0B92A481C
:10F90000B0F82A0890B1FFF7CFFE05202149087012
:10F910000CE0264890F8250040B92348B0F82A08A2
:10F9200020B1FFF7C1FE05201A4908702BE02AE03C
:10F9300029E000BF1F48007860B100201D49087011
:10F940001948B0F82A08C0B1FFF7AEFE05201149EA
:10F95000087012E01348416B0020884704200D49CD
:10F9600008700020114981F82500012081F8260047
:10F970000122C8210E4802F0BFFC04E0FFE700208E
:10F980000449087000BF00BF0649086E804710BDDB
:10F99000E1010020E00100202000002039020020C9
:10F9A00050750020483B0308FC7D0020D0870020D4
:10F9B000420200203802002010B5FF21054802F065
:10F9C000B1FC054802F0B8FC0020044981F82B0086
:10F9D00010BD0000260200202F020020EC060020AF
:10F9E00000B58BB00AA8F3F70DFC0AA8032100228A
:10F9F0000592CDE906210890104680210C220D4B7E
:10FA0000CDE90132CDE90310022000230A4A0BA1FF
:10FA100000900E48F4F7E0FA4FF400318802F3F753
:10FA200043FB62B60AA8F4F7DBF9F3F751FA0020BA
:10FA30000BB000BD80040020C9170208417070207F
:10FA40005461736B2053746172740000C003002012
:10FA500010B5C0B04FF480716846F0F798FC0024F0
:10FA60001AE004EB84012A4800EB8100007C2A287C
:10FA700011D104EB8401264800EB81004068244941
:10FA8000083989884DF82100214808388088401CB1
:10FA90001F4908398880641C1D4808384088A042E6
:10FAA000DFDC1B48083881881AA0FAF7E1FB184808
:10FAB000083881881B4B04226846F0F7EEFB0024CF
:10FAC0001CE0E11704EB91718910A4EB810179B975
:10FAD00074B1E11704EB5171C910A4EBC10121B954
:10FAE0001CB111A0FAF7C4FB02E010A0FAF7C0FBAA
:10FAF0005DF824100EA0FAF7BBFB641C044808381C
:10FB00008088A042DDDC0CA0FAF7B2FB40B010BD4B
:10FB10000C9F0020C9FDBCB6B3C9B9A62564B8F6D0
:10FB2000A3BA0A0015B502080D0A00002000000063
:10FB300025303130752000000A000000FEB5064671
:10FB400006F10C0444480088401C43490880207D8D
:10FB50002169E268CDE900210290A368E2883E486D
:10FB600001883E48FAF784FB3B484088402870DA19
:10FB70003948408888B3002531E005EB85013648D7
:10FB8000083000EB81004068A168884226D1E188F6
:10FB900005EB85023048083020F82210A16805EBFB
:10FBA000850200EB82004160E16805EB85022A488E
:10FBB000083000EB82008160216905EB8502264850
:10FBC000083000EB8200C160217D05EB85022248F0
:10FBD000083000EB82000174FEBD04E06D1C1E487D
:10FBE0004088A842C9DCE1881B48408800EB8002BD
:10FBF0001948083020F82210A1680838408800EB26
:10FC000080021548083000EB82004160E16812482C
:10FC1000408800EB80021048083000EB82008160D1
:10FC200021690D48408800EB80020B48083000EB4A
:10FC30008200C160217D0848408800EB80020648B0
:10FC4000083000EB8200017403484088401C0249E0
:10FC5000488000BFC0E70000049F0020443F030825
:10FC600010B514210148F0F792FB10BDF88B00206D
:10FC700010B521210148F0F78AFB10BD28A400200F
:10FC800070B55348407808287FD0092871D10021E9
:10FC9000084600F09FFA0021084600F001FB002111
:10FCA000084600F0EBFA4B48008840F201218842F8
:10FCB0002DD1002100F05AFB0546002D64D04548A7
:10FCC000008840F2012188425ED1812001F052FC7F
:10FCD00041490880084601880820F2F765F83D4848
:10FCE00040693E490861042210313120FCF74EF989
:10FCF00000BF3B48006800F4E0603A490843001D3B
:10FD000037490860BFF34F8F00BF00BFFEE731489F
:10FD1000008840F60411884236D1002100F026FB0D
:10FD20000546002D30D02B4840692C49086104223B
:10FD300010313120FCF72AF90021084600F062FA60
:10FD40000021084600F046FA0021084600F0A8FA13
:10FD50000021084600F0CEFA1D4800210160017123
:10FD600021480078012805D100202049887704E047
:10FD70000BE02BE003201D49887701201B4981F807
:10FD80002C001BA0FAF774FA20E02048B0F82A08EB
:10FD9000D8B9002414E00F482A3030F8140068B1B4
:10FDA0000C492A3131F8140000F046F809482A308D
:10FDB00030F8141016A0FAF75BFA05E0601C84B264
:10FDC0000448C08CA042E6DC00BF00BF00BF70BD8D
:10FDD000D1020020F49B0020DA0100200C740020E6
:10FDE0000CED00E00000FA05DC060020EC06002027
:10FDF000CAD5B0FCCDEAB3C9A3ACBFAACABCC9FD81
:10FE0000BCB6CFD4CABEC6C1200A0000FC7D00200B
:10FE100073656E642072657472616E736D697420AF
:10FE2000706B6769643A25640A00000010B500F041
:10FE3000DFF800F03DF910BD30B5C1B0054604ACA7
:10FE40000748008920800748D0F80100C4F8020064
:10FE5000E5800822222101A8FBF7C6FD41B030BD94
:10FE6000F49B0020DC06002010B500F07DF800F0C7
:10FE700013F800F0FDF800F053F900F0EFF800F08F
:10FE800091F900F09DF910BD10B5FBF7A9FA012119
:10FE90000320F3F7BBF810BD70B5274802F0F2F964
:10FEA000002846D02548848C1DE02448008D401C45
:10FEB000224908850846C18CC08C401C1F4AD0844A
:10FEC00002F12A0020F811402A38008D962808D126
:10FED00042F21071012000F095F9222003F09AFC03
:10FEE00070BD601C84B21548008C401CA042DCDC54
:10FEF0001248008D40B909201149487011A0FAF745
:10FF0000B7F9FFF7BDFE14E0F0F716FA462190FBB3
:10FF1000F1F201FB120000F596752946012000F070
:10FF2000ADF942F21071012000F0BAF909A0FAF718
:10FF30009FF900BFD4E70000579D0020F49B0020EC
:10FF4000D1020020636865636B20626567696E0A91
:10FF50000000000072657472616E736D69742062D6
:10FF60006567696E0A00000010B5174802F08AF94B
:10FF700040B31648002101600171084600F02AF9DB
:10FF80000021084600F08CF90021084600F0B2F983
:10FF90000F48007820B101200E4981F82A000EE0B8
:10FFA0000D480078012803D100200A49887702E033
:10FFB0000320084988770021FF20FEF72BFC07A0CB
:10FFC000FAF756F910BD00004E9D0020D102002026
:10FFD000D0020020EC060020DC0600206F6E6C6F63
:10FFE0006F6B65722074696D656F7574200A00000F
:10FFF00010B5114802F046F9E0B110480078052824
:020000040803EF
:1000000001D0FFF725FD0D48002101600171084670
:1000100000F05EF9FBF7E4F909480078012803D104
:1000200000200849887702E003200649887706A067
:10003000FAF71EF910BD0000E89E0020D102002052
:10004000DC060020EC0600206D617374657220757B
:100050007064617465206F7665720A0010B503489C
:1000600002F010F908B1FFF70BFE10BD729D0020E1
:1000700010B5084802F006F950B142F210710120A3
:1000800000F0C0F8232003F0C5FB03A0FAF7F0F856
:1000900010BD0000609D002072657472616E736D0A
:1000A00069742074696D656F7574200A0000000022
:1000B00010B5114802F0E6F8E0B1104800780528C4
:1000C00001D0FFF7C5FC0E480078012803D10020BD
:1000D0000C49887702E003200A4988770748002105
:1000E00001600171084600F0B7F8FBF779F906A046
:1000F000FAF7BEF810BD0000F19E0020D1020020EA
:10010000DC060020EC0600206D61737465722074BB
:100110006F74616C2074696D656F7574200A0000DE
:1001200010B5174802F0AEF840B31648007820B179
:100130000120154981F82A000AE0144800780128B6
:1001400003D100201049887702E003200E49887708
:100150000021084600F056F80021084600F03AF861
:100160000021084600F09CF8094800210160017157
:10017000292003F04FFB07A0FAF77AF810BD000022
:10018000699D0020D0020020EC060020DC06002043
:10019000D1020020746F74616C2074696D656F7595
:1001A00074200A0010B5044802F06CF818B1034836
:1001B0000078FFF70DFB10BD1DA40020D002002029
:1001C00010B5034802F05EF808B101F0E1F910BD86
:1001D00014A4002070B504460D46012C08D1072058
:1001E0000649487001222946054802F085F803E0D7
:1001F00014B9034802F0A0F870BD0000D10200203D
:10020000579D002070B504460D46012C1AD1FFF70A
:100210003BFE01210020F2F7F9FE0121FF20F1F75A
:100220001DFF03200A49087001222946094802F0EF
:1002300063F80848093002F07FF80648123002F0EF
:100240007BF803E014B9034802F076F870BD0000B3
:10025000D10200204E9D002070B504460D46012CB1
:1002600005D101222946044802F046F803E014B9FA
:10027000014802F061F870BDE89E002070B50446A8
:100280000D46012C05D101222946044802F034F81C
:1002900003E014B9014802F04FF870BD729D0020D0
:1002A00070B504460D46012C08D108200649487057
:1002B00001222946054802F01FF803E014B903485B
:1002C00002F03AF870BD0000D1020020609D0020CD
:1002D00070B504460D46012C05D10122294604487B
:1002E00002F00AF803E014B9014802F025F870BDE5
:1002F000F19E002070B504460D46012C05D1012267
:100300002946044801F0F8FF03E014B9014802F05F
:1003100013F870BD699D002070B504460D46012C90
:1003200005D101222946044801F0E6FF03E014B993
:10033000014802F001F870BD1DA4002070B504460C
:100340000D46012C08D104200649087001222946D7
:10035000054801F0D1FF03E014B9034801F0ECFFB8
:1003600070BD0000D102002014A400202DE9F05F30
:1003700005468B464FF0000A63488069634908448C
:1003800050F8046C60488069084450F8087C5E4866
:100390008069084450F80C8C5B488069084450F828
:1003A000149C8814854279D1594A394659A0F9F7E5
:1003B0005FFF574887420DD042F210710120FFF7CE
:1003C00021FF272003F026FA5BA0F9F751FF5046E2
:1003D000BDE8F09F4C48414642695BA0F9F748FFF1
:1003E0004948406940450CD042F210710120FFF7A6
:1003F00009FF252003F00EFA5CA0F9F739FF5046FB
:10040000E6E741488069A0F1140249465BA0F9F78C
:100410002FFF3D48816909F1140081420CD042F25E
:1004200010710120FFF7EEFE262003F0F3F95DA026
:10043000F9F71EFF5046CBE701214020F6F78EFE6C
:10044000F1F780FD30488069001F81082F48F1F7DF
:1004500061FDF1F771FD044600214020F6F77EFEB4
:100460002246314653A0F9F703FFB4420DD042F2C1
:1004700010710120FFF7C6FE242003F0CBF954A031
:10048000F9F7F6FE5046A3E708E057A0F9F7F0FEAB
:10049000282003F0BFF94FF0010A33E040F60410C2
:1004A00085422FD101214020F6F758FEF1F74AFD91
:1004B00015488069001F81081448F1F72BFDF1F7FA
:1004C0003BFD044600214020F6F748FE2246314617
:1004D00038A0F9F7CDFEB4420CD042F210710120E1
:1004E000FFF790FE242003F095F939A0F9F7C0FE3C
:1004F00050466DE73CA0F9F7BBFE282003F08AF9CF
:100500004FF0010A504663E7F49B00200000060804
:10051000574A4257726561645F66697863686172C1
:100520003A253038782C20666978636861723A25FC
:100530003038780A000000006669784368617220EC
:100540006572726F720D0A00726561645F66696C34
:10055000657665723A253038782C20757064617440
:10056000655F7665723A253038780A0066696C6591
:10057000566572206572726F720D0A007265616451
:100580005F66696C656C656E3A253038782C20742E
:100590006F74616C5F62797465733A253038780ADC
:1005A0000000000066696C656C656E206572726F94
:1005B000720D0A00726561645F6372633A25782C7C
:1005C000206765745F6372633A25780A0000000053
:1005D0007570646174652066696C65206372632060
:1005E0006572726F720D0A00CAD5B0FCD5FDC8B72E
:1005F0000A00000030B5E1B024AC0025802101A83C
:10060000EFF7C5FE33A0F9F733FE374800882080A6
:1006100035484068C4F8020033480088E08032481A
:100620004068A0603048008CA081802020824FF478
:10063000967529462DA0F9F71BFE2B48018C2FA09B
:10064000F9F716FE2848408C2749098C884234DC8B
:100650002548428C018C31A0F9F70AFE2248408CD3
:10066000E0812148408C401C1F494884E189491E93
:10067000314A02EBC110802201A9F1F754FF802218
:1006800001A904F11200EFF769FE922241F2040180
:1006900021A8FBF7E9F91448408C1349098C8842DA
:1006A00016DD00202549087043F698210120FFF748
:1006B000D3FD0220214948700AE000201F4908703C
:1006C00043F698210120FFF7C7FD02201B4948701F
:1006D00061B030BD6F74615F7873705F636F6E740B
:1006E000696E7565730D0A007C9D002074696D65E7
:1006F00072203D2025640D0A000000007873705FB1
:1007000075706461746520746F74616C5F706B6781
:1007100073203D2025640D0A000000006F74615FA6
:100720007873705F636F6E74696E756573207B2577
:10073000642F25647D0D0A00000006084AA40020ED
:1007400030B5E1B0054624AC802101A8EFF71FFECB
:10075000A98917A0F9F78CFD1A480088208019484C
:100760004068C4F8020017480088E08015484068D7
:10077000A0601448008CA08180202082A889E0819C
:10078000A989491E104A02EBC110802201A9F1F784
:10079000CAFE802201A904F11200EFF7DFFD9222C8
:1007A00041F2050121A8FBF75FF961B030BD0000FF
:1007B00072657065617420706B672069643A2564A6
:1007C0000A0000007C9D00200000060810B51E48AD
:1007D0000078002837D01C48801D01F053FD78B305
:1007E0001948407810B101282BD11FE001224FF4A5
:1007F000FA611548801D01F07FFD00F027F81248CE
:100800008078401C104988700846807805280CDBE9
:1008100000208870012048700020888001224FF459
:1008200096710948801D01F067FD0BE001224FF42D
:1008300096710548801D01F05FFDFFF7DBFE01E0CA
:1008400001E000BF00BF10BD4AA4002030B5C1B018
:10085000002504AC16480088641C24F8010C1448D8
:100860004068C4F8010012480088A4F80500104848
:100870004068C4F807000320E0720D484069E0605A
:100880000B48806920618020A0823220E0824FF4F2
:10089000967020832169641E2A4606A0F9F7E8FCB9
:1008A0001B2241F2030101A8FBF7DEF841B030BD85
:1008B0007C9D0020746F74616C5F62797465732035
:1008C0003D2025642C2073656E6420696E7465720A
:1008D00076616C203D2025640A00000010B50446B6
:1008E0000321012000F0F2FF802010494877042105
:1008F0000F48F1F7BBFF78B90C48407F40F010007B
:100900000A494877012C02D10220F1F72FFD00217E
:10091000FF20FDF77FFF07E0802004494877012C86
:1009200002D10120F1F722FD10BD0000EC060020ED
:100930000010014010B545480078142826DD4348D2
:10094000807818BB01204149887001F1160001F040
:10095000F3FC01224EF660213C48001D01F0CCFC66
:100960000121042000F0B2FF39A0F9F781FC3B48D7
:100970000068401C3949086008224FF47F50F0F7A6
:10098000C5FE3648016836A0F9F772FC2F4840785A
:10099000142826DD2D48C07818BB01202B49C870CB
:1009A00001F11F0001F0C8FC01224EF6602127482A
:1009B0000D3001F0A1FC0221042000F087FF2CA0E3
:1009C000F9F756FC25484068401C24494860082235
:1009D0004FF47F50F0F79AFE2048416827A0F9F7BE
:1009E00047FC1A48807870B11848001D01F04AFC95
:1009F00048B10020154908708870012000F0BAF84D
:100A000022A0F9F735FC1148C07870B10F480D30BD
:100A100001F038FC48B100200C494870C870022031
:100A200000F0A8F81EA0F9F723FC0848163001F0E2
:100A300029FC10B100200549087004481F3001F05E
:100A400021FC10B100200149487010BD343600204F
:100A5000706F7331206F6E0A00000000C00100202B
:100A6000706F7331206E756D3A25640A00000000C6
:100A7000706F7332206F6E0A00000000706F733267
:100A8000206E756D3A25640A000000007468697371
:100A900020697320706F7331206F66660A00000052
:100AA0007468697320697320706F7332206F666693
:100AB0000A0000001FB501212020F6F76FFB01217D
:100AC0002548F1F78BFE03208DF80E0048208DF8A5
:100AD0000F000320ADF80C0003A92048F1F7F2FD48
:100AE00001210846F6F75AFB00210320F1F7CAFD61
:100AF00001210320F1F7C6FD0320019000208DF8AD
:100B000008000C208DF8090001208DF80A0001A8CA
:100B1000F1F7E2FB06208DF8000002208DF80100BD
:100B200000208DF8020001208DF803006846F2F7DE
:100B300079FA07208DF8000002208DF801000120CD
:100B40008DF802008DF803006846F2F76BFA032077
:100B5000F1F7A8FB1FBD00000002300000140140A7
:100B600010B5FFF7A7FF28210148EFF710FC10BDD3
:100B70003436002010B504462146012000F0A6FEC0
:100B800010BD000010B5F2F721F8FDF7CBF9FDF725
:100B9000BFF9F7F799FE00F0B7FC03490860FBF7CF
:100BA0009DF9FBF77FF810BDD40100200FB438B5D4
:100BB00004463CB106A8009000990598F9F796FB09
:100BC0000020009038BC5DF814FB0000F8B5054625
:100BD0000F462E4606F10C04A168E088FBF762F987
:100BE00000283ED0D4F80E000090A3893289F17914
:100BF0001CA0F9F73DFBFFF73BF827482968016087
:100C000069684160A9688160208823498881D4F897
:100C10000200C1F80E00D4F80E10A089FBF742F9CB
:100C200020B100F043F8FFF723F81AE0A08940F65E
:100C30000411884215D10220174981F820000122B1
:100C40004FF47A71154801F057FB134991F82000D1
:100C50003A46294602F032FC3A46294610A0FAF7F5
:100C600083FFF8BD66697273743A253032782C734D
:100C700065636F6E643A253034782C206465735F49
:100C8000747970653A253034782C6465735F736EBF
:100C90003A25750A0000000028A400200C8C0020D2
:100CA0007873702073656E640000000010B5C2B0E8
:100CB00005AC1148808920800F48D0F80E00C4F898
:100CC00002000E48B0F80500E0800C48D0F80100A2
:100CD000A0600020E06003202074112042F2070190
:100CE000CDE900100448C379D0F80320817802A828
:100CF000FDF70AF842B010BD28A40020DC06002051
:100D000010B501220021224801F018FC2149088079
:100D10000846008818B3084600881F4908801C4907
:100D20001D4A128888183222002101F007FC194957
:100D30000880084600881849098808441549088031
:100D400008460178124801F097FC14480078012801
:100D500005D1012212491148401C01F0CDFA0F487B
:100D6000401C01F08FFA90B100200C490870FAF78E
:100D70008BFF0C480078012803D100200A498877AE
:100D800002E003200849887708A0F9F771FA10BD3E
:100D9000F88700204C0200204E02002028990020F5
:100DA000C0270900DC060020EC0600207074206FCC
:100DB00066660A0070B504464FF4A0710848EFF764
:100DC000E6FA21460648EFF712FB0548EFF708FB65
:100DD00005462A460249002002F070FB70BD000063
:100DE000729A002070B5002438E0002532E004EB50
:100DF00084011C4A02EB411105EB850201EB021153
:100E000001F13D0001F05CFA10B3012229462046B1
:100E1000FCF7F2FF064604EB8400124901EB401098
:100E200005EB850100EB011090F83900B04204D0C9
:100E30001EB12946204600F0B3F904EB84000949AD
:100E400001EB401005EB850100EB011080F83960E3
:100E5000681CC5B2022DCADB601CC4B2022CC4DB04
:100E600070BD0000389300202DE9F04786B004469D
:100E70000D4617460026B046B146B24604EB840044
:100E8000B94901EB401005EB850100EB011040680A
:100E900000287DD004EB8400B34901EB401005EB42
:100EA000850100EB0110D0F804A0002004EB8401C0
:100EB000AD4A02EB411105EB850201EB02114860DE
:100EC00004EB8400A84901EB401005EB850100EB21
:100ED0000110C06850BBA54800EB041050F8350065
:100EE00004EB8401A04A02EB411105EB850201EB02
:100EF0000211C8609D4800EB041050F8350004EB67
:100F00008401994A02EB411105EB850201EB0211C4
:100F10004861012004EB8401934A02EB411105EB87
:100F2000850201EB021181F8200011E004EB84013D
:100F30008D4A02EB411105EB850201EB0211097AA2
:100F4000481CC11700EB11710911A0EB0111CEB2C1
:100F5000864800EB041050F8350000F10108834882
:100F600000EB041000EBC500406800EB0A0904EB3D
:100F700004107F4901EB401005EB051100EB011057
:100F800006EB06110844C0F8008004EB041000E0F2
:100F9000ACE0774901EB401005EB051100EB0110C7
:100FA00006EB06110844077104EB0410704901EBCD
:100FB000401005EB051100EB011006EB061108448B
:100FC000C0F805A004EB0410694901EB401005EBE3
:100FD000051100EB011006EB06110844C0F809905A
:100FE000644800EBC40050F8250004EB0411604A8B
:100FF00002EB411105EB051201EB021106EB0612A3
:101000001144C1F80D0004EB8400574901EB401076
:1010100005EB850100EB01100672544800EB04104B
:1010200040F83580514800EB041000EBC500C0F8D3
:101030000490012004EB84014B4A02EB411105EBC3
:10104000850201EB0211087004EB0410484901EB22
:10105000401005EB051100EB011006EB06110844EA
:10106000D0F80D0004EB0411414A02EB411105EBED
:10107000051201EB021106EB06121144D1F809101A
:1010800004EB04123A4B03EB421205EB051302EB9F
:10109000031206EB06131A44D2F8052004EB0413DE
:1010A000DFF8CCC00CEB431305EB051C03EB0C1372
:1010B00006EB061C63441B79CDE90232CDE904102E
:1010C00004EB04102A4901EB401005EB051100EB7D
:1010D000011006EB0611084400686B1C621C2649CF
:1010E000CDE900600120FFF761FD3AE0012F38D122
:1010F000224800EB441000EB051080681F4901EB0B
:10110000441101EB05114968401A40F6B831884294
:1011100003D81BA0F9F7ACF823E004EB84001249D4
:1011200001EB401005EB850100EB0110406A401C0B
:1011300004EB84010C4A02EB411105EB850201EB43
:1011400002114862012004EB8401074A02EB4111BD
:1011500005EB850201EB021181F828000CA0F9F7DC
:1011600087F806B0BDE8F087389300207894002017
:1011700098940020D8980020003F0308E8980020A9
:1011800067756E2074696D652073686F72740A00EC
:1011900067756E2074696D65206C6F6E670A00005C
:1011A00070B504460D4604EB8400344901EB401051
:1011B00005EB850100EB01104068401C04EB840145
:1011C0002E4A02EB411105EB850201EB021148604A
:1011D00004EB8400294901EB401005EB850100EB8D
:1011E00001104078E0B9012104EB8400234A02EBAE
:1011F000401005EB850200EB021080F82E1004EB86
:1012000084011E4A02EB411105EB850201EB02113C
:1012100001F14600012241F2883101F06DF82CE025
:1012200004EB8400154901EB401005EB850100EB50
:10123000011090F82E00012810D104EB84010F4A10
:1012400002EB411105EB850201EB021101F14600B1
:10125000012241F2883101F04FF80EE004EB8401E5
:10126000064A02EB411105EB850201EB021101F187
:1012700046000122024901F03FF870BD389300207A
:10128000E093040010B504461448447114480472F5
:10129000562000F071FF022C0ED11248C07810B910
:1012A00004200E4948700F48C07808B9012000E0BA
:1012B00000200C49C8700FE0032C0DD109480079BB
:1012C00010B90420054948700648007908B9012082
:1012D00000E000200349087110BD0000E0A60020D6
:1012E000F88B002050020020F0B5044600250BB119
:1012F000022B7DD104EB8400814E06EB401001EB04
:10130000810600EB0610C06804EB84067C4F07EBF7
:10131000461601EB810706EB07167669B0420CD141
:1013200004EB8400764E06EB401001EB810600EBE7
:101330000610007C1070002571E004EB8400704EF4
:1013400006EB401001EB810600EB0610C06804EBD1
:1013500084066B4F07EB461601EB810706EB071679
:101360007669801B10282AD904EB8406644F07EBAA
:10137000461601EB810706EB0716367A701CC61776
:1013800000EB16763611A0EB0616167004EB8400FF
:101390005B4E06EB401001EB810600EB061090F867
:1013A000200030B3002004EB8406554F07EB4616AF
:1013B00001EB810706EB071686F820002EE004EB10
:1013C00084004F4E06EB401001EB810600EB061047
:1013D00090F8200080B1002004EB8406484F07EB12
:1013E000461601EB810706EB071686F8200001E0A0
:1013F00039E013E0107011E004EB8406404F07EB76
:10140000461601EB810706EB0716367C701CC617E3
:1014100000EB16763611A0EB061616700125107833
:1014200004EB8406364F07EB461601EB810706EB0B
:101430000716307404EB0410324E06EB401001EB3B
:10144000011600EB0610167806EB0616304400680D
:1014500004EB84062A4F07EB461601EB810706EBE7
:10146000071670614AE0012B01D0032B46D104EB33
:101470008400234E06EB401001EB810600EB0610C2
:10148000C06804EB84061E4F07EB461601EB81078C
:1014900006EB07167669B04201D1002500E0012570
:1014A00004EB8400164E06EB401001EB810600EBC6
:1014B0000610007A1070107804EB8406104F07EBCA
:1014C000461601EB810706EB0716307404EB041097
:1014D0000C4E06EB401001EB011600EB06101678DF
:1014E00006EB06163044006804EB8406044F07EB55
:1014F000461601EB810706EB071670612846F0BD22
:10150000389300209894002070B5002400250448EA
:10151000446AA40E2546F5F761FE284670BD00001A
:1015200000100240EFF7EEBC10B50F48807F022894
:101530000BD00D48807F01280FD10C48007803287C
:101540000BD00A480078042807D009480078012801
:1015500009D10020FAF7DCFB05E00548007810B956
:101560000120FAF7D5FB10BDEC060020D1020020C7
:101570001400002070B5014600200A46D5434FF400
:101580007F4606EA0524D3B244EA030070BD00009A
:1015900010B500210846FEF7BFFE00210846FEF701
:1015A000CDFE0B480078012803D100200949887737
:1015B00002E00320074988771C210748EEF7E7FE81
:1015C0000648002101600171F9F70AFF10BD000013
:1015D000DC060020EC0600200CA40020D102002034
:1015E00008B5032010237822164900902020F1F737
:1015F0002DF8022048230122134900901020F1F712
:1016000025F80220102302460F4900901846F1F7F2
:101610001DF808210C48F1F732F902204823042272
:10162000094900901020F1F711F802201023082238
:10163000054900901846F1F709F808210248F1F72A
:1016400020F908BD00140140001001402DE9F041CF
:1016500006460C4617463546142F62DDEEF710FE9F
:1016600000686178405C20281CD1012085F8350095
:101670006078302806D0312805D0322807D03328AA
:101680000AD105E000BF012085F8340009E000BF61
:10169000022085F8340004E06078303885F83400A2
:1016A00000BF1FE0EEF7ECFD00686178405C00F0E1
:1016B0009800B8B1022085F835006078412807DB32
:1016C00060785A2804DC6078403885F8340009E0F6
:1016D0006078612806DB60787A2803DC60786038FF
:1016E00085F8340054F8011F05F29110C5F89111E6
:1016F0006168C5F895112189A5F89911D4F80A10E7
:101700000A30C5F89B11D4F80E10C5F89F11618AF4
:10171000641EA5F8A3110A2205F2911102A0FAF79E
:1017200023FA0020BDE8F0817461785F7365726907
:101730006E6F0000F0B504460D461746264606F2C9
:101740008D112846F9F764FE0020F0BD2DE9F04721
:1017500006460F46904634467D1C4FF00009B8F10E
:101760000B0F02DA0120BDE8F087EEF789FD006873
:101770002978405C20281CD1012084F83500287885
:10178000302806D0312805D0322807D033280AD196
:1017900005E000BF012084F8340009E000BF02200A
:1017A00084F8340004E02878303884F8340000BF2E
:1017B00025E0EEF765FD00682978405C00F09800B0
:1017C000C0B1022084F835002878412807DB28784A
:1017D0005A2804DC2878403884F834000FE0287850
:1017E00061280CDB28787A2809DC2878603884F8AE
:1017F000340004E0012084F8350084F8340094F8C3
:101800003400082802DD082084F834000A2221462A
:101810002846F9F77BFA286844F8050F6868606085
:1018200028892081641F0F22214602A0FAF79CF923
:10183000484698E7383320736572696E6F00000080
:101840002DE9FC5F064689469246344609F10105BA
:101850004FF0000BBAF11A0F02DA0120BDE8FC9F2D
:101860000020287605F10C00EEF7FCFE6060A16018
:10187000002028732846EEF7F5FEE0602161E0685D
:101880002169CDE900016768A3683A4603A0F8F72B
:10189000EFFC012084F820005846DFE70D0A207491
:1018A0006F74616C5F7072696E63203D20256C6C93
:1018B000642C20746F74616C5F766F6C756D65203D
:1018C0003D20256C6C64200D0A00000070B50546B3
:1018D0000C46012D04D0022D2BD0042D7BD151E0DC
:1018E000012C08D120213D48F0F7C9FF08213B48D1
:1018F000F0F7C7FF1CE0022C08D140213748F0F771
:10190000BEFF10213548F0F7BCFF11E0032C0FD1CA
:1019100020213248F0F7B3FF08213048F0F7B1FF3B
:1019200040212E48F0F7ABFF10212C48F0F7A9FF1B
:1019300051E0012C08D120212848F0F7A2FF08210E
:101940002648F0F79EFF1CE0022C08D140212348D6
:10195000F0F797FF10212148F0F793FF11E0032CD7
:101960000FD120211D48F0F78CFF08211B48F0F70C
:1019700088FF40211948F0F784FF10211748F0F73D
:1019800080FF28E0012C08D120211448F0F777FFD0
:1019900008211248F0F773FF1CE0022C08D1402107
:1019A0000E48F0F76CFF10210C48F0F768FF11E0CB
:1019B000032C0FD120210948F0F761FF402107488F
:1019C000F0F75DFF08210548F0F759FF10210348A3
:1019D000F0F755FF00BF00BF70BD000000140140CC
:1019E00030B591B09648007800286AD09448807845
:1019F0000028FAD0F0F7A8FF04466CB3914800F035
:101A00009BFC8F488079562817D18F480078022890
:101A10000AD1F9F7C1FF00208B490870FEF720F9C1
:101A200000F092FB11B030BD02208749087000F031
:101A30008BFB0420FFF726FCF4E7814880795728C8
:101A400005D100231A4606216720FBF747FDFEF764
:101A500007F900F079FBE5E77C48007880B37B4824
:101A60008078A0422ED0774800F066FC74488079D8
:101A7000562816D174480078022809D1F9F78CFF4E
:101A8000002071490870FEF7EBF800F05DFBC9E734
:101A900002206D49087000F057FB0420FFF7F2FBAD
:101AA000C0E767488079572805D100231A460621E8
:101AB0006720FBF713FDFEF7D3F800F045FBB1E715
:101AC00000E0BAE000205E498870084640780528AA
:101AD0007DD2DFE800F00326496C8C0001AB0022C8
:101AE0001146722000F0ECFA0546554948792A461D
:101AF00001A901F0E3FC01224FF47A71514800F092
:101B0000FBFB4F494879012100F0E5F84C48417949
:101B10004FA0F8F7ADFB2A4601A951A0FAF724F827
:101B20008AE001AB04225149732000F0C9FA05464E
:101B3000434948792A4601A901F0C0FC01224FF42B
:101B40007A71404800F0D8FB3D494879012100F006
:101B5000C2F83B4841793EA0F8F78AFB2A4601A922
:101B60003FA0FAF701F867E001AB002211467020B0
:101B700000F0A6FA0546324948792A4601A901F043
:101B80009DFC01224FF47A712E4800F0B5FB2C49E0
:101B90004879012100F09FF8294841792CA0F8F7F5
:101BA00067FB2A4601A92EA0F9F7DEFF44E024498D
:101BB000CA794879083101F081FC01224FF47A7129
:101BC000204800F099FB1E494879012100E030E0EF
:101BD00000F081F81A4841791DA0F8F749FB184830
:101BE000C27900F108011EA0F9F7BEFF24E001AAA6
:101BF0000121862000F020FA0546114948792A463D
